:020000040802F0
:1000000040EC0020A90102083DAC02089D9E0208B8
:1000100061AA020835180208B503030800000000B1
:10002000000000000000000000000000B9C202084B
:10003000F31C020800000000A9B1020881DA0208DE
:10004000C3010208C3010208C3010208C301020878
:10005000C3010208C30102085D420208734202089C
:10006000C3010208C3010208C3010208C301020858
:10007000C3010208C3010208C3010208C301020848
:10008000791B0208891B0208C30102080000000056
:100090000000000000000000000000007D42020897
:1000A000C3010208C3010208C3010208C301020818
:1000B000C301020891DD0208C3010208C30102085E
:1000C000C3010208C3010208C3010208C3010208F8
:1000D000C30102088DF402089DF40208000000002C
:1000E00067420208C3010208C301020800000000C1
:1000F000000000000000000000000000C301020832
:1001000000000000C3010208C3010208C301020885
:1001100000000000000000000000000000000000DF
:10012000991B0208A91B0208B91B0208C301020897
:10013000C3010208000000000000000000000000F1
:10014000000000000000000000000000C3010208E1
:10015000C3010208C91B0208D91B0208ADF402083A
:10016000C3010208C30102080000000000000000F3
:10017000000000000000000000000000000000007F
:1001800000000000C30102080000000000000000A1
:10019000C3010208DFF80CD000F04AFC0048004719
:1001A000F51B030840EC002006488047064800473E
:1001B000FEE7FEE7FEE7FEE7FEE7FEE7FEE7FEE717
:1001C000FEE7FEE771DB0208950102082DE9F05F0A
:1001D0000546002092469B468846064681464024B6
:1001E0001BE0284641464746224600F020F8534689
:1001F0005A46C01A914110D311461846224600F0C3
:10020000C3FA2D1A67EB01084F4622460120002150
:1002100000F0BAFA17EB00094E41201EA4F10104C8
:10022000DFDC484631462A464346BDE8F09F202A97
:1002300004DB203A21FA02F00021704721FA02F390
:10024000D040C2F12002914008431946704740EA6D
:1002500001039B0703D009E008C9121F08C0042A44
:10026000FAD203E011F8013B00F8013B521EF9D22B
:100270007047D2B201E000F8012B491EFBD2704753
:100280000022F6E710B513460A4604461946FFF762
:10029000F0FF204610BD421E12F8013F002BFBD19B
:1002A00011F8013B02F8013B002BF9D1704730B542
:1002B00005462A460B4612F8010B13F8014B08B10C
:1002C000A042F8D01CB1002802D06D1CF1E72846EE
:1002D00030BDCAB2401E10F8011F8A4202D0002968
:1002E000F9D100207047421C10F8011B0029FBD1F6
:1002F000801A704710B5002200E0521C835C8C5CB1
:10030000A34201D1002BF8D1D8B2E1B2401A10BDFE
:1003100030B504460020034600E05B1C934203D244
:10032000E05CCD5C401BF8D030BD034611F8012BDA
:1003300000F8012B002AF9D11846704730B5054660
:100340000020034600E05B1C934205D2EC5CC85CD5
:10035000201A01D1002CF6D130BD70B5064610F040
:1003600095F9046805460A220021304600F07CFA1F
:100370002C6070BD2DE9FE4F804681EA0300C00F5E
:100380000C46009021F0004123F00045B8EB02003C
:10039000A94105D24046214690461C460B460246DE
:1003A00023F00040104347D0270DC7F30A00C3F3E2
:1003B0000A510290401A019040286BDAC3F31300EF
:1003C00040F4801B0098924620B10023D2EB030A30
:1003D00063EB0B0B01985946C0F14002504600F008
:1003E000D3F906460D4650465946019A00F0DBF90E
:1003F00010EB08006141002487EA115284EAE77398
:100400001A4340D0009A62B3019A012A4FEA075278
:1004100015DC001B61EB02014FF0004202EA0752BB
:10042000CDE90042001C41F5801132462B4600F018
:1004300099FA03B0BDE8F08F40462146F9E7001B6A
:1004400061EB0201001C41F5801300185B4120188C
:10045000A2F5001747EB030140EAD570B6196D41CC
:1004600011E06D084FEA360645EAC0754FEA0752BB
:10047000001B61EB0201001C41F5801149084FEAA5
:1004800030000019514132462B4603B0BDE8F04F11
:1004900000F059BA0098012240000023D0EB02027C
:1004A00063EBE073009821464FEAE074B8EB00007C
:1004B00061EB0401E9E783F000435BE781F0004171
:1004C00058E72DE9FE4F81EA030404F0004421F0CF
:1004D000004100944FF0000B23F0004350EA010468
:1004E0005ED052EA03045BD0C3F30A54C1F30A5549
:1004F0002C44A4F2F3340194A0FB0254C1F3130181
:1005000041F48011C3F3130343F4801301FB02444D
:1005100000FB034E840A970A44EA815447EA835752
:10052000A4FB076802958D0A05FB07854FEA932C0B
:1005300004FB0C542705029D4FEA065847EA16377C
:10054000B5EB08056EEB070C870E920E47EA811794
:1005500042EA8312A7FB0201B6EB0B0164EB000435
:100560002B0D43EA0C335E1844EB1C50DA4651461F
:10057000E7FB0201C5F313044FEA0B3343EA1453BC
:100580004FEA0432019C43EA0603A4F10C040294EE
:10059000009CCDE900B400F0E5F903B0BDE8F08FB0
:1005A00000200146F9E72DE9F04D81EA030404F04B
:1005B000004B21F0004514464FF0000A23F00041A3
:1005C00050EA050220D054EA01021DD0C5F30A57B3
:1005D0000246C5F31303C1F31300C1F30A5640F4F6
:1005E000801543F48013A7EB0608101BD64608F2CB
:1005F000FD3873EB050002D308F1010801E0921801
:100600005B41B8F1000F03DA00200146BDE8F08D30
:1006100000204FF48011064684460EE0171B73EB52
:10062000050705D3121B63EB050306434CEA010CD7
:1006300049084FEA300092185B4150EA0107EDD1BA
:1006400052EA030012D082EA040083EA050108435B
:1006500005D0101BAB4106D20122002306E0002288
:100660004FF0004302E06FF0010253101AEB060056
:100670004CEB085110EB0A0041EB0B01BDE8F04DCB
:1006800000F061B90EB540F2334102910021CDE98D
:1006900000110A460B4600F065F903B000BD00F0FA
:1006A000004230F000400AD0C10D01F56071C0F386
:1006B000160042EA0151C20840071143704700206A
:1006C0000146704730B5041E71F1000404DB4FF0A1
:1006D0000044404264EB0101141E73F1000405DB89
:1006E0001C464FF00043524263EB04038B4208BFA9
:1006F000824230BD30B5041E71F1000404DB4FF0BE
:100700000044404264EB0101141E73F1000405DB58
:100710001C464FF00043524263EB0403994208BF6A
:10072000904230BD01F0004330B421F0004150EA66
:10073000010206D00A0DA2F56072C1F31301002A6E
:1007400002DC30BC00207047440F44EAC104C10001
:10075000E01830BC00EBC25000F0BEB830B50B461C
:10076000014600202022012409E021FA02F59D42E1
:1007700005D303FA02F5491B04FA02F52844151EB5
:10078000A2F10102F1DC30BD202A04DB203A00FA9C
:1007900002F1002070479140C2F1200320FA03F3D8
:1007A000194390407047202A06DBCB17203A41FAC4
:1007B00002F043EAE07306E041FA02F3D040C2F1EE
:1007C0002002914008431946704700000FB40023EF
:1007D00000B589B00CA900910B996FF00042CB6075
:1007E0001E4B06931E4B07930423CDE901321D4A8D
:1007F000089202466B46002000F0CEF909B05DF881
:1008000014FB70B586B006464FF0FF300091CDE97D
:100810000101002015460C4604903246694604A8A2
:10082000FFF7D4FF02460498211825B108B1084605
:1008300000E020462860049800280DD0002A02DD40
:100840000098884208D0081B0094CDE90104324684
:10085000694604A8FFF7BAFF06B070BDD10D0208C3
:10086000EF0D02085D0A02082DE9F04791460F4698
:1008700080460446002614F8015B2DB100F0EAF82A
:100880000068405DC007F6D12B2D02D02D2D18D069
:10089000641E4A463946204600F0BAFA27B1396844
:1008A000A14201D1C7F8008071054FF002040BD5B9
:1008B0004042002803DD0FF0E9FE0460A007BDE818
:1008C000F08746F48066E4E70028F8DA0FF0DEFEF1
:1008D00004606FF00040F2E70029A8BF7047401C99
:1008E000490008BF20F00100704710B4B0FA80FC46
:1008F00000FA0CF050EA010404BF10BC704749B183
:10090000CCF1200421FA04F411FA0CF118BF0121F2
:1009100021430843A3EB0C01CB1D4FEA00614FEAD2
:10092000102042BF002010BC704700EBC3501044A1
:100930000029A4BF10BC7047401C490008BF20F02C
:10094000010010BC704710B5141E73F1000408DAE2
:10095000401C41F1000192185B411A4301D120F083
:10096000010010BD2DE9F04D92469B4611B1B1FA40
:1009700081F202E0B0FA80F220329046FFF704FFE5
:1009800004460F4640EA0A0041EA0B0153465A4624
:10099000084313D0114653EA010019D0C8F14002B0
:1009A0005046FFF744FC05460E465046594642461F
:1009B000FFF7EAFE084305D0012004E0204639464F
:1009C000BDE8F08D0020054346EAE0762C4337432E
:1009D0000A986305E40AA0EB08000022FD0A44EA35
:1009E00047540A3002D500200146E9E701051019F5
:1009F0006941DDE9084500196941BDE8F04DA2E70C
:100A0000C1F30A52C1F3130140F2FF3341F48011E4
:100A10009A4202DA00200146704740F233439A427C
:100A2000A2F2334202DC5242FFF701BCFFF7ACBE38
:100A3000064C074D06E0E06840F0010394E807002B
:100A400098471034AC42F6D3FFF7A8FB10370308E1
:100A500030370308004870477029030810B5044672
:100A6000FFF7F8FF0068005D00F0010010BD000016
:100A70002DE9FF4F087883B09946FF2805D0491C1F
:100A80002D2804D00024002008E000200BE00124E1
:100A9000F9E700EB800003EB4000491C0B78FF2BCB
:100AA000F7D104B1404200230293147819461D4641
:100AB0002D2C01D02B2C04D1521C2D2C13D0002412
:100AC0000294AA461478FF2C0FD00A25A3FB0578C0
:100AD00001FB05814FF0000C03FB0C11521CE319C4
:100AE0004AEB0101EEE70124EAE7814453EA010001
:100AF00002D019F5C87F06DA03980021C0E9001179
:100B000007B0BDE8F08F0025AE4E2F46DFF8B88263
:100B1000184600F0DAF9CDE90001B9F1000002DA77
:100B2000C9F1000400E004460023A74A1AEB030BB6
:100B300042EB045A12E0E00707D02A463346384613
:100B40004146FFF7BEFC074688462A463346104614
:100B50001946FFF7B6FC05460E466410002CEAD194
:100B6000DDE90001B9F1000F5A46534606DAFFF7F6
:100B70001AFD3A464346FFF716FD05E0FFF7A1FCD4
:100B80003A464346FFF79DFC029A0AB181F00041C4
:100B9000039AC2E90001B3E72DE9FF4F1F468DB06C
:100BA000D7E901464FF0FF382E2045464FF00009A7
:100BB0000B90B9696D1C0E988847396A8246884740
:100BC0000028F6D1BAF1FF3F0AD024F4D064002EF9
:100BD00011DDBAF12B0F08D0BAF12D0F0BD102E0C5
:100BE000404611B08DE744F48064B9696D1C0E98DD
:100BF00088478246761E6946600501D52D2000E0B3
:100C00002B208DF8000001F1010B0DF1200809E007
:100C1000B9696D1C0E98884782460F9844F4007499
:100C2000761E0560002E02DDBAF1300FF0D00B9970
:100C30008A453ED144F0800406E00F99681CA9F172
:100C4000010944F400740860B9696D1C761E0E98A1
:100C5000884782463028F0D02BE00B998A4505D191
:100C6000200603D444F08004761E18E050460FF0AE
:100C7000E1FE08B30DF11301761E44F400748B45B8
:100C800008D2AAF130000BF8010B200607D5A9F114
:100C9000010003E0200602D409F101008146A0050D
:100CA00002D50F99681C0860B9696D1C0E988847B9
:100CB0008246002ED1DC53E0002E51DDBAF1650FE3
:100CC00002D0BAF1450F4BD1A00549D5B9696D1CC9
:100CD00024F44074761E0E9888478246002E0CDD60
:100CE0002B2804D0BAF12D0F07D144F48074B969D0
:100CF0006D1C0E9888478246761EE00501D52D2191
:100D000000E02B2108F8011BCDF82C8021E00DF12B
:100D10002901761E44F4007488450CD2AAF13000F3
:100D200010F0FF0088F8000002D10B99884509D91E
:100D300008F1010806E0E00501D5244801E042F28F
:100D40000F708146B9696D1C0E98884782460F98CE
:100D50000560002E04DD50460FF06CFE0028D6D151
:100D6000F9690E988847FF208BF8000088F800008A
:100D70000020069007904B466A4608A906A8FFF790
:100D800077FEA00502D46FF001002AE714F0240FCB
:100D90000AD0E00714D1DDE906123868031D3B6074
:100DA0000068C0E900120BE0DDE90601FFF7BAFCBC
:100DB0000146E00704D13868021D3A60006801600E
:100DC00028460EE7000014400000F03FF1D8FFFF76
:100DD000426842B1016811F8013B23B1521EC0E9DB
:100DE0000012184670470121C160881E7047426892
:100DF0005AB1C368016843B983688B4205D0491E64
:100E0000521CC0E90012002070474FF0FF307047BD
:100E10002DE9F05F82460078002715468B460AF1DF
:100E20000104B946302801D09DB113E014F8010B3C
:100E30000127782803D0582801D045B10AE00DB128
:100E4000102D07D10027102514F8010B02E008250A
:100E500000E00A250026B0460EE005FB080005FB71
:100E600006F1012701EB10461FFA80F8B6F5803F26
:100E700000D3B94614F8010B294600F018F80028F1
:100E8000EBDABBF1000F05D00FB1641E00E0544651
:100E9000CBF80040B9F1000F06D00FF0F7FB0221AC
:100EA0000160C81EBDE8F09F48EA0640FAE73A280C
:100EB00000D2303820F02002412A01D3A2F13700BD
:100EC000884201D34FF0FF3070470EB540F23342F5
:100ED00002920022CDE900221346FFF743FD03B042
:100EE00000BD70B58C1810F8015B15F0070301D137
:100EF00010F8013B2A1106D110F8012B03E010F87D
:100F0000016B01F8016B5B1EF9D12B0705D400239F
:100F1000521E0DD401F8013BFAE710F8013BCB1A41
:100F2000921C03E013F8015B01F8015B521EF9D536
:100F3000A142D8D3002070BD70B50546AC6B206CC3
:100F400000F0500050BB206C40F40070206420681A
:100F5000806800F04050E8B9A069D8B92068C06A3C
:100F600000F4700020B12068806800F4806088B9C7
:100F70002068406820F0200021684860206C20F440
:100F800080702064206C00F4805018B9206C40F010
:100F900001002064204604F0F1F803E0A06BC16C6E
:100FA0002846884770BD70B50546AC6B402020646C
:100FB000606C40F004006064204604F0E1F870BD0D
:100FC00070B50446A56B284604F0D9F870BD000042
:100FD000014600220023022901DB00207047002285
:100FE00006E0064800EB820030F811000344521C72
:100FF000642AF6D36420B3FBF0F0EFE75CDA00205C
:1010000010B5C82202490348006804F04DF910BD2C
:101010005CDA00204006002054494A6822F440323D
:101020004A604A6843681A434A600268526822F478
:10103000807203685A6002685368026943EA0222B8
:1010400003685A600268526822F0407203685A606E
:101050000268526883681A4303685A60026892689B
:1010600022F4006203689A6002689268C3681A43B7
:1010700003689A603E4B826A9A4218D0026892686E
:1010800022F0706203689A6002689268836A1A4369
:1010900003689A600268926822F0405203689A607E
:1010A00002689268C36A1A4303689A600BE0026898
:1010B000926822F0706203689A600268926822F077
:1010C000405203689A600268926822F00202036844
:1010D0009A6002689368826943EA420203689A60F0
:1010E000026AA2B10268526842F4006203685A6060
:1010F0000268526822F4604203685A6002685368CA
:10110000426A521E43EA423203685A6005E00268AE
:10111000526822F4006203685A600268D26A22F4BC
:1011200070020368DA620268D36A828B521E43EA55
:1011300002520368DA620268926822F4007203685D
:101140009A6002689368026B43EA422203689A60DD
:101150000268926822F4806203689A600268936869
:10116000426943EA822203689A6070470023014083
:101170000100000F01490860704700004006002090
:1011800010B500200E49088000F008FC09F074F842
:1011900008F0E4F906F07EFF09F078F803F082FC2D
:1011A0000EF086F80748B0F85600012801D10CF07F
:1011B00053FD0AF023F809F0F9FF0FF0DBF910BD39
:1011C0001E000020E81F002008B500200AF08CFD5A
:1011D00010F0D6FE0AF01AFA00F0A8FB0BF022FB82
:1011E000FFF70EFF00F054F809F02CF81248B0F8A1
:1011F0005600012802D10CF01DFD08E00E48B0F8A1
:101200005600022803D109F005FE09F019FD03F08C
:1012100083FA0EF03FF810F0AFFF084808F068F9C5
:101220000020074B4FF47A720121009003480068B8
:1012300008F0EAF908BD0000E81F002000000020C7
:1012400045B1020810B5FFF79BFF0E4800780E4924
:10125000097888420ED00C4800780A490870084680
:10126000007810B10EF054F904E00020074908603E
:1012700010F01AF90348007808B110F09BFF08F04D
:10128000A3FF10BD2E0000202D00002064060020CA
:1012900010B5012010F07BFD0D490870084600785C
:1012A000132802D110F0ACFD10E00A4809F03AF81A
:1012B000084800780649087008460078332802D1AB
:1012C00008F0FEFF02E000200349C88710BD0000BF
:1012D0005406002055060020E81F002038B50021E4
:1012E0000F2010F03FFA834908600021824810F077
:1012F000D3FA8048008800F48040002871D04FF471
:10130000804200210F2010F0C8FB0021102010F0B7
:1013100029FA7A490870084600787949087000224D
:1013200076480178774810F071FA77487549B1F836
:101330000110018075487349B1F8051001807148AA
:1013400000787349097888427ED16E48407A202817
:10135000FAD16C48C0786F4908706A4800796E49C4
:1013600008706848807A6D49087068486549B1F826
:101370000510018069480078420062490B316848D5
:10138000FEF765FF65480078420064480078400039
:101390000B305C4BC1186348FEF759FF5F4800787B
:1013A0000B2101EB8000574901445F480988018007
:1013B00000205E49088002205D490870002013E08B
:1013C000574931F810105B4A126891420AD15549C9
:1013D00031F8102058498989114409B2574A1180BF
:1013E00006E074E0411CC8B24C4909788842E7DB4A
:1013F00000BF4648008800F05DFA5149088049481E
:1014000030F91400401C60B10846007841B24B48E6
:10141000B0F9000000F06EFC4A49494A128841F8D0
:1014200022004748008848490988884214D1464824
:10143000008843490880354802884348018800886D
:10144000401C414B188000E040E0404820F811204B
:1014500001203F49087002E000203D4908702F48F4
:1014600000783C49097888420BDD2C4800783949DE
:1014700008702A480078420022490B313648FEF7AE
:10148000E6FE002414E00B2000EB44001D49084454
:1014900000880090BDF8000026490968884205D1FF
:1014A00000202E490870204600F05CF8601CC4B291
:1014B0001A4800788442E6DB1848007884420BD151
:1014C000012026490870204600F04CF804E0244A28
:1014D00000210F2010F0E1FA0FF0FEFF0121064875
:1014E00010F0DAF9002010F01DFA002010F0A2F937
:1014F00038BD00005002002000D023245C020020F0
:101500005D020020603F002064020020660200208F
:10151000D70100206E0200206F020020710200201F
:101520003C45002094470020740200200A0000205F
:101530001A020020CC010020E81F00205C030020DC
:10154000780200209C4E002076020020EC4900200A
:101550005F020020720200208C4000206002002008
:101560000090272410B5044657480470574858493E
:101570000988A0F8011057490988C18156480078A8
:101580005249C871084655490988A0F8051010F05D
:101590001BFB534A03C253480078A0421AD151485A
:1015A000007800EB800040F29E2101EB8000C4EB4C
:1015B000041101EB810100EB01100004C117083A8E
:1015C000D2E90032C0185141000A40EA01604649A0
:1015D000086018E04348007800EB800040F29E214C
:1015E00001EB8000C4EB041101EB810100EB011061
:1015F0000004C1173A4B0CCB80185941000A40EA4D
:101600000160394908603848006810F03DF93549F3
:101610000978491C091BC1EB011101EB81010A2268
:1016200002EB011010F063F92F48006820F0010070
:101630000021090241EA106100022C4A03C2284835
:101640000CC822481A3010F043FD28480CC81F4827
:101650001E3010F03DFD1D482549898941842548EB
:1016600000781A490870244800788874212048724C
:101670000846C574C07C00F00F00C87400223C20EE
:1016800010F057FA00213C2010F066FA012010F00B
:1016900087F91A490870002019490870174800781E
:1016A00080B904E016480078052800DD09E0002133
:1016B0000F2010F057F81349086000F08000002850
:1016C000F0D000BF10BD00006B020020F63F0020EC
:1016D000CC0100201C000020EA010020660200204E
:1016E00080020020710200205402002040020020ED
:1016F000E81F0020D70100206802002061020020BE
:101700002006002050020020014800887047000099
:10171000A405002010B500F003F8002010BD000063
:1017200010B52648FFF726FD254900200AF054FD94
:10173000002108460AF032FC2023224A00210846F4
:101740000AF096FB2023204A032100200AF090FB98
:1017500040231D4A012100200AF08AFB80231A4AF7
:10176000022100200AF084FB184900200EF0A0FBA3
:10177000174901200EF09CFB164902200EF098FB41
:101780004FF480620F49002001F002F901220D4957
:10179000022001F0FDF84FF480520A49012001F0C7
:1017A000F7F840220C49002003F072F94FF4805200
:1017B0000549012003F06CF9002010BD28DC002051
:1017C000D0DC00200004024000000240A0DD002028
:1017D00020DE0020E0DD00200008024010B51148A6
:1017E0000088002802DD01200F4908800E4800888B
:1017F000B8B10C48008800280CDD0A480088401E5B
:10180000084908800120094908700C21084805F0A2
:10181000F7FD06E00020054908700C21044805F09A
:101820000FFE10BD0400002006000020090000206B
:1018300028DD002000BFFEE710B504460021024865
:1018400009F020F910BD000065D3020810B502466A
:101850000B460020002103E0545C0444A0B2491C64
:101860009942F9D3C443A0B210BD00002DE9F04164
:1018700004460D4616460748006838B10648324609
:10188000294603682046034F3F68B8470020BDE85B
:10189000F0810000680500206C05002010B50021D3
:1018A00003480FF0F9FF0FF017FE0FF0FDFD10BD1C
:1018B00000D0232431B500240AE00A4800EB44019B
:1018C00002226846FEF724FD00B905E0601C84B2E0
:1018D000054800888442F0DB00BF0020034908551A
:1018E000204638BDEC49002076020020704D0020D3
:1018F0000EB50021084A0948CDE901210090A0F267
:10190000E220B0F8A01200F2C22300F2A22200F5F9
:10191000207009F01FFA0EBDA9AC0208CA220020EF
:1019200001480078704700008103002000B587B0AF
:101930001C216846FEF7A4FC00208DF8010002205F
:101940008DF800000F4801904FF480700290C000A5
:10195000049040200590694600200EF049F80A489E
:101960000A49C1F890050A48C1F89C050948C1F820
:1019700098050948C1F89405084607F097FC07B098
:1019800000BD00005C650020FB1A0208BC5F00205F
:10199000ED1A0208351B0208491B02081CB5FFF7A7
:1019A000BFFF10B907F0F4FB97E0FFF7B9FF01287C
:1019B0002FD1002001900090694602200EF004F81B
:1019C00020E09DF80400032812D14448006850B17B
:1019D00007F0BEFD41490968401AC8280BD900200C
:1019E00000F0C2F807E007F0B3FD3C49086002E0F0
:1019F00000203A4908604FF47A73012201A9009847
:101A000006F05DF901A900200DF020FF0028D8D0D4
:101A100063E0FFF785FF02282FD10020019000909E
:101A2000694602200DF0D0FF20E09DF80400032855
:101A300015D12B48006868B107F08AFD284909686C
:101A4000401AC8280ED9012026490870002000F04D
:101A50008BF807E007F07CFD2149086002E00020D8
:101A60001F4908609DF804000EF0A6FC01A90020A3
:101A70000DF0ECFE0028D8D02FE0FFF751FF03282F
:101A80002BD100200190002420E09DF804000328C1
:101A900015D11548006868B107F05AFD1249096868
:101AA000401AC8280ED901200E490870002000F005
:101AB0005BF807E007F04CFD0B49086002E00020EE
:101AC000094908609DF804000EF076FC01A9002089
:101AD0000DF0BCFE0028D8D000BF1CBD8403002040
:101AE00088030020820300208C03002010B50446E8
:101AF000214600200DF0AAFE10BD0FB410B5ADF5C3
:101B0000027D85A881904FF4007101A8819B849A81
:101B10000EF0A6FD0020819001A8FEF7E4FB04462C
:101B2000224601A900200EF07DFA0DF5027D10BCC1
:101B30005DF814FB31B500240122694600200EF047
:101B400071FA0446204638BD70B50446002520468B
:101B5000FEF7C9FB06463246214600200EF062FA27
:101B60000546284670BD000001460248017000206D
:101B7000704700008103002010B5024803F07EFC8E
:101B800010BD000020DF002010B5024803F076FCF5
:101B900010BD000080DF002010B5024803F06EFC8D
:101BA00010BD000070DC002010B5024803F066FC98
:101BB00010BD0000E0DF002010B5024803F05EFC1D
:101BC00010BD000060DE002010B5024803F056FC96
:101BD00010BD000040E0002010B5024803F04EFCAC
:101BE00010BD0000C0DE0020014608781038182320
:101BF000B0FBF3F20848805CC865032A05D9086881
:101C00006FF30900001D886503E008686FF30900A1
:101C10008865886D70470000CE28030801460020C3
:101C20008A6A8B69CBB932B1012A0DD0022A03D05E
:101C3000032A10D10EE000BFCB6A03F08073B3F12A
:101C4000807F00D1012007E0CB6AB3F1C07F00D1D3
:101C5000012001E000E000BF34E08B69B3F5005FD4
:101C60001AD132B1012A07D0022A03D0032A11D196
:101C70000AE000BF01200EE0CB6A03F08073B3F1ED
:101C8000807F00D1012006E0CB6AB3F1C07F00D194
:101C9000012000E000BF15E032B1012A05D0022A80
:101CA00004D0032A0CD103E000BF00BF012008E0EC
:101CB000CB6A03F08073B3F1807F00D1012000E094
:101CC00000BF00BF704730B50468246824F4802446
:101CD00005682C60046863608468402C04D1046843
:101CE000A2600468E16003E00468A1600468E26047
:101CF00030BD70470246104B33F91130D01A00281E
:101D000001DB034600E04342B3F57A7F03DB0B4B74
:101D10005B5C032B06DD0020084B5854064820F876
:101D2000112004E00548405C401C044B5854024814
:101D300030F9110070470000C45B0020D655002028
:101D400001201A4948720220194948720320194992
:101D500048720420184948721448184909780170DB
:101D6000144816490978017011481449097801701E
:101D70000E4813490988A0F805100E481049098833
:101D8000A0F805100A480E490988A0F801100A4871
:101D90000B490988A0F801100A4809490988A0F8E8
:101DA000011007490988A0F8051070478409002030
:101DB000E2090020A609002098090020D701002090
:101DC000CC010020F809002010B509F0C1FE382030
:101DD0000BF048FE01200FF0A7FB08200BF042FE9D
:101DE0000FF0DCFC0F4908600F48007818B10F486D
:101DF0000FF020FA02E00E480FF01CFA01210D4806
:101E00000FF04AFD48F283000FF083FD00200FF031
:101E1000BFFD4FF47A700FF085FD00200FF00AFD32
:101E200010BD0000C4000020770100204400002005
:101E30003900002000D023242DE9F04391B007465B
:101E40000D4614463C22934902A8FEF700FAD7F843
:101E50000880D8F83400D0F800902846362D73D08A
:101E600013DC04283FD007DCC0B1012832D002289F
:101E700037D0032869D135E00E2867D00F2867D006
:101E8000152876D03528F5D1C6E0373808285CD239
:101E9000DFE800F0C4C5C6C7C8C9CACB00207E4968
:101EA00008607E4908607C48006800EB400002AB97
:101EB00053F820207848006800EB400003EB8000D6
:101EC0004168404606F02EF874480068401C73498B
:101ED0000860DBE0404606F047F8484607F0F2FAB3
:101EE000D4E000BF00BF042D37D16B48006800EB81
:101EF000400002A901EB8000007A00F0040030B33A
:101F000000206649086064480068401C6249086017
:101F100008460068052805D300226149384606F0C6
:101F200031FC10E05C48006800EB400002AB53F865
:101F300020205948006800EB400003EB8000416816
:101F4000404605F0EFFFA1E067E09DE052E000E0D1
:101F50008EE0012011B0BDE8F0834F48006800EB2F
:101F6000400002A901EB80008068022D02D101210E
:101F700001E06EE00221084018B3002047490860E4
:101F800045480068401C4449086008460068052828
:101F900005D300224249384606F0F4FB29E03E48CA
:101FA000006800EB400002AB53F820203A4800687C
:101FB00000EB400003EB80004168404605F0B2FFB3
:101FC00017E036480068401C34490860084600683D
:101FD000032805D300223349384606F0D3FB08E036
:101FE0000E203B4642F2107200210090484606F057
:101FF000ADFB4BE02848006800EB400002AB53F813
:1020000020202548006800EB400003EB8000416879
:10201000404605F087FF39E000BF00BF00BF00BFAA
:1020200000BF00BF00BF00BF00BF26461A480068BF
:1020300010B101280AD104E0D6E9000108F0A4FD9E
:1020400005E0D6E9000108F0B7FD00E000BF00BFE1
:102050001CE026466B4614A2D6E9000107F00AFCF4
:10206000012800D012E0DDE9000108F07BFD0DE061
:10207000002008F017FD012805D100220D490E4867
:1020800006F080FB02E001E0012063E700BF0020D2
:1020900060E70000942703080C05002010050020CD
:1020A00034270308D42603082B434349443A202508
:1020B000700D0A00C4260308F4BA00202DE9F84385
:1020C00004460D469046A668706B0768032D78D0CD
:1020D00005DC5DB1012D23D0022D6FD127E0042D49
:1020E00070D00E2D6CD00F2DF7D1B3E04FF46120DE
:1020F000614908600846016801200DF0FDFD0020DF
:102100005E4908705E4908605E4908600E202346FB
:102110004FF47A7200210090384606F017FBA8E0D1
:10212000304605F021FF384607F0CCF9A1E05348CE
:102130000078012812D14FF461204F490860084609
:10214000016801200DF0D8FD0E2023464FF47A726D
:1021500000210090384606F0F9FA8AE0002049494B
:10216000086047480068401C454908600846006808
:10217000032818D340480068B0F5E13F09D1012099
:102180003E49087040A241F28831304605F0CAFE4F
:1021900012E00321002008F099FC00223F4920466C
:1021A00006F0F0FA08E00E2023464FF47A72002180
:1021B0000090384606F0CAFA5BE002E056E001E023
:1021C00033E056E02F480068401C2E49086000208C
:1021D0002B4908602B480068052812D14FF4E130E4
:1021E000254908600846016801200DF085FD0E2094
:1021F00023464FF47A7200210090384606F0A6FA82
:1022000012E0204800680A2805D900222449204607
:1022100006F0B8FA08E00E2023464FF47A72002147
:102220000090384606F092FA23E01448007801281E
:1022300009D10321002008F049FC0022174920465B
:1022400006F0A0FA15E017A241F28831304605F0F9
:1022500069FE0EE0002008F025FC012805D10022CF
:102260001249134806F08EFA03E002E00120BDE8AF
:10227000F88300BF0020FAE70005002004050020D5
:10228000F8040020FC04002041542B4950523D39F1
:1022900032313630303B26570D0A00000427030840
:1022A000D4260308415445300D0A0000C426030813
:1022B000F4BA00202DE9F04105460E461446AF68F9
:1022C00036B1012E16D0022E18D0032E1ED116E0E4
:1022D000A046FFF719FA104908801049D8F8040001
:1022E00008600D4803880EA241F28831384605F097
:1022F00019FE0EE0384605F037FE0AE000BF002266
:1023000006480168284606F03DFA02E00120BDE8D3
:10231000F08100BF0020FAE7AC0500201006002085
:1023200041542B434C564C3D25750D0A00000000CE
:102330002DE9F84305460E461446AF6836B1012E26
:102340001ED0022E20D0032E26D11EE0A046012052
:10235000144908701449D8F804000860134800684C
:10236000006800901148006811A241F2883143686A
:10237000384605F0D7FD0D4800680BF0BFFE0EE0B3
:10238000384605F0F1FD0AE000BF0022064801686A
:10239000284606F0F7F902E00120BDE8F88300BF07
:1023A0000020FAE7AA05002014060020B40500204A
:1023B00041542B514C544F4E453D312C252E2A7300
:1023C0000D0A00002DE9F04105460E461446AF689F
:1023D00036B1012E14D0022E1BD0032E21D119E0CC
:1023E000A0461349D8F80400086012A241F28831CF
:1023F000384605F097FD4FF480201249086013E03D
:1024000000201149087011490870384605F0ACFDEC
:102410000AE000BF002206480168284606F0B2F92B
:1024200002E00120BDE8F08100BF0020FAE70000D3
:102430001806002041542B514C544F4E453D300D51
:102440000A000000180C0240AA050020AB0500207D
:102450002DE9F84305460E461446AF6836B1012E05
:102460001ED0022E20D0032E26D11EE0A046012031
:10247000144908701449D8F804000860134800682B
:10248000006800901148006811A241F28831436849
:10249000384605F047FD0D4800680BF083FE0EE05E
:1024A000384605F061FD0AE000BF002206480168D9
:1024B000284606F067F902E00120BDE8F88300BF76
:1024C0000020FAE7A805002008060020B00500203B
:1024D00041542B515454533D322C22252E2A732221
:1024E0000D0A00002DE9F04105460E461446AF687E
:1024F00036B1012E14D0022E1BD0032E21D119E0AB
:10250000A0461349D8F80400086012A241F28831AD
:10251000384605F007FD4FF480201149086013E0AC
:1025200000201049087010490870384605F01CFD5D
:102530000AE000BF002206480168284606F022F99A
:1025400002E00120BDE8F08100BF0020FAE70000B2
:102550000C06002041542B515454533D300D0A00B9
:10256000180C0240A8050020A905002010B504465B
:10257000FFF7CAF81D490988884204D0204600F0B8
:1025800043F8002010BD1A48007858B90BF0C6FD7A
:10259000184908600846006868B1204600F086F8CF
:1025A0000020EFE714480078012804D1204600F00D
:1025B00093F80020E6E71148007858B90BF064FD65
:1025C0000F4908600846006868B1204600F03AF8F4
:1025D0000020D7E70B480078012804D1204600F0FE
:1025E00047F80020CEE74FF0FF30CBE7AC050020E6
:1025F000A8050020B0050020A9050020AA0500209C
:10260000B4050020AB0500201CB504460020009056
:10261000E06B40680190E06B4068406804494860A6
:10262000002088606A46E06B06F0ACF800201CBD14
:10263000D8050020012002490870002070470000E2
:10264000AB0500201CB5044600200090E06B4068FC
:102650000190E06B40684068044948600020886051
:102660006A46E06B06F08EF800201CBDE8050020ED
:102670001CB5044600200090E06B40680190E06BC0
:102680004068406804494860002088606A46E06B02
:1026900006F078F800201CBDF80500200120024952
:1026A0000870002070470000A90500201CB50446F2
:1026B00000200090E06B40680190E06B406840684B
:1026C00004494860002088606A46E06B06F05AF8CA
:1026D00000201CBDB80500201CB504460020009059
:1026E000E06B40680190E06B4068406804494860D6
:1026F000002088606A46E06B06F044F800201CBDAC
:10270000C80500202DE9F84305460E461446D5F8C5
:102710000880022E18D003DC3EB1012E2CD10FE030
:10272000032E12D00A2E27D116E0274615497868C5
:10273000086015A241F28831404605F0F3FB1EE027
:10274000404605F011FC1AE000BF00220D48016868
:10275000284606F017F812E00020009027466B4646
:102760000CA2D7E9000107F085F8022800D006E0A6
:10277000009808F04DFA02E00120BDE8F88300BFA0
:102780000020FAE77804002041542B4353510D0AEE
:10279000000000002B4353513A2025642C252A0DBC
:1027A0000A0000001CB5044600200090E06B406861
:1027B0000190E06B406840680449486000208860F0
:1027C0006A46E06B05F0DEFF00201CBD68040020B7
:1027D00010B5044608F014FA012802D12046FFF78C
:1027E000E1FF4FF0FF3010BD2DE9F04104460D46EA
:1027F0001746A66835B1012D0BD0022D0DD0032D43
:1028000016D10BE00DA241F28831304605F08AFB6B
:1028100011E0304605F0A8FB0DE000BF022108469C
:1028200008F054F900220849204605F0ABFF02E009
:102830000120BDE8F08100BF0020FAE741542B439E
:1028400046554E3D300D0A00242703087FB5E0B001
:1028500005460E46144622464FF4C0716846639BF7
:102860000DF0FEFE684605F0DBFD002064B070BD93
:1028700000B595B000208DF8390002208DF83800A1
:1028800025480F904FF420601090244811900420A8
:102890001290102013900EA901200DF0A9F818B184
:1028A0004FF0FF3015B000BD1D4806F021FE10B1FD
:1028B0004FF0FF30F6E71B4803901B480490382088
:1028C00005901A4806901A4807901A4808901A4826
:1028D00009904FF4C0600A9018480B904FF4C06004
:1028E0000C900F480D9003A9154805F069FB10B135
:1028F0004FF0FF30D6E701201149124B12A2CDE96B
:1029000000101349074805F0DFFE1249054805F09D
:1029100015FF0020C6E700005CA400207C04002016
:1029200080040020F4BA0020E8230308293D0208AF
:10293000093F0208A13D02085CAE00205CB4002003
:102940005CBA0020A8250308454336303053000008
:10295000A42603084D28020810B50548006928B1CF
:10296000034A918A1069012203F000FA002010BD89
:10297000DCBA002010B50548006928B1034A918AE5
:102980001069002203F0F2F9002010BDDCBA00202B
:102990000346044840F8331000EBC3008280002057
:1029A00070470000DCBA002010B50548006828B167
:1029B000034A91881068002203F0D8F9002010BD66
:1029C000DCBA002010B50548006828B1034A918898
:1029D0001068012203F0CAF9002010BDDCBA002003
:1029E0002DE9F04105460E461446D5F8088036B16B
:1029F000012E0ED0022E10D0092E26D11DE000206F
:102A00001549086015A241F28831404605F08AFA5E
:102A10001EE0404605F0A8FA1AE00F4800680128B9
:102A200005D100221049284605F0ACFE04E0002242
:102A30000E49284605F0A6FE0AE02746064B0CA2E2
:102A4000D7E9000106F016FF02E00120BDE8F081A1
:102A500000BF0020FAE700003005002041542B435E
:102A6000474154543F0D0A007427030834270308D4
:102A70002B43474154543A20256400002DE9F0438C
:102A800093B005460C469146002720210BA8FDF780
:102A9000F7FBAE68706BD0F8008024228D4902A845
:102AA000FDF7D5FB07F0E6FF074605228AA1384669
:102AB000FDF744FC28B1052289A13846FDF73EFC0C
:102AC00028B989A220210BA806F0C7FF22E0052221
:102AD00087A13846FDF732FC28B987A220210BA830
:102AE00006F0BBFF16E0052285A13846FDF726FC5F
:102AF00028B97DA220210BA806F0AFFF0AE005222D
:102B000081A13846FDF71AFC20B981A220210BA82B
:102B100006F0A3FF032C31D005DC5CB1012C25D0DD
:102B2000022C7DD129E0042C29D00E2C79D00F2C39
:102B3000F7D1C8E0002078490860784908607648F5
:102B4000006800EB400002AB53F820207248006898
:102B500000EB400003EB80004168304605F0E2F9ED
:102B60006E480068401C6D490860AFE0304605F0D3
:102B7000FBF9404606F0A6FCA8E000BF00BF042C0D
:102B800033D16548006800EB400002A901EB8000EA
:102B9000007A00F0040020B30020604908605E481D
:102BA0000068401C5C49086008460068032805D39B
:102BB00000225B49284605F0E5FD11E05648006813
:102BC00000EB400002AB53F820205348006800EBB4
:102BD000400003EB80000BAB4168304605F0A2F9E2
:102BE00074E0012013B0BDE8F083022C0AD14A48FA
:102BF000006800EB400002A901EB8000007A00F0C1
:102C0000010060B9032C32D14348006800EB40005A
:102C100002A901EB8000007A00F0020038B301E065
:102C200052E03DE000203D4908603B480068401C00
:102C30003949086008460068032805D3002238494E
:102C4000284605F09FFD2AE03348006800EB40006D
:102C500002AB53F820203048006800EB400003EB43
:102C600080000BAB4168304605F05CF917E02B485B
:102C70000068401C2949086008460068032805D3FD
:102C800000222849284605F07DFD08E00E202B464D
:102C900042F2107200210090404605F057FD15E009
:102CA0001D48006800EB400002AB53F820201A4892
:102CB000006800EB400003EB80000BAB416830463E
:102CC00005F030F902E001E001208BE700BF0020B1
:102CD00088E70000D0270308343630303000000089
:102CE0003436303032000000434D4E455400000071
:102CF0003436303031000000554E494E4554000006
:102D000034363030360000003436303033000000C6
:102D100043544E4554000000280500202C05002097
:102D200064270308A42603082DE9F04104460D4654
:102D30001746A66825B1012D03D00F2D15D101E04E
:102D400016E015E00C480078012808D100200A4957
:102D5000087000220949204605F014FD08E03046BD
:102D600001F06CF800B903E002E00120BDE8F08159
:102D700000BF0020FAE70000980400203427030871
:102D8000F8B507460D4614460F2D0FD005DC4DB1A2
:102D9000012D08D0042D24D109E01A2D0DD0272DA6
:102DA0001FD11AE01FE00AF091FB1CE01BE000229B
:102DB0000E49384605F0E6FC15E026460020009056
:102DC0006B460BA2D6E9000106F054FD012800D0A5
:102DD00009E000980AF09EFC05E001200A4908700D
:102DE00001E00120F8BD00BF0020FBE7B426030886
:102DF0002B51495552433A2022636C6F736564220C
:102E00002C25640D0A000000980400202DE9F041F3
:102E100004460D461746A66825B1012D03D00F2D97
:102E200006D101E007E006E0304600F0E3FF02E0F3
:102E30000120BDE8F08100BF0020FAE770B505462B
:102E40000C46164624B1012C03D0042C08D101E015
:102E500008E007E000220549284605F093FC01E060
:102E6000012070BD00BF0020FBE70000B42603086E
:102E70002DE9F04104460D461746A66835B1012DEF
:102E80000BD0022D0DD0032D16D10BE00DA241F277
:102E90008831304605F046F811E0304605F064F818
:102EA0000DE000BF0321022007F010FE00220849B8
:102EB000204605F067FC02E00120BDE8F08100BF7C
:102EC0000020FAE741542B4346554E3D310D0A0090
:102ED0003427030870B505460C46164624B1012C6C
:102EE00009D00F2C1CD107E0FFF75EFD0221002066
:102EF00007F0ECFD16E015E0002007F0D3FD0128F7
:102F000003D10221002007F0E1FD002007F0D4FDED
:102F1000012804D100220549284605F033FC01E0D0
:102F2000012070BD00BF0020FBE70000D42603088D
:102F30002DE9F84305460E469046AC68606B07687D
:102F400026B1012E1AD00E2E60D11BE00020E062C7
:102F500000BF2046216988470028FAD00020E0629F
:102F60002D490870FFF720FD0E202B4640F6B832A1
:102F700000210090384605F0E9FB4AE0384606F0AB
:102F8000A1FA46E02448007830B1012813D0022885
:102F900025D0032838D131E001201F490870FFF700
:102FA00011FD0E202B464FF47A7200210090384616
:102FB00005F0CCFB28E0022017490870FFF7CCFC95
:102FC0004FF4612101200CF097FE0E202B464FF4A8
:102FD0007A7200210090384605F0B8FB14E0032017
:102FE0000D490870FFF7C6FC0E202B464FF44872BF
:102FF00000210090384605F0A9FB05E000220749B2
:10300000284605F0BFFB00BF00BF02E00120BDE87D
:10301000F88300BF0020FAE7DC040020E426030860
:10302000F8B507460D461446142D13D005DC4DB1F6
:10303000012D08D0042D31D106E0332D1AD0342DC6
:103040002CD121E02CE02BE000221749384605F076
:1030500099FB25E02646002000906B4613A2D6E996
:10306000000106F007FC012800D019E000980AF0E2
:103070002BFB15E0264612A13068FDF73BF900B1A5
:103080000EE0FFF70BFB0BE0264610A13068FDF7C2
:1030900031F900B104E0FFF7CDFA01E00120F8BDFD
:1030A00000BF0020FBE70000B42603082B51495560
:1030B00052433A202272656376222C256400000078
:1030C0002B515454533A20300D0A00002B514C54CC
:1030D0004F4E453A20300D0A00000000034611B162
:1030E000012902D100E002E001E00120704700BFA9
:1030F0000020FBE72DE9F04105460C461646AF6877
:10310000052C1FD2DFE804F0030E1213140007F0A1
:10311000B5FC804643460EA241F28831384604F0A1
:1031200001FF12E0384604F01FFF0EE000BF00BFB1
:10313000304607F013FD084800224168284605F094
:1031400021FB02E00120BDE8F08100BF0020FAE78A
:1031500025730D0A00000000A00400202DE9F843AB
:1031600004460E461546A768786BD0F80090072EE7
:1031700074D005DC5EB1012E1AD0022E6FD11EE094
:10318000082E6DD00E2E6CD00F2EF7D1C5E000208A
:103190006849087068490860684908600120684902
:1031A000087068A241F28831384604F0BBFEBEE0E8
:1031B000384604F0D9FE484606F084F9B7E05D4889
:1031C0000078A8BB00205E4908705C4800680128B0
:1031D00003D05A480068052811D1012055490870CC
:1031E000002055490860554908600120544908707D
:1031F00057A241F28831384604F094FE4EE04E4822
:103200000068401C4C49086008460068642805D9DD
:1032100000225249204605F0B5FA88E00E202346E8
:103220004FF4FA6200210090484605F08FFA35E02D
:10323000FFE740480078012830D10020404908705D
:103240003E480068012803D03C480068052809D1A1
:1032500043480068401C424908600BE01FE063E0FF
:103260002BE039E000203E49086033480068401CEC
:10327000314908603A480068032805D300223949DB
:10328000204605F07FFA08E00E2023464FF4FA624C
:1032900000210090484605F059FA00BF47E0A846D3
:1032A0002448007840B9254B2FA2D8E9000106F048
:1032B000E1FA022800D03AE039E0A8461D4800783B
:1032C000012808D11D4B2CA2D8E9000106F0D2FA42
:1032D000022800D02BE02AE01648007860B90020D0
:1032E0001649086001201649087027A241F288316A
:1032F000384604F017FE0FE00E48007801280BD185
:1033000000200E49086001200D49087010A241F20A
:103310008831384604F006FE09E00948007810B903
:10332000384600F067FD02E00120BDE8F88300BFE9
:103330000020FAE7140500201C05002018050020D5
:103340002405002041542B43455245473F0D0A00B8
:1033500041542B43475245473F0D0A00B42603080A
:1033600020050020542703082B43455245473A20A7
:10337000252A2C25640000002B43475245473A205C
:10338000252A2C256400000041542B435245473F19
:103390000D0A00002DE9F04104460D461646A768C7
:1033A00035B1012D0ED0022D11D0032D19D10DE014
:1033B0000F4806600FA243F698210368384604F0D0
:1033C000B1FD11E0384604F0CFFD0DE000BF084824
:1033D00000680AF09FF900220B49204605F0D2F957
:1033E00002E00120BDE8F08100BF0020FAE7000004
:1033F0004005002041542B5149434C4F53453D2536
:10340000642C31300D0A0000742703082DE9FE4FAB
:1034100005460E461446AF68786BD0F80090032E30
:103420003CD005DC4EB1012E30D0022E74D134E0F8
:103430000E2E72D0162EF9D14BE04648046000687B
:103440000AF0F2F88046434800680AF0DBF882464A
:10345000404800680AF018F9012801D13EA000E0B8
:103460003EA08346CDE901A800903A483CA241F233
:1034700088310368384604F055FD0E202B46414A3A
:1034800000210090484605F061F95FE0384604F0FD
:103490006BFD484606F016F858E057E02D480068E6
:1034A0000AF05CF938480068401C37490860084653
:1034B0000068032807D3002008600022334928460B
:1034C00005F060F904E000223149284605F05AF978
:1034D0003CE0A04600200290019001A8009002ABC1
:1034E0002CA2D8E9000106F0C5F9022800D02DE091
:1034F00018480068029988421ED1019870B90020CE
:1035000021490860134800680AF046F90022204962
:10351000284605F037F90FE015E00EE00D48006889
:103520000AF01CF918480068401C1749086000227E
:103530001749284605F026F908E0002214492846D4
:1035400005F020F902E00120BDE8FE8F00BF002059
:10355000FAE700003805002054435000554450005D
:1035600041542B51494F50454E3D312C25642C225E
:103570002573222C222573222C25752C302C300DFE
:103580000A00000020BF02003C050020A42603081A
:10359000742703082B51494F50454E3A2025642C7F
:1035A00025640D0A000000002DE9FC4106460F4687
:1035B0001446D6F80880022F25D003DC3FB1012F36
:1035C00057D10EE0032F10D01B2F52D121E02C48F1
:1035D00004602CA241F288310368404604F0A2FC4A
:1035E0004AE0404604F0C0FC46E0254800680AF086
:1035F0007FF8234800680AF08DF8002226493046FB
:1036000005F0C0F838E000222349304605F0BAF84A
:1036100032E0002001902546009001AB1FA2D5E9C1
:10362000000106F027F9012804D0154800680AF0C7
:103630005FF821E0019820B9114800680AF058F8B5
:103640001AE06B4618A2D5E9000106F013F902282A
:1036500004D00B4800680AF04BF80DE00848DDE99B
:10366000001200680AF044F9054800680AF0CEF834
:1036700002E00120BDE8FC8100BF0020FAE7000065
:103680004405002041542B514952443D25642C31BE
:103690003032340D0A000000742703082B514952C0
:1036A000443A2025640D0A002B514952443A202502
:1036B0002A0D0A25650000002DE9F04385B0054676
:1036C0000E461446AF68786BD0F80090032E50D0A9
:1036D00005DC4EB1012E1CD0022E74D120E00E2E3E
:1036E0007DD0172EF9D153E04548046000204549AC
:1036F000087005F02DFF4449414A126841F8220044
:103700003F4842A241F288310368384604F00AFC7F
:1037100072E0384604F028FC484605F0D3FE6BE022
:103720003848007801280AD100203D49344A1268FF
:10373000885400223B49284605F024F818E005F09B
:1037400007FF39492E4A126851F82210401A3749AA
:10375000884208D32A48006809F0DCFF002030497D
:10376000274A1268885400222E49284605F00AF894
:1037700042E000202A49224A126888542048006802
:1037800009F0C8FF00222749284604F0FBFF33E078
:103790000020049003900290A04602A803A9CDE95E
:1037A000001004AB22A2D8E9000106F063F8032858
:1037B0000BD01348006809F0ADFF002219492846D4
:1037C00004F0E0FF18E013E009E0029818B90120C6
:1037D0000C49087002E000200A4908700CE0084813
:1037E0000AA241F288310368384604F09BFB03E0EB
:1037F000012005B0BDE8F08300BF0020F9E700001C
:10380000500500205405002024BB002041542B51BA
:103810004953454E443D25642C300D0A00000000FC
:10382000340500207427030830BB0020905F01009E
:103830002B514953454E443A2025642C25642C25B0
:10384000640D0A002DE9F84305460E461746D5F8E3
:1038500008800024032E33D005DC5EB1012E27D072
:10386000022E77D12BE0102E34D0182E4AD0192EEC
:103870007BD170E040480760006809F0E5FE04462F
:1038800004B975E0204606F08AF93C49086008460C
:10389000006800B96CE0394800684068009036481C
:1038A00037A241F288310368404604F03BFB5FE0F9
:1038B000002032490860404604F056FB58E057E0CB
:1038C0002D48006809F026FF00223249284604F0FE
:1038D00059FF4DE004F0CEFB012807D1274A1268BA
:1038E0005168264A1268106804F040FE23480068B8
:1038F00043682248006844F620610268404604F0AC
:103900003BFB35E01C48006809F09EFE044604B904
:103910002EE01A480168204606F019F901211E48D8
:10392000154A1268815405F013FE1C49124A1268A8
:1039300041F8220008461049096850F8210018494A
:103940000D4A126841F8220000221249284604F06C
:1039500019FF0DE009E00848006809F0DBFE0022CD
:103960000C49284604F00EFF02E00120BDE8F88370
:1039700000BF0020FAE70000480500204C050020A9
:1039800041542B514953454E443D25642C25750D1A
:103990000A000000742703083405002024BB00201F
:1039A00030BB00202DE9F041044600260025002709
:1039B00005F0CEFD804600BF35E0284609F054FEF4
:1039C00003280BD1042128460AF03AF82A462D494B
:1039D000E06B04F0D7FE0020BDE8F081284609F036
:1039E00043FE042806D12A462749E06B04F0CAFEAC
:1039F0000020F1E7284609F037FE052806D12A46BF
:103A00002049E06B04F0BEFE0020E5E7284609F0FF
:103A10004BFE012806D12A461C49E06B04F0B2FE99
:103A20000020D9E76D1C032DC7DB19480068401C36
:103A3000032190FBF1F201FB120500261DE0284650
:103A400009F012FE062811D1284609F0FDFD0746AF
:103A500067B1384606F0A3F840B10D4805602A4624
:103A60000C49E06B04F08EFE0020B5E7681C0321D2
:103A700090FBF1F201FB1205761C032EDFDB4FF009
:103A8000FF30A9E704280308F427030814280308D3
:103A900058050020242803082DE9F0432DED028B62
:103AA00091B004460D469146A668706B07689FED7D
:103AB000370AB0EE408A042D58D005DC4DB1012DF7
:103AC00011D0022D58D14FE00E2D4ED0322D53D1B2
:103AD00010E00E20234642F210720021009038467A
:103AE00004F034FE4EE0304604F03EFA384605F06D
:103AF000E9FC47E007F034FCBCEEC00A244880ED46
:103B0000000A24488088000B4FF47A7110FB01F002
:103B100020498988C1F3032101EBC10202EB0111A5
:103B200000EB81001B490979C1F3031101EB81010D
:103B300000EB41001749097901F00F0108441649CB
:103B4000086013480368084614A1026802A80CF034
:103B500073FD1949086002A8FCF7C5FB8046414681
:103B600002A80AF0F1FA0DE000BF00BF00221349DD
:103B7000204604F007FE05E0012011B0BDEC028BE9
:103B8000BDE8F08300BF0020F7E700000000000060
:103B9000E4040020E81F0020F0040020C9E8B1B8C8
:103BA000B1E0BAC52564CAA3D3E0B5E7C1BFB0D9B7
:103BB000B7D6D6AE25640000EC040020F426030836
:103BC0002DE9F84304460D469046A668706B0768D9
:103BD000102D6FD2DFE805F008141B252F6E6E6ED6
:103BE0006E6E6E6E5D6E3D61002035490870354920
:103BF000086035A241F28831304604F093F95BE069
:103C0000304604F0B1F9384605F05CFC54E00E2073
:103C1000234640F6B83200210090384604F096FD65
:103C20004AE00E2023464FF47A7200210090384675
:103C300004F08CFD40E022480078012805D10022E4
:103C40002449204604F09EFD02E00120BDE8F883EF
:103C500032E01B480078012805D100221D4920468A
:103C600004F090FD14E0174800680A280BD21548AC
:103C70000068401C1349086013A241F288313046A5
:103C800004F050F904E000221349204604F07AFDC4
:103C900012E001200A4908700EE0002006F002FF41
:103CA000012805D100220D490D4804F06BFD03E009
:103CB00002E0FFE70120C9E700BF0020C6E70000DF
:103CC000050500200805002041542B4350494E3F74
:103CD0000D0A00001427030824270308C42603083C
:103CE000F4BA002010B50446022006F0DBFE0128DD
:103CF00012D100200A490860E06B40684860E06B20
:103D00004068406807494860002088600022E06BF6
:103D100004F038FD002010BD4FF0FF30FBE700003D
:103D2000A0040020BC04002070B505460C462146C6
:103D300001200BF08BFD70BD0648416805E0064888
:103D4000814201D10120704749680029F7D1002044
:103D5000F9E70000F4BA00206427030810B5044610
:103D6000022006F0A9FE012812D100200A490860AD
:103D7000E06B40684860E06B406840680749486015
:103D8000002088600022E06B04F0FCFC002010BDE5
:103D90004FF0FF30FBE70000A0040020CC0400201F
:103DA00070B506460D461446285D68B944B1601EDC
:103DB000285C0A2804D1294606A004F079FB03E018
:103DC000294608A004F074FB2246294601200CF085
:103DD00029F970BD5B41542053656E645D202573E5
:103DE000000000005B41542053656E645D20257324
:103DF0000D0A000010B50446204600F067F808B927
:103E0000002010BD2046FEF7B1FB08B90020F8E7FE
:103E1000204600F003FA08B90020F2E72046FFF739
:103E200061FF08B90020ECE72046FFF797FF08B9CB
:103E30000020E6E74FF0FF30E3E7000070B50546ED
:103E400005F086FB0446284600F040F808B900203B
:103E500070BD2846FEF78AFB08B90020F8E728461F
:103E6000FFF7A0FD08B90020F2E72846FEF7B0FCF6
:103E700008B90020ECE712480068201A42F21071DD
:103E8000884208D90E48046000220E490E4804F00A
:103E900079FC0020DCE7284600F0C0F908B90020D2
:103EA000D6E72846FFF71EFF08B90020D0E72846CE
:103EB000FFF754FF08B90020CAE74FF0FF30C7E70B
:103EC0009C04002084270308F4BA002010B504469F
:103ED000002006F0F1FD012803D10321002006F0A7
:103EE000F5FD002006F0DEFD012806D10022044980
:103EF000044804F047FC002010BD4FF0FF30FBE702
:103F0000C4260308F4BA00207FB5044600200390BD
:103F10002CB1E06818B1606A08B1A06A18B94FF016
:103F2000FF3004B070BD14E103A92046E268904759
:103F300010B14FF0FF30F4E79DF80C10E26A501C0E
:103F4000E062606A81540020E26A616A8854E06A33
:103F500007280CD1072290A0616AFCF7D9F930B983
:103F600001208F49087001F007FF8E490860E06A60
:103F700007280CD107228CA0616AFCF7C9F930B977
:103F800002208749087001F0F7FE86490860E06A60
:103F90000A280CD10A2286A0616AFCF7B9F930B967
:103FA00003207F49087001F0E7FE7E4908607C48E5
:103FB0000078012807D07A480078022803D0784892
:103FC0000078032809D101F0D7FE76490968401A24
:103FD00040F2DC51884200D9C1E0714800780128E4
:103FE0001FD176A1606AFCF762F90546C5B10020D1
:103FF000029002AB72A2E16A606A05F03BFC012804
:1040000000D0ACE0029800B9A9E0606A281A801CD0
:10401000029908446D4908600A206149087000BF90
:1040200097E05F480078022829D164A1606AFCF714
:104030003EF9054615B366480068B0F1FF3F0ED162
:104040000020029002AB63A2E16A606A05F012FCF4
:10405000012800D083E05E490298086000BF5C48F8
:10406000006800B97BE0606A281A801C584909681A
:104070000844564908600A204949087069E04848E0
:104080000078032825D1002002904CA1606AFCF73B
:104090000EF901900198D8B101A8009002AB50A28E
:1040A000E16A606A05F0E6FB052800D057E0606A27
:1040B0000199081A001D02990844444908600A2021
:1040C000374908704149E06A0968884200D146E0F2
:1040D0003FE0334800780A2805D13C49E06A096886
:1040E000884236D13BE09DF80C000D2803D1012019
:1040F00084F830000AE09DF80C000A2806D194F8F4
:104100003000012802D1022084F8300094F83000F9
:10411000022816D1E06A022804D10020E06284F867
:1041200030000EE0002084F830001D4800780A2896
:1041300006D100201A490870E06284F8300000E0DF
:104140000DE0E06A012804D1606A00783E2800D1C1
:1041500005E0D4E90A01401E8142FFF4E5AE00BF4C
:10416000E16A606A05F06CFB012810D1E06A50B189
:10417000E06A401E616A085C0A2804D11FA0616AD7
:1041800004F096F903E021A0616A04F091F900209F
:104190000349087000BFC4E62B514952443A20003D
:1041A0008C04002094040020434F4E4E454354009D
:1041B0002B514D54524543563A2000000D0A000041
:1041C0002B514952443A20256400000090040020FD
:1041D00088040020434F4E4E454354202564000080
:1041E0002B514D54524543563A20252A2C252A2C32
:1041F000252A2C25752C2565000000005B415420E4
:10420000526563765D202573000000005B415420F9
:10421000526563765D2025730D0A000010B50446D3
:1042200006F094FC012812D100200A490860E06BD6
:1042300040684860E06B406840680749486000207B
:1042400088600022E06B04F09DFA002010BD4FF062
:10425000FF30FBE7A0040020AC04002010B50120D3
:1042600001F084FC10BD10B54FF4805001F07EFCCD
:1042700010BD10B5022001F079FC10BD10B54FF44F
:10428000007001F073FC10BD70B586B004460D4699
:10429000002000900190022005900120029020460D
:1042A00006F096F803906119481E06F091F806464C
:1042B000204606F08DF8301A401C0490694601A88B
:1042C00001F0D6FA18B14FF0FF3006B070BD0020F3
:1042D000FBE7000010B5002201B909E0012901D176
:1042E0000A0205E0022901D10A0201E04FF44072FE
:1042F0000E4B1B6823F440730C4C236023461B6851
:104300001343236023461B6823F0F80323602346EE
:104310001B68022444EAC0042343044C2360234660
:104320001B6843F48033236010BD0000103C024042
:104330001C48006800F40070B0B11A48006820F40E
:1043400000701849086000BF0846006840F400602B
:1043500008600846006820F40060086000BF084656
:10436000006840F4007008600E48006800F4806047
:10437000B0B10C48006820F480600A49086000BFB2
:104380000846006840F4805008600846006820F441
:104390008050086000BF0846006840F480600860F4
:1043A00070470000003C02400A4A126822F4407242
:1043B000084B1A601A46126842F004021A601A4644
:1043C00012684FF4803343EA00231A43014B1A600A
:1043D00070470000103C0240074A126822F4407205
:1043E000054B1A601A4612681A601A46126842F0A3
:1043F00001021A6001707047103C024010B5094973
:10440000096821F44071074C21602146096841F494
:10441000407121602146096841F00101216002607C
:10442000436010BD103C0240084A126822F44072FA
:10443000064B1A601A46126842F480721A601A46D5
:10444000126842F001021A6001807047103C02407D
:10445000084A126822F44072064B1A601A46126823
:1044600042F400721A601A46126842F001021A60A1
:1044700001607047103C02402A48006800F01000BC
:1044800040B12948C06940F010002749C861102098
:10449000244908602348006800F0200040B1224809
:1044A000C06940F008002049C86120201D4908600B
:1044B0001C48006800F0400040B11B48C06940F053
:1044C00004001949C8614020164908601548006871
:1044D00000F0800040B11448C06940F00200124969
:1044E000C86180200F4908600E48006800F48070A1
:1044F00048B10D48C06940F001000B49C8614FF454
:104500008070084908600748006800F0020040B168
:104510000548C06940F020000349C86102200149F4
:10452000086070470C3C0240A0E0002070B50446D3
:10453000002500201449C86101F01EFC054609E071
:10454000601C38B124B101F017FC401BA04201D916
:10455000032070BD0D48006800F480300028EFD1C2
:104560000A48006800F0010010B101200749086006
:104570000648006800F4F97018B1FFF77DFF0120CC
:10458000E7E70020E5E70000A0E000200C3C024047
:104590002DE9F84307460D4614460026B046002094
:1045A000009024E0042C0CD24FF0FF300090002645
:1045B00003E0A85D0DF80600761CA642F9D3A046DC
:1045C00003E0286800904FF00408F3200A490860CF
:1045D000002339460220009A01F0A0F918B14FF0EB
:1045E000FF30BDE8F88347444544A4EB0804002CA1
:1045F000D8D10020F5E700000C3C02400FB4F8B51C
:1046000004460D4600261CB9701EF8BC5DF814FB6C
:10461000E06A08B90020F8E709A80090E76A29468F
:104620002046009B089AB847064600200090304676
:10463000EBE7F0B504460D461E4600210027002397
:10464000214600BF10E042F8331002EBC300476080
:1046500002EBC3075B1C6868D1F804C0604502D157
:1046600037600020F0BD49680029ECD1481EF9E709
:104670002DE9F0410546002700264FF6FF7000EABD
:104680001547AEB20848046809E02088B84205D151
:1046900000223146204603F0B1FF02E06469002C9D
:1046A000F3D100BFBDE8F081C80600202DE9F0413C
:1046B00086B006460F464FF000080025002402A8E9
:1046C00004AB12A239460090304605F0D3F8022818
:1046D00003D0601E06B0BDE8F081DDE9020105F0FF
:1046E00060F800F0FF0804980578012403E00498BE
:1046F000005D4540641C0598A042F8D8454502D0AD
:104700004FF0FF30E6E70020E4E700002425702AA0
:1047100025700D0A0000000010B588B000F024FAE2
:1047200000F0D4FB00208DF805008DF8040022482D
:1047300002904FF480600390204804904FF4206072
:1047400005900220069001A90BF052F9B0211C48F7
:1047500005F006F81BA20A211948401C05F07DF956
:104760001749086219A20A2115480B3005F075F99E
:104770001349486217A20A211148153005F06DF956
:104780000F4988620120154908701548B0F8540097
:104790001349B1F8521040EA0124B4F5612F02D850
:1047A000B4F5165F01D24FF4E134214602200BF03C
:1047B000A3FA08B010BD00005C6600205C6A00200F
:1047C0006C74002024474E4747410000244750475F
:1047D00053560000244742475356000092030020DE
:1047E000E81F002030B58FB004460D46282104A8EC
:1047F000FBF746FD29462046FFF758FF18B14FF05A
:10480000FF300FB030BD23482349244A244BCDE963
:104810000021029023A22946204605F02BF80F28FC
:1048200002D04FF0FF30ECE71A490868FBF795FD1E
:10483000284908701849086800210BF035FF264800
:1048400080ED000B1549086800210BF02DFF23486F
:1048500080ED000B0F490868FBF77FFD1D490870CC
:10486000084600781E4908600846006838B10C48C0
:1048700000681C4902680A608088888007E014216B
:104880001848FBF7FDFC174817A1097801700020B4
:10489000B7E700001C040020040400200C040020E2
:1048A0002404002024252A2C25702C25702C252A50
:1048B0002C25702C252A2C25702C252A2C252A2CD9
:1048C000252A2C252A2C252A2C252A2C252A2C255C
:1048D0002A2A000090030020F0030020F8030020A3
:1048E000000400201C7500203000000070B596B058
:1048F00004460D4628210CA8FBF7C2FC0AA808A90B
:1049000006AA04ABCDE9002102903D4A2946204683
:1049100004F0B0FF15281AD13A480088001D394923
:1049200008800498FBF719FD06460698FBF715FD6D
:1049300006440898FBF711FD06440A98FBF70DFDA5
:1049400030443149098808442F49088054E008A8B8
:1049500006A904AB2DA2CDE900102946204604F09B
:1049600089FF112816D127480088C01C25490880D6
:104970000498FBF7F2FC06460698FBF7EEFC0644AB
:104980000898FBF7EAFC30441F49098808441E498F
:10499000088031E006A804AB2AA2294600902046F0
:1049A00004F068FF0D2812D116480088801C1549B4
:1049B00008800498FBF7D1FC06460698FBF7CDFC6F
:1049C00030441149098808440F49088014E004ABB9
:1049D00027A22946204604F04DFF09280CD109489A
:1049E0000088401C074908800498FBF7B6FC06497C
:1049F0000988084404490880002016B070BD0000F2
:104A0000F82A03082E0400202C04002024252A2C38
:104A1000252A2C252A2C252A2C252A2C252A2C250A
:104A20002A2C25702C252A2C252A2C252A2C257069
:104A30002C252A2C252A2C252A2C25702C252A2A9F
:104A40000000000024252A2C252A2C252A2C252A82
:104A50002C252A2C252A2C252A2C25702C252A2C7D
:104A6000252A2C252A2C25702C252A2A0000000016
:104A700024252A2C252A2C252A2C252A2C252A2CAB
:104A8000252A2C252A2C25702C252A2A00000000F6
:104A9000034B43F8301003EBC0039A8070470000CB
:104AA0005C7400200EB500200290019000906946D1
:104AB0000AF08AFF2DE0FCF733FF012803D0FCF752
:104AC0002FFF022806D14FF47A73012201A9009822
:104AD00003F0F5F89DF8040000F09AF89DF8041032
:104AE000194802680068401C174B18601748815429
:104AF00018460068B0F5007F07D3184601681348D0
:104B000006F0C6F800201049086004F021FD1049A5
:104B1000086001A902200AF099FE02900028CAD07C
:104B20000948006870B104F013FD09490968401A8A
:104B3000322807D904480168044806F0A9F8002083
:104B4000014908600EBD00003804002030750020C7
:104B50003C04002010B5034A91899068002201F0BE
:104B600005F910BD5C74002010B5034A9189906866
:104B7000012201F0FBF810BD5C74002010B5044662
:104B80001D480470012C06D0022C0FD0052C18D023
:104B90000A2C2CD120E00E22184902200BF042FAF8
:104BA0001522174902200BF03DFA21E00E2215498B
:104BB00002200BF037FA1522114902200BF032FACD
:104BC00016E00E22104902200BF02CFA15220C4997
:104BD00002200BF027FA0BE00E220C4902200BF00A
:104BE00021FA1522064902200BF01CFA00E000BF52
:104BF00000BF002010BD000091030020B103002081
:104C00009C030020BF030020CD030020DB03002015
:104C100030B589B004469F4AD2E900109268CDE9C8
:104C2000070206919B4A0C3207CA03AB07C3994A95
:104C3000183207CA8DE807009748007830B101287C
:104C400019D0022851D003287DD169E0242C11D13C
:104C50000120914908700020C1F8AC000846D0F846
:104C6000AC10D0F8AC00401C8B4AC2F8AC0002F18A
:104C70002C0044540AE18848D0F8AC10D0F8AC00BD
:104C8000401C854AC2F8AC0002F12C0044542C3878
:104C9000D0F8AC001146096A884225D31046411C61
:104CA000026A2C30FBF734FB18B902207A490870ED
:104CB0001AE0794800F10B01426A2C30FBF728FB1F
:104CC00018B90220744908700EE0734800F115010C
:104CD000826A2C30FBF71CFB18B902206E49087061
:104CE00002E000206C490870D0E06B48D0F8AC10AE
:104CF000D0F8AC00401C684AC2F8AC0002F12C00AD
:104D000044542C38D0F8AC007F2803D3002011463F
:104D10000870BBE00D2C02D103205F490870B5E09C
:104D20005D48D0F8AC10D0F8AC00401C5A4AC2F82C
:104D3000AC0002F12C0044540A2C6FD15748007883
:104D400040B9574800E0A0E0B0F870005549097834
:104D5000884207D0002051490870514991F87000ED
:104D6000FFF70CFF4C4800F11501826A2C30FBF76D
:104D7000CFFA28B94848D0F8AC102C30FFF7B6FD70
:104D80004548411C026A2C30FBF7C2FA00286CD15E
:104D90004148D0F8AC102C30FFF724FD00223E48EB
:104DA000D0F8AC00801E3C492C310A543E480078B3
:104DB00078B100203C4908703C4908603C480368D1
:104DC0003C480268084601683B48006807F0F6FA6C
:104DD0004BE00120344908703848006838490978A8
:104DE00088420DD036480078042808D103A8FBF784
:104DF0007AFA0546294603A809F0A6F900BF00BFC4
:104E00002F48007806281CD2DFE800F003090D1BAC
:104E100012174FF408402549086017E031E0882058
:104E20002249086012E04FF08810204908600DE028
:104E30004FF408001D49086008E022481B4908603B
:104E400004E0204888301949086000BF00BF1848B6
:104E5000036818480268154801681748006807F099
:104E6000ADFA174800781549086004F071FB16493F
:104E70000968401AB0F57A7F03D304F069FB124940
:104E8000086000200449087000E000BF00BF09B0BE
:104E900030BD0000B42303086C740020920300208E
:104EA000E81F002091030020340400206806002041
:104EB000700600206C0600206406002030040020EC
:104EC00090030020008888009403002010B50C4A4D
:104ED00091881068012200F049FF0A2000F0B4FC1C
:104EE000074A91881068002200F040FF0A2000F075
:104EF000ABFC034A91881068012200F037FF10BD17
:104F00005C7400202DE9F04F95B0044688461546A4
:104F100099460020009082462E46CB4600271CB1C1
:104F2000B8F1000F00D025B94FF0FF3015B0BDE843
:104F3000F08F4AE000203870142301AA3B2130464C
:104F400004F0A2FD00900098122838D926A10198FB
:104F5000FBF7D0F900B138E0BAF1000F14D1B24636
:104F600020212046029A04F078FD202104F120003F
:104F7000039A04F072FD0C98FBF7EFF908B10120D9
:104F800000E0002084F8400041460398FBF7B2F9A6
:104F9000A8B920212046029A04F05FFD202104F1E7
:104FA0002000049A04F059FD0C98FBF7D6F908B1DB
:104FB000012000E0002084F840000020B6E7B81C83
:104FC000801BABEB000BBE1C00BF5A4607A130464E
:104FD00004F09DFD071EADD1BAF1000F01D1401EB6
:104FE000A4E70020A2E70000535452000D0A00007D
:104FF00038B502460020009000BF92F83C0001281E
:1050000001D1022038BD012082F83C0000BF0868B1
:10501000092816D91068C0680C780A3C04EB4405CE
:105020000724AC40A0431468E0600C780A3C04EB11
:1050300044048868A0401468E46820431468E06071
:1050400013E0106800690C7804EB44050724AC40B9
:10505000A043146820610C7804EB44048868A040E5
:10506000146824692043146820614868072817D20F
:105070001068406B0C79641E04EB84051F24AC405F
:10508000A04314686063088880B20C79641E04EB46
:105090008404A0401468646B20431468606331E0AA
:1050A00048680D2817D21068006B0C79E41F04EBD8
:1050B00084051F24AC40A04314682063088880B294
:1050C0000C79E41F04EB8404A0401468246B204393
:1050D0001468206316E01068C06A0C790D3C04EB7C
:1050E00084051F24AC40A0431468E062088880B2A5
:1050F0000C790D3C04EB8404A0401468E46A20435E
:105100001468E062194B1A4C1068A04206D1086876
:10511000122803D1586840F480005860144C10687D
:10512000A0421CD10868102802D00868112816D1A6
:10513000586840F400005860086810280FD10D48E6
:1051400000680D4CB0FBF4F000EB800040000090D4
:1051500002E00098401E009000980028F9D100BF9E
:10516000002082F83C0000BF00BF4BE70023014055
:1051700000200140C406002040420F0070477047E5
:105180007047000070B5044600250CB9012070BDC1
:105190001549A06A884200D000BF206C30B90020B9
:1051A000606484F83C00204600F020F8206C00F099
:1051B000100088B9206C20F4885040F00200206470
:1051C0002046FBF729FF00206064206C20F00200DD
:1051D00040F00100206400E0012500BF002084F8B9
:1051E0003C0000BF2846D2E70100000F10B586B092
:1051F00004462149206888423CD100BF002000902D
:105200001E48006840F480701C4908600846006829
:1052100000F48070009000BF00BF022001900320C6
:1052200002900020039001A9154800F0ADFC15483C
:105230001549086000204860002113488160C16062
:105240004FF4806101614900416189008161491128
:10525000C1614FF4403101620021416200F02EFA39
:1052600018B17E2109A00BF0BDF900BF0648A0636C
:10527000846300BF06B010BD0020014044380240E6
:10528000000002401064024070DC00202E2E2F53DC
:1052900072632F73746D3332663478785F68616C33
:1052A0005F6D73702E630000F8B504460D46164618
:1052B0000020009000BF94F83C00012801D102209A
:1052C000F8BD012084F83C0000BF2068806800F031
:1052D0000100A0B92068806840F001002168886062
:1052E0003C4800683C49B0FBF1F000EB4000009006
:1052F00002E00098401E009000980028F9D1206834
:10530000806800F00100002862D0206C40F201614A
:10531000884340F4807020642068406800F4806016
:1053200028B1206C20F4005040F480502064206CA0
:1053300000F4805020B1606C20F00600606401E051
:105340000020606400BF002084F83C0000BF234FB1
:105350002348A16BC8632348A16B08642248A16B52
:10536000C8646FF02200216808602068406840F03F
:105370008060216848602068806840F480702168FF
:105380008860226802F14C0133462A46A06B00F087
:105390000BFA786800F01F0058B92068806800F0A8
:1053A000405028B92068806840F0804021688860BB
:1053B0000EE00E49206888420AD12068806800F01B
:1053C000405028B92068806840F08040216888609B
:1053D000002075E7C406002040420F000023014072
:1053E000390F0208C10F0208A70F02080020014070
:1053F000014691F83500022803D08020486501203D
:105400007047052081F835000868006820F0010029
:105410000A6810600020F3E770B504460CB901205B
:1054200070BD94F83500022800D1F9E720680068C3
:1054300020F00100216808600020216808602168D0
:105440004860216888602168C8602168086121205F
:10545000216848612046FCF7C7FB054694F85C10BC
:105460003F208840A8600020606584F8350000BFB8
:1054700084F8340000BF00BFD2E70000F8B504464E
:10548000002000908C4800684FF41651B0FBF1F7F3
:10549000A56D2E6894F85C1008208840304098B1C3
:1054A0002068006800F0040070B12068006820F0F7
:1054B00004002168086094F85C1008208840A86007
:1054C000606D40F00100606594F85C100120884038
:1054D000304068B12068406900F0800040B194F825
:1054E0005C1001208840A860606D40F0020060659B
:1054F00094F85C1004208840304068B1206800684F
:1055000000F0020040B194F85C1004208840A860CC
:10551000606D40F00400606594F85C1010208840D5
:10552000304078B32068006800F0080050B394F869
:105530005C1010208840A8602068006800F480207B
:1055400080B12068006800F4002028B9206CC8B140
:105550002046216C884715E0A06C98B12046A16CCC
:1055600088470FE02068006800F4807028B9206840
:10557000006820F0080021680860206C10B1204607
:10558000216C884794F85C10202088403040002827
:1055900065D02068006800F0100000285FD094F803
:1055A0005C1020208840A86094F83500052828D198
:1055B0002068006820F016002168086020684069B3
:1055C00020F0800021684861206C08B9A06C28B1E7
:1055D0002068006820F008002168086094F85C10DA
:1055E0003F208840A86000BF002084F8340000BF3E
:1055F000012084F83500206D10B12046216D8847C8
:10560000F8BD2068006800F4802080B12068006840
:1056100000F4002028B9606C10B12046616C884706
:105620001DE0E06BD8B12046E16B884717E02068A9
:10563000006800F4807068B92068006820F01000ED
:105640002168086000BF002084F8340000BF0120FA
:1056500084F83500E06B10B12046E16B8847606D3F
:1056600038B3606D00F00100F0B1052084F835001A
:105670002068006820F001002168086000BF0098E1
:10568000401C0090B84200D905E02068006800F096
:1056900001000028F3D100BF00BF002084F83400CF
:1056A00000BF012084F83500E06C10B12046E16CA9
:1056B000884700BFA4E70000C40600202DE9F041A0
:1056C0000446002500F058FB074614B90120BDE848
:1056D000F081606A00B100BF00BF002084F8340090
:1056E00000BF022084F835002068006820F0010027
:1056F000216808600AE000F03FFBC01B052805D9BF
:1057000020206065032084F83500E0E72068006809
:1057100000F001000028EED120680568214805400E
:10572000D4E901010843E16808432169084361693C
:105730000843A1690843E1690843216A0843054316
:10574000606A042803D1D4E90B01084305432068AB
:1057500005602068456925F00705606A0543606AB1
:1057600004280DD1A06A0543E06A48B12046FCF741
:1057700055FA28B140206065012084F83500A6E77D
:10578000206845612046FCF72FFA064694F85C1025
:105790003F208840B06000206065012084F835001B
:1057A000002094E73F8010F02DE9F04704460D46B5
:1057B00016461F464FF00008D4F8589000BF94F8E2
:1057C0003400012802D10220BDE8F087012084F8CE
:1057D000340000BF94F8350001282BD1022084F852
:1057E0003500002060653B46324629462046FCF7DE
:1057F0006AFA94F85C103F208840C9F808002068D5
:10580000006840F01600216808602068406940F098
:10581000800021684861206C28B12068006840F051
:105820000800216808602068006840F001002168D5
:10583000086006E000BF002084F8340000BF4FF08D
:1058400002084046C0E7000070B5044600F094FA34
:1058500006462546681C10B104480078054400BF80
:1058600000F08AFA801BA842FAD370BDC00600205F
:105870002DE9F04104460E460127002500BF2548CA
:10588000007E012802D10220BDE8F08101202149DB
:10589000087600BF4CF25030FEF748FE0746002F56
:1058A00031D1401E3060206801280FD1207C616812
:1058B000FEF77AFD4CF25030FEF738FE07461648E8
:1058C000006820F00400144908601AE0A56812E09E
:1058D000217C2846FEF7FEFC4CF25030FEF726FEF7
:1058E00007460D48006820F0FA000B4908600FB128
:1058F000356005E06D1CD4E902100844A842E7D8E1
:1059000000BFFEF715FD00BF00200249087600BF6A
:105910003846B9E7A0E00020103C02402DE9F041F4
:1059200006460F4614461D464FF0010800BF1F48AB
:10593000007E012802D10220BDE8F08101201B4930
:10594000087600BF4CF25030FEF7F0FD8046B8F10B
:10595000000F23D126B9E1B23846FEF73DFD12E033
:10596000012E04D1A1B23846FEF75EFD0BE0022EF7
:1059700004D121463846FEF76BFD04E022462B4653
:105980003846FEF73BFD4CF25030FEF7CFFD804627
:105990000748006820F001000549086000BF0020AA
:1059A0000249087600BF4046C6E70000A0E000209C
:1059B000103C024000200949096801F0004159B13A
:1059C0000749064A0C3A1160064911600349096803
:1059D00001F0004101B1012070470000103C02407D
:1059E00023016745AB89EFCDF0B50C4600250022B9
:1059F0000023002181E0012606FA01F504EA0502F0
:105A0000AA4279D106684FEA410C032707FA0CF73E
:105A1000BE430660CF0800F1200656F827604F0706
:105A20004FEAD76C0F2707FA0CF7BE434FEAD10CA9
:105A300000F1200747F82C6086684FEA410C0327E5
:105A400007FA0CF7BE438660476801268E40B743CD
:105A50004760C6684FEA410C032707FA0CF7BE43BC
:105A6000C660284E8F0856F827308E07370F0F264E
:105A7000BE403340244EB04201D1002614E0234EF4
:105A8000B04201D101260FE0214EB04201D10226E1
:105A90000AE0204EB04201D1032605E01E4EB0427E
:105AA00001D1042600E007268F073F0FBE409E422B
:105AB00022D18E07370F0F2606FA07F3114E8F08F3
:105AC00056F827609E430F4F4FEA910C47F82C6021
:105AD000124E36689643114F3E603E1D366896431F
:105AE0003F1D3E603E1D366896433F1D3E603E1D95
:105AF000366896433F1D3E60491C1029FFF47BAF7A
:105B0000F0BD0000083801400000024000040240DF
:105B100000080240000C024000100240003C01401E
:105B200010B50446B4F5805F01D105F03FFB012CB0
:105B300004D19FED0B0A0B4880ED000AB4F5007FFD
:105B400004D10948007808B9FBF7C8FBB4F5007F19
:105B500005D105480078012801D109F005FE10BDE6
:105B6000000000001C0600207701002010B504464C
:105B700004480068204020B1024804602046FFF736
:105B8000CFFF10BD143C0140F8B503460A4600257E
:105B9000002400200021CDE0012606FA01F5166858
:105BA00006EA0504AC4273D15668022E02D056684C
:105BB000122E13D1CF0803F1200656F827004E0706
:105BC000F70E0F26BE40B0434F07FF0E1669BE40CA
:105BD0003043CF0803F1200646F8270018684F002D
:105BE0000326BE40B043167906F003064F00BE40C0
:105BF000304318605668012E08D05668022E05D032
:105C00005668112E02D05668122E13D198684F0094
:105C10000326BE40B0434F00D668BE403043986074
:105C2000586801268E40B0431679C6F300168E40A0
:105C300030435860D8684F000326BE40B0434F0041
:105C40009668BE403043D860566806F08056B6F17C
:105C5000805F6ED100BF00260096384E366846F44D
:105C60008046364F3E603E46366806F480460096D3
:105C700000BF00BF324E8F0856F827008E07370F3F
:105C80000F26BE40B0432F4EB34202D1002615E08E
:105C90004FE02D4EB34201D101260FE02B4EB3420F
:105CA00001D102260AE02A4EB34201D1032605E0C3
:105CB000284EB34201D1042600E007268F073F0F8C
:105CC000BE4030431E4E8F0846F82700224E3068F3
:105CD000A043566806F48036B6F5803F00D12043D5
:105CE0001D4E3060361D3068A043566806F40036FD
:105CF000B6F5003F00D12043174E361D3060361DEB
:105D00003068A043566806F48016B6F5801F00D1AF
:105D10002043114E08363060361D3068A043566867
:105D200006F40016B6F5001F00D120430A4E0C36CB
:105D30003060491C1029FFF42FAFF8BD44380240F1
:105D40000838014000000240000402400008024000
:105D5000000C024000100240003C01400246136962
:105D60000B400BB1012000E0002070470AB18161B7
:105D700001E00B0483617047014800687047000030
:105D8000B80600200348006803490978084401491F
:105D900008607047B8060020C006002010B50D4806
:105DA000006840F400700B4908600846006840F441
:105DB000806008600846006840F480700860032036
:105DC00000F0B6F8002000F007F800F02BF80020F3
:105DD00010BD0000003C024070B504460E4800783B
:105DE0004FF47A71B1FBF0F00C490968B1FBF0F5A2
:105DF000284600F090FF08B1012070BD102C07D29A
:105E000000222146501E00F054F80548046001E0CD
:105E10000120F2E70020F0E7C0060020C4060020C1
:105E2000BC06002010B5032000F082F800221146C5
:105E30006FF00B0000F03DF8002211466FF00A00F1
:105E400000F037F8002211466FF0090000F031F839
:105E500000221146501F00F02CF800221146101F9E
:105E600000F027F800221146901E00F022F80022D0
:105E70001146501E00F01DF810BD000000BF00F0DC
:105E80001F0201219140034A430942F8231000BF39
:105E90007047000080E100E000BF00F01F02012118
:105EA00091404209920002F1E022C2F8001100BFC5
:105EB00070472DE9F05F80460D461646002704F036
:105EC000DDFF074639462A46334601F00700C0F198
:105ED000070ABAF1040F02D94FF0040A01E0C0F139
:105EE000070AD14600F1040ABAF1070F02D24FF0B7
:105EF000000A01E0A0F1030AD4464FF0010A0AFAB1
:105F000009FAAAF1010A0AEA020A0AFA0CFA4FF09F
:105F1000010B0BFA0CFBABF1010B0BEA030B4AEA8A
:105F20000B042146404604F0B1FFBDE8F09F00009D
:105F300000BF00F00702064B19684FF6FF03194037
:105F4000044B0B4343EA0221014B196000BF704729
:105F50000CED00E00000FA050D4A126822F0030281
:105F600002430B4B1A600B4A126842F00402094BC1
:105F70001A60012901D130BF02E040BF20BF20BF1D
:105F8000044A126822F00402024B1A6070470000B3
:105F90000070004010ED00E070B504460D460CB9ED
:105FA000012070BD5848006800F00F00A84209D2D7
:105FB00055490D700846006800F00F00A84201D056
:105FC0000120EEE7207800F0020002281DD12078A1
:105FD00000F00400042805D14C48006840F4E0506B
:105FE0004A490860207800F00800082805D1474891
:105FF000006840F46040454908604448006820F06B
:10600000F000A168084341490860207800F00100D1
:10601000A8B36068012807D13C4808380068C0F37D
:106020004040B8B90120BCE76068022802D060682F
:10603000032807D1354808380068C0F3406048B9E4
:106040000120AEE7314808380068C0F3400008B9C5
:106050000120A6E72D48006820F00300616808438E
:106060002A490860FFF788FE064609E0FFF784FE2C
:10607000801B41F28831884202D9032091E707E072
:106080002248006800F00C006168B0EB810FEDD190
:106090001D48006800F00F00A84209D91A490D7088
:1060A0000846006800F00F00A84201D0012078E700
:1060B000207800F00400042807D11448006820F478
:1060C000E050E168084311490860207800F00800BA
:1060D000082808D10D48006820F46040216940EA92
:1060E000C1000A49086000F03DF808490968C1F399
:1060F0000311074A515CC840064908600020FFF7B9
:106100006BFE00204DE70000003C024008380240D2
:10611000D6280308C4060020014800687047000024
:10612000C406002000B5FFF7F7FF04490968C1F372
:106130008221034A515CC84000BD0000083802407B
:10614000E628030800B5FFF7E7FF04490968C1F333
:106150004231034A515CC84000BD0000083802408B
:10616000E62803082DE9F047002400250026A14673
:106170002548006800F00C0020B1042805D008284C
:106180003AD105E0DFF8849039E0DFF8849036E01A
:106190001D48001F006800F03F041B48001F0068F6
:1061A00000F4800078B11A481749091F0968C1F343
:1061B0008811A0FB01700146224600233846FAF7F9
:1061C00005F805460EE011480F49091F0968C1F39B
:1061D0008811A0FB01700146224600233846F9F7DA
:1061E000F5FF05460848001F0068C0F30140401C49
:1061F0004600B5FBF6F902E0DFF8109000BF00BFE3
:106200004846BDE8F0870000083802400024F4004A
:1062100000127A00F8B504460CB90120F8BD2078C8
:1062200000F00100002874D0F948006800F00C006C
:1062300004280DD0F648006800F00C00082813D19F
:10624000F348001F006800F48000B0F5800F0BD108
:10625000EF4808380068C0F34040002859D0606813
:10626000002856D10120D9E700BF6068B0F5803F13
:1062700008D1E7480838006840F48030E44908391C
:1062800008601EE06068B0F5A02F0DD1E048083826
:10629000006840F48020DE4908390860084600683C
:1062A00040F4803008600CE0D9480838006820F4D9
:1062B0008030D749083908600846006820F48020FB
:1062C000086000BF606890B1FFF756FD054606E024
:1062D000FFF752FD401B642801D903209EE7CC48FC
:1062E00008380068C0F340400028F1D011E0FFF703
:1062F00043FD054606E0FFF73FFD401B642801D93A
:1063000003208BE7C24808380068C0F340400028EB
:10631000F1D1207800F0020002285FD1BC4800686B
:1063200000F00C0058B1BA48006800F00C000828D2
:106330001CD1B748001F006800F48000B0B9B44811
:1063400008380068C0F3400020B1E068012801D09F
:10635000012063E7AE480838006820F0F8002169A2
:1063600040EAC100AA490839086037E0E06800B394
:106370000120A8490860FFF7FFFC054606E0FFF78B
:10638000FBFC401B022801D9032047E7A04808383E
:106390000068C0F340000028F1D09D48083800682C
:1063A00020F0F800216940EAC100994908390860E5
:1063B00014E0002097490860FFF7DEFC054606E080
:1063C000FFF7DAFC401B022801D9032026E790489A
:1063D00008380068C0F340000028F1D1207800F0B0
:1063E000080008282CD16069A8B101208A490860FA
:1063F000FFF7C2FC054606E0FFF7BEFC401B022883
:1064000001D903200AE782486C300068C0F34000DD
:106410000028F1D014E000207F490860FFF7ACFCB1
:10642000054606E0FFF7A8FC401B022801D903201F
:10643000F4E677486C300068C0F340000028F1D1E2
:10644000207800F00400042870D10026704838300D
:10645000006800F0805090B900BF002000906C48A8
:106460003830006840F0805069493831086008468B
:10647000006800F08050009000BF00BF0126674810
:10648000006800F48070B0B96448006840F480701F
:1064900062490860FFF770FC054606E0FFF76CFCF8
:1064A000401B022801D90320B8E65C48006800F4CC
:1064B00080700028F2D000BFA068012808D154489D
:1064C0006830006840F001005149683108601DE003
:1064D000A06805280DD14E486830006840F00400DF
:1064E0004B49683108600846006840F001000860C8
:1064F0000CE047486830006820F0010044496831EA
:1065000008600846006820F00400086000BFA0682A
:10651000A8B1FFF731FC054609E0FFF72DFC401B51
:1065200041F28831884202D9032077E626E03848D4
:1065300068300068C0F340000028EED013E0FFF799
:106540001BFC054608E0FFF717FC401B41F28831B1
:10655000884201D9032061E62D4868300068C0F305
:1065600040000028EFD1012E07D1294838300068BB
:1065700020F0805026493831086000BFA069B8B3C8
:106580002348006800F00C0008285ED0A0690228AB
:1065900046D100201F490866FFF7EEFB054606E0DE
:1065A000FFF7EAFB401B022801D9032036E6184812
:1065B00008380068C0F340600028F1D1D4E9070131
:1065C0000843616A40EA81110122A06AC2EB5000CF
:1065D00041EA00412C20005D41EA00600C49091F9E
:1065E000086001200B490866FFF7C6FB054607E077
:1065F0002DE0FFF7C1FB401B022801D903200DE667
:10660000034808380068C0F340600028F1D01EE05D
:106610000838024000004742800E474200700040A8
:1066200000200C490866FFF7A7FB054606E0FFF7C8
:10663000A3FB401B022801D90320EFE506480068B0
:10664000C0F340600028F2D101E00120E6E500201F
:10665000E4E5000000004742003802404FF0E0202F
:10666000006940F002004FF0E0210861704710B56A
:1066700004460CB9012010BD022084F851002068A6
:10668000006820F0400021680860204600F050F8C3
:106690000020606584F8510000BF84F8500000BFFE
:1066A00000BFE8E710B504460CB9012010BD606AD0
:1066B00000B900BF0021A16294F8510028B9002060
:1066C00084F85000204600F04BF8022084F8510076
:1066D0002068006820F0400021680860D4E90101CA
:1066E0000843E16808432169084361690843218B35
:1066F00001F400710843E1690843216A0843A16A73
:106700000843216808600421A06901EA1040616A19
:106710000843216848602068C06920F4006021684F
:10672000C86100206065012084F851000020BDE7A9
:1067300010B5044607492068884209D10648006818
:1067400020F4805004490860E0210448FFF74CF928
:1067500010BD0000003001404438024000000240FB
:1067600010B586B004461249206888421DD100BF8A
:10677000002000900F48006840F480500D490860E8
:106780000846006800F48050009000BF00BFE02081
:106790000190022002900020039003200490052025
:1067A000059001A90448FFF7EFF906B010BD0000FD
:1067B0000030014044380240000002402DE9F84317
:1067C00004460D4617461E464FF00008C146606855
:1067D000B0F5827F0DD1A06858B9042084F851002B
:1067E0003B462A4629462046009600F070F9BDE84F
:1067F000F88300BF94F85000012801D10220F6E789
:10680000012084F8500000BFFFF7B6FA804694F8E4
:106810005100012802D04FF002097BE005B117B901
:106820004FF0010976E0042084F8510000206065F3
:10683000A563A787E7872063A086E086206460645D
:10684000A068B0F5004F05D12068006820F48040B2
:10685000216808602068006800F04000402805D0EA
:106860002068006840F0400021680860E068E8B9EE
:1068700018E02068806800F0010038B12068007BD3
:1068800028706D1CE08F401EE0870BE03EB1701C4D
:1068900040B1FFF771FAA0EB0800B04202D34FF00D
:1068A000030937E0E08F0028E3D11CE018E02068FE
:1068B000806800F0010038B12068C0682880AD1CF5
:1068C000E08F401EE0870BE03EB1701C40B1FFF747
:1068D00053FAA0EB0800B04202D34FF0030919E0CD
:1068E000E08F0028E3D16068B0F5827F0DD1A06809
:1068F000B0F5004F03D0A068B0F5806F05D12068D7
:10690000006820F0400021680860606D08B14FF019
:10691000010900BF012084F8510000BF002084F865
:10692000500000BF484662E72DE9F84304460D4693
:1069300017461E464FF00008C14600BF94F85000AD
:10694000012802D10220BDE8F883012084F850001C
:1069500000BFFFF711FA804694F85100012802D0D9
:106960004FF00209A9E005B117B94FF00109A4E001
:10697000032084F85100002060652563A786E78620
:10698000A063A087E08760642064A068B0F5004F32
:1069900005D12068006840F48040216808602068C4
:1069A000006800F04000402805D02068006840F0F2
:1069B000400021680860E068B0F5006F2AD1606887
:1069C00010B1E08E012806D128882168C860AD1C6E
:1069D000E08E401EE08619E02068806800F002002A
:1069E000022807D128882168C860AD1CE08E401EAF
:1069F000E0860BE03EB1701C40B1FFF7BDF9A0EBA3
:106A00000800B04202D34FF0030956E0E08E0028A0
:106A1000E2D129E0606810B1E08E012806D1287823
:106A2000216808736D1CE08E401EE08619E0206826
:106A3000806800F00200022807D1287821680873D6
:106A40006D1CE08E401EE0860BE03EB1701C40B134
:106A5000FFF792F9A0EB0800B04202D34FF0030910
:106A60002BE0E08E0028E2D13346012202212046AD
:106A7000CDF8008005F0B8FB10B14FF003091CE021
:106A800042463146204605F077FB20B14FF0010920
:106A90002020606511E0A06850B900BF0020009080
:106AA0002068C068009020688068009000BF00BF28
:106AB000606D08B14FF0010900BF012084F851005A
:106AC00000BF002084F8500000BF48463BE72DE996
:106AD000FE4F04460D4616461F46DDF830804FF047
:106AE000000A0020029081464FF0010B019000BF88
:106AF00094F85000012802D10220BDE8FE8F012049
:106B000084F8500000BFFFF737F9814694F851A090
:106B100060680290BAF1010F0BD00298B0F5827F45
:106B200004D1A06810B9BAF1040F02D0022001907C
:106B3000D2E00DB106B117B901200190CCE094F874
:106B40005100012802D1052084F851000020606521
:106B5000A663E787A7872563E786A7862064606426
:106B60002068006800F04000402805D020680068D8
:106B700040F0400021680860E068B0F5006F43D144
:106B8000606810B1E08E012806D128882168C860AD
:106B9000AD1CE08E401EE0862FE0BBF1000F10D050
:106BA000E08E70B12068806800F00200022808D1F1
:106BB00028882168C860AD1CE08E401EE0864FF03A
:106BC000000BE08F68B12068806800F0010040B1E0
:106BD0002068C0683080B61CE08F401EE0874FF010
:106BE000010B08F1010040B1FFF7C6F8A0EB090066
:106BF000404502D3032001906EE0E08E0028CCD106
:106C0000E08F0028C9D142E0606810B1E08E012811
:106C100006D12878216808736D1CE08E401EE0863E
:106C20002FE0BBF1000F10D0E08E70B120688068BB
:106C300000F00200022808D115F8010B2168087342
:106C4000E08E401EE0864FF0000BE08F68B12068B8
:106C5000806800F0010040B12068C06806F8010BB0
:106C6000E08F401EE0874FF0010B08F1010040B1BA
:106C7000FFF782F8A0EB0900404502D30320019002
:106C80002AE0E08E0028CCD1E08F0028C9D143460D
:106C9000012202212046CDF8009005F0A5FA10B19E
:106CA0000320019018E04A464146204605F064FA68
:106CB00020B101200190202060650DE0A06850B94E
:106CC00000BF002000902068C068009020688068A5
:106CD000009000BF00BF00BF012084F8510000BF3A
:106CE000002084F8500000BF019806E7042808D16E
:106CF0004FF0E021096941F004014FF0E0221161F9
:106D000007E04FF0E021096921F004014FF0E02293
:106D100011617047704770B504462546681EB0F192
:106D2000807F01D301200FE0681E4FF0E021486111
:106D30000F214FF0FF3004F0A9F800204FF0E021C0
:106D4000886107200861002070BD10B5FFF7E2FFE1
:106D500010BD4FF0E020006920F002004FF0E0216C
:106D6000086170477047704710B50346002200BFA6
:106D700093F83800012801D1022010BD012083F8CA
:106D8000380000BF22F0FF00CC6840EA040222F481
:106D900040708C6840EA040222F480604C6840EA4B
:106DA000040222F400600C6840EA040222F48050DD
:106DB0000C6940EA040222F400504C6940EA0402E3
:106DC00022F480408C6940EA040222F400408C697D
:106DD00040EA04021868426400BF002083F83800CB
:106DE00000BF00BFC9E7024600BF92F83800012883
:106DF00001D102207047012082F8380000BF022034
:106E000082F839001068406820F0700013685860FC
:106E1000106840680B6818431368586010688068F1
:106E200020F0800013689860106880684B681843F1
:106E300013689860012082F8390000BF002082F8B2
:106E4000380000BF00BFD5E710B50446022084F823
:106E5000390000BF2068006A41F21111084050B9A2
:106E60002068006A8910084028B92068006820F06E
:106E700001002168086000BF204600F023F80020D0
:106E800084F8390000BF84F8380000BF10BD10B589
:106E900004460CB9012010BD94F8390028B900202F
:106EA00084F83800204600F021F8022084F83900E8
:106EB000211D206806F074FF012084F839000020AD
:106EC000E9E7000010B5044606492068884208D169
:106ED0000548006820F00200034908601D20FEF705
:106EE000CDFF10BD000400404038024038B50446D4
:106EF0000E492068884217D100BF002000900C483E
:106F0000006840F002000A4908600846006800F086
:106F10000200009000BF00BF002211461D20FEF7B6
:106F2000C8FF1D20FEF7B8FF38BD00000004004078
:106F30004038024001460868C06840F001000A6815
:106F4000D0600868006840F001000A681060002006
:106F5000704701460868C06820F001000A68D060E8
:106F600000BF0868006A41F21112104050B9086869
:106F7000006A9210104028B90868006820F00100EB
:106F80000A68106000BF002070472DE9F0410446F8
:106F90000D46002600BF94F83800012802D10220D7
:106FA000BDE8F081012084F8380000BF022084F899
:106FB00039002068866826F0770626F47F46206828
:106FC0008660286850283BD00CDC202860D004DC88
:106FD000002853D0102865D155E030285DD04028D6
:106FE00060D141E0602835D070280DD0B0F5805FC9
:106FF00003D0B0F5005F55D115E02068806820F01F
:107000000700216888604EE0D5E902136A682068AD
:1070100006F02CFF2068866826F0770646F0770693
:10702000206886603FE0D5E902136A68206806F0B0
:107030001DFF2068806840F480402168886032E04D
:10704000EA686968206806F0F3FF5021206806F0BE
:1070500019FF28E0EA686968206806F0FEFF6021F1
:10706000206806F00FFF1EE0EA686968206806F0F5
:10707000DFFF4021206806F005FF14E000212068B2
:1070800006F000FF0FE01021206806F0FBFE0AE08A
:107090002021206806F0F6FE05E03021206806F089
:1070A000F1FE00E000BF00BF012084F8390000BFFE
:1070B000002084F8380000BF00BF71E7704710B5AA
:1070C000044620680069C0F34000D8B12068C06859
:1070D000C0F34000B0B16FF00200216808610120E8
:1070E00020762068806900F0030018B12046FFF781
:1070F000E5FF05E0204600F0C7F8204600F07EF9E5
:107100000020207620680069C0F38000D8B1206894
:10711000C068C0F38000B0B16FF00400216808615E
:10712000022020762068806900F4407018B1204663
:10713000FFF7C4FF05E0204600F0A6F8204600F067
:107140005DF90020207620680069C0F3C000D8B146
:107150002068C068C0F3C000B0B16FF008002168BB
:107160000861042020762068C06900F0030018B18F
:107170002046FFF7A3FF05E0204600F085F82046F3
:1071800000F03CF90020207620680069C0F3001070
:10719000D8B12068C068C0F30010B0B16FF0100023
:1071A00021680861082020762068C06900F44070DA
:1071B00018B12046FFF782FF05E0204600F064F892
:1071C000204600F01BF9002020762068006900F0BE
:1071D000010058B12068C06800F0010030B16FF0C4
:1071E000010021680861204600F068F92068006904
:1071F000C0F3C01058B12068C068C0F3C01030B1EF
:107200006FF08000216808612046FFF7ABFD206821
:107210000069C0F3801058B12068C068C0F38010C6
:1072200030B16FF0400021680861204600F0D2F9CB
:1072300020680069C0F3401058B12068C068C0F3EE
:10724000401030B16FF02000216808612046FFF740
:107250008AFD10BD10B586B00446094920688842F1
:107260000CD1C014019002200290002003900490E1
:107270000120059001A90348FEF786FC06B010BD69
:107280000000014000000240704770B504460D4602
:10729000164600BF94F83800012801D1022070BDC5
:1072A000012084F8380000BF022084F8390036B18C
:1072B000042E1BD0082E31D00C2E5ED145E029467D
:1072C000206806F0E9FD2068806940F00800216828
:1072D00088612068806920F0040021688861206846
:1072E0008069296908432168886147E02946206848
:1072F00006F004FE2068806940F40060216888611F
:107300002068806920F48060216888612068806935
:10731000296940EA0120216888612FE02946206818
:1073200006F024FE2068C06940F008002168C861AA
:107330002068C06920F004002168C8612068C06925
:10734000296908432168C86118E02946206806F0C9
:1073500043FE2068C06940F400602168C86120686D
:10736000C06920F480602168C8612068C06929690B
:1073700040EA01202168C86100E000BF00BF012091
:1073800084F8390000BF002084F8380000BF00BF37
:1073900085E710B504460CB9012010BD94F83900FA
:1073A00028B9002084F83800204600F00DF80220AB
:1073B00084F83900211D206806F0F2FC012084F8D1
:1073C00039000020E9E7000008B50A4A0168914247
:1073D0000FD100BF002100910749096841F0010168
:1073E000054A11601146096801F00101009100BFD2
:1073F00000BF08BD00000140443802407047000053
:1074000030B504460D4601222946206806F020FDCD
:107410000A492068884201D1012000E0002028B1FB
:107420002068406C40F4004021684864206800688F
:1074300040F0010021680860002030BD00000140DC
:1074400030B504460D4600222946206806F000FDAE
:1074500019492068884201D1012000E0002090B144
:1074600000BF2068006A41F21111084050B920683D
:10747000006A8910084028B92068406C20F4004058
:107480002168486400BF00BF2068006A41F2111102
:10749000084050B92068006A8910084028B920685F
:1074A000006820F001002168086000BF012084F816
:1074B0003900002030BD00000000014010B5044636
:1074C00035480088401C3449088034480078401C06
:1074D0003249087030480088B0F57A7F51DB0020CF
:1074E0002D4908802E480088401C2D4908802D48D1
:1074F00090ED000AF7EE000A30EE200A80ED000A57
:10750000012029490870264800880A2821DDFAF759
:1075100007FA03281DD000BF00BF00BF00BF00BF97
:10752000BFF34F8F00BF00BF00BF2048006800F4CA
:10753000E0601F490843001D1C49086000BF00BFF0
:1075400000BFBFF34F8F00BF00BF00BF00BF00BF31
:10755000FDE71848B0F8580098B94FF40071164884
:10756000FEF7FCFB68B1FAF7DBF9032809D01348F2
:10757000036813480268134801681348006804F060
:107580001DFF0548008811490968884202D1012081
:107590000F49087010BD00001C00002020060020CC
:1075A0001E0000201C060020200000200CED00E042
:1075B0000000FA05E81F00200004024070060020C9
:1075C0006C06002068060020640600203C010020B4
:1075D000D9010020704710B504460CB9012010BD38
:1075E000242084F83900204600F0F2F80020E063FF
:1075F00084F8390084F83A0000BF84F8380000BFEE
:1076000000BFECE710B50446204608F071FC10BD41
:107610002DE9F0470446206805682068C6682068A0
:1076200047694FF00008C14605F00F08B8F1000F98
:107630000AD105F0200038B106F0200020B1204624
:1076400006F0E2FEBDE8F087B8F1000F6DD007F05C
:10765000010018B906F49070002866D005F001000A
:1076600030B106F4807018B1E06B40F00100E063C7
:1076700005F0040030B107F0010018B1E06B40F0F4
:107680000200E06305F0020030B107F0010018B11C
:10769000E06B40F00400E06305F0080030B107F053
:1076A000010018B1E06B40F00800E063E06B68B3E4
:1076B00005F0200028B106F0200010B1204606F0A9
:1076C000A3FE20684069C0F38019E06B00F0080059
:1076D00010B9B9F1000F22D0204606F06BFE2068E9
:1076E000406900F04000B0B12068406920F04000DF
:1076F00021684861606B50B11748616B0865606B29
:10770000FDF776FE10B1606B016D88470CE02046F6
:10771000FFF778FF08E02046FFF774FF04E02046FB
:10772000FFF770FF0020E0638CE705F0800030B1C8
:1077300006F0800018B1204607F068F882E705F0EF
:10774000400030B106F0400018B1204606F042FE7D
:1077500078E700BF76E70000B9E2020810B50446FA
:107760000CB9012010BDA06900B100E000BF94F881
:10777000390028B9002084F83800204600F082F84B
:10778000242084F839002068C06820F40050216863
:10779000C860204606F086FE2068006920F490400C
:1077A000216808612068406920F02A00216848614A
:1077B0002068C06840F400502168C8600020E06381
:1077C000202084F8390084F83A000020CAE700003D
:1077D00010B5044625492068884214D12448006821
:1077E00020F01000224908604FF4C0612148FEF7E4
:1077F000FBF8606BFDF710FE206BFDF70DFE2520FA
:10780000FEF73CFB30E01C492068884215D118483F
:10781000001F006820F400301549091F08600C2182
:107820001448FEF7E1F8606BFDF7F6FD206BFDF7FD
:10783000F3FD2620FEF722FB16E01049206888425F
:1078400012D10B48006820F0200009490860C021CF
:107850000B48FEF7C9F8606BFDF7DEFD206BFDF706
:10786000DBFD4720FEF70AFB10BD000000100140C1
:10787000443802400000024000440040001401402F
:107880000008024010B586B00446AA492068884224
:107890006CD100BF00200090A748006840F01000A5
:1078A000A54908600846006800F01000009000BF7D
:1078B00000BF4FF4C06001900220029001200390AD
:1078C000032004900720059001A99C48FEF75CF96D
:1078D0009B489C4908604FF000604860002199482F
:1078E0008160C1604FF4806101610021416181616B
:1078F0004FF48071C161002101624162FDF7DEFE3B
:1079000020B140F2651190A008F06CFE00BF8D48D8
:107910006063846300BF8A487830924908604FF002
:107920000060486040218F4881600021C1604FF4B1
:1079300080610161002141618161C1610162416237
:10794000FDF7BCFE20B140F277117FA008F04AFE9F
:1079500000BF84482063846300BF002201212520EA
:10796000FEF7A7FA2520FEF797FAE0E07E492068A7
:1079700088426DD100BF002000906F48001F006852
:1079800040F400306C49091F08600846006800F4A4
:107990000030009000BF00BF0C2001900220029038
:1079A00001200390032004900720059001A963485B
:1079B000FEF7EAF86D486E4908604FF000604860D5
:1079C00000216B488160C1604FF48061016100213A
:1079D000416181614FF48071C161002101624162A6
:1079E000FDF76CFE20B14FF4D27157A008F0FAFDFC
:1079F00000BF5F486063846300BF5C4818305D4926
:107A000008604FF00060486040215A4881600021C2
:107A1000C1604FF480610161002141618161C161F8
:107A200001624162FDF74AFE20B14FF4DB7146A0CE
:107A300008F0D8FD00BF4F482063846300BF0022D8
:107A400001212620FEF735FA2620FEF725FA6EE002
:107A50004949206888426AD100BF0020009036481A
:107A6000006840F02000344908600846006800F0D3
:107A70002000009000BF00BFC020019002200290B3
:107A800001200390032004900820059001A93B48A1
:107A9000FEF77AF82A4818383949086080054860A6
:107AA000002137488160C1604FF48061016100218D
:107AB000416181614FF48071C161002101624162C5
:107AC000FDF7FCFD20B140F2E3111FA008F08AFD94
:107AD00000BF2B486063846300BF194860302949A8
:107AE00008604FF0206048604021264881600021F6
:107AF000C1604FF480610161002141618161C16118
:107B000001624162FDF7DAFD20B140F2F5110EA0ED
:107B100008F068FD00BF1B482063846300BF00229B
:107B200001214720FEF7C5F94720FEF7B5F906B059
:107B300010BD000000100140443802400000024027
:107B40004064024060DE00202E2E2F5372632F739C
:107B5000746D3332663478785F68616C5F6D737012
:107B60002E630000C0DE0020004400408860024018
:107B700020DF002080DF00200014014000080240C8
:107B8000E0DF002040E0002077B581B004461546D4
:107B900094F83A00202850D1029800B115B901207C
:107BA00004B070BD00BF94F83800012801D1022054
:107BB000F6E7012084F8380000BF0298A062A5858E
:107BC0000020E063222084F83A001D48616BC863FE
:107BD0001C48616B08641C48616BC8640020616BC1
:107BE000086502AE32682368191D2B46606BFDF7ED
:107BF000DBFD00BF00200090206800680090206836
:107C00004068009000BF00BF00BF002084F838002B
:107C100000BF2068C06840F480702168C860206898
:107C2000406940F00100216848612068406940F0E7
:107C30004000216848610020B2E70220B0E7000060
:107C40001DE3020863E30208CDE2020810B5034613
:107C500093F83A00202829D101B10AB9012010BDBA
:107C600000BF93F83800012801D10220F7E7012076
:107C700083F8380000BF99629A85DA850020D863BE
:107C8000222083F83A0000BF002083F8380000BFAC
:107C90001868406940F001001C6860611868C0689D
:107CA00040F490701C68E0600020D8E70220D6E71E
:107CB00010B50446204608F055F910BD70472DE96F
:107CC000F84304460D4616461F464FF0000994F847
:107CD000390020285CD105B116B90120BDE8F88330
:107CE00000BF94F83800012801D10220F6E70120F6
:107CF00084F8380000BF0020E063212084F83900B8
:107D0000FEF73AF88146A684E6842BE0E08C401E1C
:107D1000E084A068B0F5805F16D14B460022802138
:107D20002046009706F0A6FD08B10320D6E7A84636
:107D3000B8F80000C0F3080021684860206908B95D
:107D4000AD1C0FE06D1C0DE04B460022802120464B
:107D5000009706F08FFD08B10320BFE715F8010B6F
:107D600021684860E08C0028D0D14B460022402199
:107D70002046009706F07EFD08B10320AEE72020E4
:107D800084F8390000BF002084F8380000BFA5E760
:107D90000220A3E7F7B50446154694F839002028D9
:107DA0003DD1019800B10DB90120FEBD00BF94F88E
:107DB0003800012801D10220F7E7012084F83800BB
:107DC00000BF01982062A584E5840020E0632120A3
:107DD00084F839001348216BC8631348216B086489
:107DE0001248216BC8640020216B086501AE23682E
:107DF0001A1D31682B46206BFDF7D6FC6FF0400052
:107E00002168086000BF002084F8380000BF2068A7
:107E1000406940F08000216848610020C5E70220E9
:107E2000C3E7000071E30208A7E30208CDE20208FD
:107E300010B5034693F83900202823D101B10AB9BF
:107E4000012010BD00BF93F83800012801D10220A5
:107E5000F7E7012083F8380000BF19629A84DA84BA
:107E60000020D863212083F8390000BF002083F868
:107E7000380000BF1868C06840F080001C68E060EF
:107E80000020DEE70220DCE710B50446204608F0BB
:107E90009FF910BD70472DE9FE4304460025A84612
:107EA00000260020029000270CB1606808B9BDE8E8
:107EB000FE83A068402800D9F9E700252CE0204681
:107EC00000F0DEF82E464FF000081DE0606A825D8B
:107ED00002AB4146204600F07CF90746022F0DD147
:107EE000606A0090E06A01906068029A00EBC2004C
:107EF0006A464168204600F0A1F808E007B906E0AC
:107F000000BF761C08F10108E06AB042DED800BF6D
:107F1000022F00D103E06D1CE06AA842CFD800BF59
:107F200000BFC4E70FB438B504460D4607A800905B
:107F3000D4E90601009B069A08F092FB206200201B
:107F4000009008480078012803D1216AA06900F058
:107F500047FB29462046236AA26900F00DF838BC89
:107F60005DF814FBEC06002010B50446A06B01F090
:107F7000A9FA002010BD0000F8B504460D461646CB
:107F80001F463A46314620466369984750B9204615
:107F9000FFF7EAFF0094084B2A460021A06B01F08E
:107FA00033FB06E00094054B01220021A06B01F099
:107FB0002BFB0020F8BD000001810208F1800208BF
:107FC00070B504460D468021204601F0C9FB2868A3
:107FD000E06368686060A868A060E868E06028699D
:107FE000206168696061A869A061E869E0610020BA
:107FF0002062286A6062686AA0620020E06284F8F9
:108000003000A86A606304F1380001F071FA10B121
:108010004FF0FF3070BD204600F002F8FAE7000094
:10802000014611B94FF0FF307047034800680860FF
:10803000014801600020F7E7E806002070B504461B
:108040000D461646022D06D0032D05D0042D04D072
:10805000052D07D102E000BF00BF00BF2046FFF79B
:1080600083FF00E000BF00BF32462946E06B00F00E
:10807000C5FA70BD0148007870470000EC0600208A
:1080800010B504460122402104F14000F8F7F1F850
:1080900010BD000010B50024124804681EE0204600
:1080A00021698847C8B910480078012810D1E16AD1
:1080B000606A01F0C5FB012803D1606A00F0B0F9E5
:1080C00006E0E16A606A00F051FA08A000F0A8F941
:1080D0002046FFF7E0FE0020E0622468002CDED19D
:1080E00010BD0000E8060020EC0600200D0A00008C
:1080F00010B50446002205212046FFF79FFF10BD62
:1081000010B50446002204212046FFF797FF10BD5A
:1081100070B504460D46204600F02FF8012801D125
:10812000801E70BD2068401CE168B0FBF1F201FBCD
:108130001200206026692368A16803FB06103246FE
:108140002946F8F784F80020EBE710B58160C2609B
:108150000361012444600024046010BD01460868E6
:10816000401CCA68B0FBF2F302FB13004A6890425D
:1081700001D1012070470020FCE701460868801CFF
:10818000CA68B0FBF2F302FB13004A68904201D1C7
:10819000012070470020FCE770B504460D462046DC
:1081A000FFF7DCFF012801D1801E70BD2669D4E9EC
:1081B000013003FB060132462846F8F748F86068AC
:1081C000401CE168B0FBF1F201FB1200606000208E
:1081D000EBE7F0B504460D46002600211BE004F154
:1081E0004000405C012815D1606850F83100405DC6
:1081F000904204D0002704F1400047540AE0761C66
:10820000606850F83170681C385C18B903B11960A7
:108210000220F0BD491CA0688842E0D80EB90020B9
:10822000F7E70120F5E700002DE9F04104460D468F
:108230009C46002700210023344E15B9481EBDE896
:10824000F0810320B5FBF0F800FB185020B90320A3
:10825000B5FBF0F0870004E00320B5FBF0F0401C14
:108260008700781C844502D24FF0FF30E7E70020FA
:10827000D055002100232AE0E05C06EBA000007846
:108280005054E05C80074FEA9068581C205C48EA34
:10829000201016F80080481C02F80080581C205C52
:1082A00000074FEA9068981C205C48EAA01016F876
:1082B0000080881C02F80080981C205C00F03F00C1
:1082C00016F80080C81C02F80080DB1C091DB81ECF
:1082D0008842D1D80320B5FBF0F800FB18500128E4
:1082E00002D002280FD108E04FF03D08881E02F8A6
:1082F0000080481E02F8008005E04FF03D08481E4F
:1083000002F8008000BF00BF002098E7CC360308C9
:1083100010B5024612B94FF0FF3010BD00BF106813
:108320008842FCD31068401A106050680844D36833
:10833000B0FBF3F403FB140050600020EDE710B530
:10834000024612B94FF0FF3010BD106808441060AB
:1083500000BFD36810689842FBD890680844D3687F
:10836000B0FBF3F403FB140090600020ECE7F0B5E1
:108370000446002522B11BB1E6682068B04202D352
:108380004FF0FF30F0BD2668E068801B884202D2C3
:108390004FF0FF30F6E7A0680844E668B0420BD91A
:1083A000D4E90260851B2668E068801B4E19B04244
:1083B00002D24FF0FF30E5E7A0682844E668B0FB42
:1083C000F6F706FB17001060681818600020D9E760
:1083D000014648687047014688687047024612B9EE
:1083E0004FF0FF3070470020506090601060D16007
:1083F00000BFF7E7014609B901207047086808B9CE
:108400000120FAE70020F8E7014609B9012070478A
:108410000A68C868904201D10120F8E70020F6E719
:108420000FB410B5ADF5027DF9F77AFA28B1002046
:108430000DF5027D10BC5DF814FB002485A8819029
:108440004FF4007101A8819B849A08F009F9044651
:1084500000208190B4F5007F01D340F2FF14224642
:1084600001A9002007F0DEFD0020E1E70FB410B500
:10847000ADF5027D002485A881904FF4007101A81C
:10848000819B849A08F0ECF8044600208190B4F5B2
:10849000007F01D340F2FF14224601A9002007F01B
:1084A000C1FD00200DF5027D10BC5DF814FB00003D
:1084B0000FB430B5ADF5097DF9F732FA28B10020D7
:1084C0000DF5097D30BC5DF814FB0024FDF754FC6C
:1084D0004FF47A71B0FBF1F201FB12059DF81E001A
:1084E0009DF81D109DF81C20CDE90405CDE9022161
:1084F0009DF81B009DF81A10CDE90010BDF818304A
:1085000011A24FF4007108A801F0A7FA0446224610
:1085100008A9002007F086FD8DA888904FF400710F
:1085200008A8889B8C9A08F09BF804460020889045
:10853000B4F5007F01D340F2FF14224608A90020C1
:1085400007F070FD0020BBE7253034752D25303253
:10855000752D2530327520253032753A253032752B
:108560003A253032752E253033752000F0B591B0A4
:1085700006460C46F9F7D4F910B1002011B0F0BD51
:10858000002515480078012801D00020F6E700BF3B
:10859000102C01D9102500E02546402101A8F7F74D
:1085A0006FFE0120402301AA29460090304601F0C9
:1085B0008BF80AA101A8F7F76EFE01A8F7F793FE62
:1085C00007463A4601A9002007F02CFD641B2E4403
:1085D000002CDDD10020D1E7800300200D0A00002F
:1085E00070B504460D46F9F79BF908B1002070BD3F
:1085F0002A462146002007F015FDF8E72DE9FC4149
:1086000004460D4617464FF00008002660880128F2
:108610001FD1206950B960680068CDE900051AA231
:1086200000212046E368FBF7E9FF12E0206950F8DB
:10863000250000782D280CD0206950F825006168AD
:108640000968CDE9001018A200212046E368FBF775
:10865000D5FF66683A4629462046F3689847804623
:108660000BE0706840B170683A462946C3682046FE
:1086700098478046766800E002E0B8F1010FF0D03C
:1086800000BFBDE8FC81000046534D3A252D3873EC
:108690002053544154453A252D32387320455645D0
:1086A0004E543A25750D0A0046534D3A252D387320
:1086B0002053544154453A252D32387320455645B0
:1086C0004E543A25730D0A002DE9F04704460E4634
:1086D00017469846DDE9089A00250CB9BDE8F087F1
:1086E00030212046F7F7CCFDC4F80890C4F810807C
:1086F0006660E7600021A16261620E480088208008
:10870000A4F802A00C48006860610B4804600948A6
:108710000088401C07490880656806E06560002203
:1087200011462046FFF76AFFAD68002DF6D100BF65
:10873000D4E70000CC060020C8060020024612B98B
:108740004FF0FF307047D1620020FBE72DE9F8437E
:1087500005460E4617461C46DDF820904FF00008EF
:108760002188484661F31F408046054B3A46314612
:108770002846CDF8008000F047FFBDE8F8830000F0
:10878000714602082DE9F04196B005460E4617469F
:10879000D5F80480002400201590444629E06C6040
:1087A000002201212846FFF729FFA64205D13A46BB
:1087B00000212846FFF722FF1DE0502101A8F7F70E
:1087C0005FFD15AB01AA21463046FBF732FF78B9B1
:1087D0000AE01598006868603A4600212846FFF7CD
:1087E0000DFF15984068159015980028F1D102E00A
:1087F0006468002CD3D100BFB46806E06C603A46D0
:1088000000212846FFF7FAFEA468002CF6D116B026
:10881000BDE8F081016E05E000F17C024B1CD35CE9
:108820005354491CC26D8A42F6D8704710B5C26DC8
:10883000511E05E000F17C02545C4B1CD454491ECF
:10884000026E8A42F6DD10BD70B505460C46A87969
:1088500010B101282ED100E000BF432C1BD004DC56
:10886000412C0CD0422C22D10FE0442C19D07E2C6C
:108870001DD100220821284600F028FB18E0002224
:108880000321284600F022FB12E0002204212846A2
:1088900000F01CFB0CE000220621284600F016FB2D
:1088A00006E000220521284600F010FB00E000BF92
:1088B00000BF2CE0432C1BD004DC412C0CD0422CFC
:1088C00022D10FE0442C19D07E2C1DD1002208218A
:1088D000284600F07FF818E000220321284600F027
:1088E00079F812E000220421284600F073F80CE029
:1088F00000220621284600F06DF806E0002205213E
:10890000284600F067F800E000BF00BF00BF00BFCE
:1089100070BD70B504460D46432D45D008DC1B2DB7
:108920000DD0332D24D0412D3CD0422D4CD13AE0F6
:10893000442D3AD05B2D10D07E2D45D123E02079F7
:1089400010B1042804D100E000BF0120207102E032
:108950000020207100BF00BF39E02079012802D13A
:108960000220207102E00020207100BF00BF2EE035
:108970002079022802D10320207102E0002020711A
:1089800000BF00BF23E02079032806D129462046F6
:10899000FFF75AFF0420207102E00020207100BF81
:1089A00000BF14E000BF00BF00BF2079022806D13D
:1089B00029462046FFF748FF0420207102E00020EE
:1089C000207100BF00BF02E00020207100BF00BF87
:1089D000207970BD2DE9F04104460D461746092D5A
:1089E00002D00020A066E0660A2D6FD2DFE805F015
:1089F0006E0540CDFDFCFBFAF9F8607910B1012855
:108A000033D100E000BFE06D63282BD23846D4F8A4
:108A1000981588472046FFF709FF04F17C00216E76
:108A20004754206E401C2066E06D401CE065266EB9
:108A30004FF0000808E004F17C02905DD4F898152E
:108A40008847761C08F10108E06DB042F3D803E0D6
:108A50000820D4F898158847B8F10000A8F101085B
:108A6000F6D100BF0020607100E000BF00BF28E227
:108A7000E06D20B9FEA0D4F89415884721E2607912
:108A800010B1012866D122E0002104F17C00E26DE2
:108A90008154616F01EBC10202EB011204F5A27176
:108AA00001EB8200C839F7F740FC606F401C60673B
:108AB000606F0A2801DB00206067A06F401CA06780
:108AC000A06F0A2801D30A20A06744E0F8E100BFA4
:108AD00000BF206F00EBC00202EB001204F5A27091
:108AE00000EB8201642204F22C50F7F7B0FB266FF2
:108AF00019E0701C0A21B0FBF1F201FB120808EB2F
:108B0000C80202EB081304F5A27202EB830106EB24
:108B1000C60202EB061304F5A27202EB8300642284
:108B2000F7F795FB4646606F09300A2190FBF1F29A
:108B300001FB1200B042DCD106EBC60101EB0612CC
:108B400004F5A27101EB8200642204F22C51F7F7C4
:108B50007EFB00E000BF00BFC6A0D4F89415884794
:108B6000204600F0A9FC04F17C0000F007FC002086
:108B700000F0A2FC00202066E065606F0A302067EC
:108B8000BDA0D4F8941588479BE1607910B1012805
:108B900053D100E000BFA06F00B94FE0A06F0A28DA
:108BA00003D1D4E91C0188420ED1A06F0A2841D01C
:108BB000606F0A30A16F401A0A21B0FBF1F201FB8D
:108BC0001200216F884235D0206F09300A21B0FB96
:108BD000F1F201FB12002067206F00EBC00205E0FC
:108BE00008E1CCE08EE07EE072E029E002EB0012CA
:108BF00004F5A27000EB8201C838F7F796FB04F188
:108C00007C00F7F770FBE065E06D20669BA0D4F870
:108C100094158847226F02EBC20303EB021304F59D
:108C2000A27202EB8300D4F89415884794A0D4F87C
:108C3000941588470120607100E000BF00BF40E14B
:108C4000607910B1012840D100E000BFA06F00B9E9
:108C50003CE0606F09300A2190FBF1F201FB120049
:108C6000216F88422ED0206F401C0A21B0FBF1F208
:108C700001FB12002067206F00EBC00202EB001224
:108C800004F5A27000EB8201C838F7F74EFB04F13F
:108C90007C00F7F728FBE065E06D206677A0D4F84C
:108CA00094158847226F02EBC20303EB021304F50D
:108CB000A27202EB8300D4F89415884770A0D4F810
:108CC000941588470120607100E000BF00BFF8E004
:108CD000206E002806DD206E401E20660820D4F895
:108CE00098158847EDE0D4E91710884209D204F1BD
:108CF0007C02236ED05CD4F898158847206E401C07
:108D00002066DEE0607910B1012835D100E000BFB7
:108D1000E06D70B3206E00282BDD0820D4F8981584
:108D20008847266E4FF0010808E004F17C02905D50
:108D3000D4F898158847761C08F10108E06DB04218
:108D4000F3D82020D4F89815884703E00820D4F8F9
:108D500098158847B8F10000A8F10108F6D1206EF7
:108D6000401E20662046FFF755FDE06D401EE06581
:108D700000BF0020607100E000BF00BFA1E060798B
:108D800010B1012833D100E000BFE06D60B3206E68
:108D9000002829DDD4E91701884225D0206E461C21
:108DA0004FF0010808E004F17C02905DD4F89815BA
:108DB0008847761C08F10108E06DB042F3D8202006
:108DC000D4F89815884703E00820D4F89815884708
:108DD000B8F10000A8F10108F6D12046FFF71AFD0E
:108DE000E06D401EE06500BF0020607100E000BF44
:108DF00000BF66E0607910B101285ED100E000BFDD
:108E0000E06D98B3E06E50B90120E06604F17C019A
:108E100004F1E000E26DF7F71AFAE06D60663CE0FD
:108E2000A06E00F0F1FA064604F1E001626EF7F779
:108E300085FAE0B913A0D4F894158847A06E00F025
:108E4000E3FA0646D4F894158847A06E00F0DCFAE1
:108E50000646314604F17C00F7F767FA04F17C001E
:108E6000F7F741FAE065E06D20660FE022E011E0DF
:108E70000D0A3E000D0A00003E0000000D3E0000FD
:108E80001B5B4A000D1B5B4A3E000000A06E401CAD
:108E9000A06607E0A06E401CA06600F0AFFAA16ECD
:108EA0008842BDD800BF00F0A9FAA16E884201D85F
:108EB0000020A0660020607100E000BF00BF00E05D
:108EC00000BF00BFBDE8F081002070472DE9F041F0
:108ED00004460E461746092E7DD2DFE806F07C05D3
:108EE000457C7C9BA6BDF800E06D63283BD2A07951
:108EF000012804D12A20D4F89815884703E0384681
:108F0000D4F8981588472046FFF790FC04F17C00C0
:108F1000216E4754206E401C2066E06D401CE065C9
:108F2000256E4FF0000810E0A079012804D12A2016
:108F3000D4F89815884705E004F17C02505DD4F818
:108F4000981588476D1C08F10108E06DA842EBD820
:108F500003E00820D4F898158847B8F10000A8F17C
:108F60000108F6D1ECE0EBE0E06D30B9A07920B972
:108F700075A0D4F894158847E2E0A07910B10128D3
:108F800045D115E0002104F17C00E26D815472A00E
:108F9000D4F8941588470120A07100202066E06570
:108FA00004F17C02102104F10C0000F056FD2FE0CA
:108FB000002104F17C00E26D81540020E06504F1A1
:108FC0007C02402104F11C0000F047FD04F11C016B
:108FD00004F10C0000E0B2E000F070F950B962A0BA
:108FE000D4F8941588470220A07100202066E0651F
:108FF00060710BE060A0D4F89415884752A0D4F8B3
:10900000941588470020A0712066E06500E000BF4D
:1090100000BF95E0206E002806DD206E401E206611
:109020000820D4F8981588478AE0D4E917108842B8
:1090300011D2A079012804D12A20D4F898158847A4
:1090400006E004F17C02236ED05CD4F898158847C2
:10905000206E401C206673E0E06DB0B3206E0028E7
:1090600033DD0820D4F898158847256E4FF00108A5
:1090700010E0A079012804D12A20D4F89815884757
:1090800005E004F17C02505DD4F8981588476D1C0A
:1090900008F10108E06DA842EBD82020D4F898151B
:1090A000884703E00820D4F898158847B8F10000F5
:1090B000A8F10108F6D1206E401E20662046FFF779
:1090C000A9FBE06D401EE06500BF39E0FFE7E06D01
:1090D000A0B3206E002831DDD4E9170188422DD0DD
:1090E000206E451C4FF0010810E0A079012804D142
:1090F0002A20D4F89815884705E004F17C02505DD9
:10910000D4F8981588476D1C08F10108E06DA84255
:10911000EBD82020D4F89815884703E00820D4F82D
:1091200098158847B8F10000A8F10108F6D120464B
:10913000FFF770FBE06D401EE06500BF00E000BF80
:1091400000BFBDE8F08100000D0A757365726E61A5
:109150006D653A20000000000D0A70617373776F2F
:1091600072643A20000000000D0A57656C636F6D51
:1091700065210D0A3E0000000D0A557365722076C8
:109180006572696679206661696C65642E0000000D
:1091900038B5002000900024424804687EE076E064
:1091A00000F0D6F905469DF800102046FFF7B1FB08
:1091B00000B16CE0FFF788FE01280AD1A068281AE8
:1091C0003949884207D9A5600020A071E065206672
:1091D00001E00220A071A07910B101282BD100E09C
:1091E00000BF9DF800000D2806D19DF80020022147
:1091F0002046FFF76BFE1DE09DF800000A2819D0FD
:109200009DF80000082805D1002207212046FFF71D
:109210005DFE0FE09DF80000092805D1002209211C
:109220002046FFF753FE05E09DF80020012120466F
:10923000FFF74CFE29E09DF800000D2806D19DF8AF
:10924000002002212046FFF7C5FB1DE09DF800002D
:109250000A2819D09DF80000082805D1002207210E
:109260002046FFF7B7FB0FE09DF80000092805D165
:10927000002209212046FFF7ADFB05E09DF8002004
:1092800001212046FFF7A6FB00BF00BF00BF6846D4
:10929000D4F89C158847002882D02468002C7FF4DD
:1092A0007EAF38BDF006002040771B0002490968F8
:1092B0000160014908607047F00600200246002066
:1092C0007047000000BFEFF3058000B1704707480A
:1092D000006820B9012080F3108800BF00BF034858
:1092E0000068401C0149086000BFEFE7D00600207D
:1092F00070B504460D4600F099F850B100F096F8AC
:10930000D0F8900528B100F091F8D0F8901502A09F
:109310008847002070BD00001B5B481B5B4A0000B3
:1093200030B502460C460021002302B114B94FF0BB
:10933000FF3030BD0021002315E00E4850F8310009
:1093400080B952F833000B4D45F8310002EBC300F1
:10935000406805EBC105686007480068401C064D81
:1093600028605B1C491C502901D2A342E5D3002090
:10937000DFE70000FC060020F8060020F0B595B0FD
:109380000446002600E0641C20782028FBD02046FC
:10939000F6F7A9FF10B9002015B0F0BD2046F6F78A
:1093A000A2FF2044461E02E000203070761E307876
:1093B0002028F9D0142301AA2021204600F064FBC4
:1093C0000746002511E00C4951F835002146F6F713
:1093D00091FF48B9084800EBC50001A9426838462A
:1093E000904700B905E004E06D1C00F007F8A842C2
:1093F000E9D800BF0020CFE7FC0600200148006844
:1094000070470000F80600200146054800688142C8
:1094100001D304A07047044850F83100FAE7000077
:10942000F806002000000000FC060020014800684B
:1094300070470000F40600202DE9F04106460F4673
:1094400000252AE0002412E0FFF7F0FF70B1FFF7DB
:10945000EDFFD0F8900548B1FFF7E8FFD0F8902570
:109460002819114B53F8301010A09047641C052C9C
:1094700004DAFFF7C3FF29198842E5D8FFF7D6FFC2
:1094800050B1FFF7D3FFD0F8900528B1FFF7CEFF1A
:10949000D0F8901507A088476D1DFFF7AFFFA842D1
:1094A000D0D80020BDE8F081FC060020252D313603
:1094B000730000000D0A00000149086070470000B9
:1094C000F40600200146202902D34FF0FF307047F8
:1094D0000120C1EBC102054B43F822000020C1EB83
:1094E000C10203EB8202D06000BFF0E7C0E00020C1
:1094F00070B5054600240DB9601E70BD00240DE056
:10950000C4EBC4000C4951F8200030B90120C4EB71
:10951000C401094A42F8210002E0641C202CEFD368
:1095200000BF202C05D105A0FEF77AFF4FF0FF30D9
:10953000E3E72C600020E0E7C0E0002074696D657F
:10954000722049442069732066756C6C0D0A000016
:109550000148006870470000D806002010B50024BC
:1095600000BF4AE0C4EBC400254951F8200002289E
:1095700042D1C4EBC40001EB8000C06821490968F6
:10958000081AC4EBC4011E4A02EB81010969884232
:1095900032D9C4EBC400114601EB8000806928B3C6
:1095A000C4EBC40001EB8000007928B90120C4EBB2
:1095B000C40142F821000CE00220C4EBC401104AAF
:1095C00042F821000F480068C4EBC40102EB81019E
:1095D000C860C4EBC4020A4B03EB82025069C4EBBF
:1095E000C40203EB82029169884705E00120C4EBC5
:1095F000C401034A42F82100641C202CB2D310BDE0
:10960000C0E00020D8060020F0B50446059D202CBF
:1096100002D34FF0FF30F0BD0220C4EBC406114F5F
:1096200047F82600C4EBC4003E4606EB80000171FB
:109630000D480068C4EBC40607EB8606F060C4EB77
:10964000C4003E4606EB80000261C4EBC40006EB9A
:1096500080008361C4EBC40006EB800045610020FC
:10966000D9E70000C0E00020D806002007480068C5
:10967000401C06490860064802684068521C40F1D8
:10968000000003490A60486070470000D8060020C7
:10969000E006002000BFEFF3058000B170470948E5
:1096A000006820B107480068401E06490860054868
:1096B000006820B9002080F3108800BF00BF00BF01
:1096C000ECE70000D00600202DE9F04305460C46EB
:1096D0009846079F0026002399460DB102B114B9A0
:1096E0000020BDE8F083012F01D1032000E002201B
:1096F0006043401C404501D90020F2E7002618E0F5
:1097000015F806904FEA191000F019F819465B1C7D
:10971000505409F00F0000F012F819465B1C505429
:10972000012F05D14FF0200C18465B1C02F800C039
:10973000761CA642E4D30020D0541846D1E7014657
:10974000092903DC01F13000C0B270470A2905DBAA
:109750000F2903DC01F13700C0B2F6E73020F4E74F
:1097600070B504460D4629462046F6F789FD70BDC2
:109770000146302904DB392902DCA1F130000EE07A
:10978000412904DB462902DCA1F1370007E0612909
:1097900004DB662902DCA1F1570000E00020C0B222
:1097A000704710B502460B46002406E01078FFF71C
:1097B000DFFF00EB0414521C5B1E002BF6D1204689
:1097C00010BD00B50246002305E01078FFF7D0FF7A
:1097D00000EB0313521C10780028F6D1184600BD88
:1097E00070B588B005460C4600200790069005909D
:1097F00004902846F6F777FD064604A805A906AAB0
:1098000007ABCDE9002102900AA23146284600F0BC
:1098100031F8042803D04FF0FF3008B070BD07982E
:109820002070069860700598A0700498E070002081
:10983000F3E7000025642E25642E25642E256400A0
:1098400002460B46002100BF10E0505C202803DBDD
:10985000505C7E2800DC08E0505C0D2802D0505C93
:109860000A2800D101E000207047491C9942ECD33E
:109870000120F9E70FB42DE9F847044600200090D5
:109880000022202600270CB10B9820B90020BDE84B
:10989000F8075DF814FB0CA80090D4E041B90B98D0
:1098A0000078252803D10B984078652800D0CFE0B8
:1098B0000B980078252874D10B98401C0B900B98BE
:1098C00010F8016B0B90652E6CD004DC2A2E07D0AB
:1098D000642E68D113E0702E7AD0782EF9D144E04E
:1098E00008E020780B9B1B78984202D0641C491E2C
:1098F00000E001E00029F4D100BF521C92E04FF0DB
:10990000000CE046002300252020DDF8009059F8E7
:10991000045BCDF800901AE02078B8F1000F06D172
:109920002D2804D14FF0010C4FF001080DE0302834
:109930000ADB392808DC4FF00108A0F1300903EBFD
:10994000830A09EB4A0300E003E0641C491E002976
:10995000E2D100BFBCF1010F03D16FEA030909F1A5
:10996000010305B12B60521C5CE000230025DDF8EB
:1099700000C05CF8045BCDF800C022E020783028FD
:1099800006DB392804DCA0F1300C0CEB031316E0E5
:10999000612809DB662807DCA0F1570C0CEB0313E8
:1099A0000DE043E033E03AE0412807DB462805DCE0
:1099B000A0F1370C0CEB031301E009E003E0641C99
:1099C000491E0029DAD100BF05B12B60521C29E0E5
:1099D000DDF800C05CF8040BCDF800C000250023C2
:1099E00025460CE094F800C0DDF82C8098F8008043
:1099F000C44501D05B1C00E003E0641C491E002943
:109A0000F0D100BF08B105604360521C0AE0009B22
:109A100001CB009300B10460521C012702E0012732
:109A2000002200BF00BF012F0DD111E020780B9B59
:109A30001B78984205D1641C0B98401C0B90491E62
:109A400001E0002204E00B98007800287FF426AFA4
:109A500000BF00200090104619E70FB4F8B5064685
:109A60000C46002509A8009021463046009B089A24
:109A700006F0F6FD054600200090A54200D3651EC5
:109A80002846F8BC5DF814FBF0B504460E461D46AA
:109A9000214600230DB104B10AB90020F0BD1846DB
:109AA0005B1C42F820100AE00878B04206D1002082
:109AB0000870481C1F465B1C42F82700491C0878A8
:109AC00008B1AB42F0D31846E8E770B5064600256A
:109AD000002478213046F6F7FCFB044624B95821CF
:109AE0003046F6F7F6FB04465CB1641C05E02078CE
:109AF000FFF73EFE00EB0515641C20780028F6D128
:109B000003E03046F6F729FC0546284670BD2DE9EE
:109B1000F04106460F4614463846F6F7E4FB054684
:109B200015B93046BDE8F081A54201D90020F9E71A
:109B300009E0641E2A4639463046F6F7E9FB08B9C3
:109B40003046EFE7761CAC42F3D20020EAE770B56E
:109B500004460D4604B115B94FF0FF3070BD012128
:109B600004F11000FEF7D4FB04F12000A968FEF711
:109B7000CFFB0020F2E770B504460D4604B115B9DD
:109B80004FF0FF3070BD012104F11000FEF7D7FB4C
:109B900004F12000A968FEF7D2FB0020F2E710B51F
:109BA00004460CB9002010BD04F11000FEF722FCA1
:109BB000012801D10020F6E704F12000FEF71AFC8D
:109BC000012801D10020EEE704F11000FEF700FCAF
:109BD00000EB4000216801EB8000E4E77CB504461F
:109BE0000E46002500200190009004B97CBD04F1D0
:109BF0001000FEF709FC08B10020F7E76B4601AA48
:109C0000314604F12000FEF7B2FB08B10020EDE779
:109C100004F11000FEF7DFFB00EB4000216801EBD0
:109C20008005A0680199084428606E600098A860CB
:109C30002846DBE72DE9F04104460E4617461D464F
:109C40004FF0000805EB4500B7EB800F03D84FF04D
:109C5000FF30BDE8F08105EB45004FEA8008266043
:109C6000C4F8048060683044A060A7EB0801E1609C
:109C7000294604F11000FEF7B1FB04F12000E16871
:109C8000FEF7ACFB0020E4E710B5044621460CA02B
:109C9000FEF7C6FB1048007868B11048006803F072
:109CA000E3FC012804D00D48006803F0F3FB02E058
:109CB0000020094908700A480068FFF703FC10BD3E
:109CC0004572726F72206F636375727265642040B3
:109CD00025730D0A000000005C05002060050020CF
:109CE0006405002038B504460D4635480078022842
:109CF0002BD134480068C82821D12CB932A0FFF7F5
:109D0000C3FF4FF0FF3038BD002060552B46224680
:109D100036493748FBF7F6F828B136A0FFF7B4FF0D
:109D20004FF0FF30EFE7042002F05EFB3A48008876
:109D300082B23A493A48006803F0F4FB3DE039A0AA
:109D4000FFF7A2FF4FF0FF30DDE71D480078032842
:109D500019D11C480068C8280FD1052002F044FB27
:109D6000002039490860394B4EF6602201460090C8
:109D700037480068FFF748FC1FE036A0FFF784FF74
:109D80004FF0FF30BFE70E480078052815D12CB9F9
:109D900039A0FFF779FF4FF0FF30B4E700202B4BDD
:109DA0004EF660220146009029480068FFF72CFC1F
:109DB0002A462146C820F7F759FD0020A3E70000F6
:109DC0005C050020800500202E2E5C464D4C5C4931
:109DD0006E7465726E65745C4E54524950436C6982
:109DE000656E742E633A333230000000BCBB002035
:109DF000DCBB00202E2E5C464D4C5C496E746572B7
:109E00006E65745C4E54524950436C69656E742E95
:109E1000633A333237000000700500203CBB00205D
:109E2000600500202E2E5C464D4C5C496E746572B8
:109E30006E65745C4E54524950436C69656E742E65
:109E4000633A3333360000007805002069E20208E7
:109E5000640500202E2E5C464D4C5C496E74657284
:109E60006E65745C4E54524950436C69656E742E35
:109E7000633A3335300000002E2E5C464D4C5C4971
:109E80006E7465726E65745C4E54524950436C69D1
:109E9000656E742E633A33353800000005E003A187
:109EA00009A006F0A1FB05F0D7FAF8E72E2E2F53F4
:109EB00072632F73746D3332663478785F69742EF1
:109EC000633A38350000000025732055525452651E
:109ED00073746172740000002DE9F04106460C466F
:109EE000002514E016F8017B3A111449022303FB04
:109EF000051013A106F0A0FB07F00F026900491C32
:109F00000E4BC8180EA106F097FB681CC5B2A542FF
:109F1000E8DB0D20094A02F814000A216000401C09
:109F20001154F7F7FDFC022805D16000821C03499B
:109F3000002006F077F8BDE8F0810000AE170020A1
:109F40002578000010B500224FF400510D48FBF7B2
:109F50000DFF00224FF480410A48FBF707FF0A205B
:109F600007F021F9012251030648FBF7FFFE0A2002
:109F700007F019F900224FF400510248FBF7F6FEF2
:109F800010BD00000004024010B500224FF4005143
:109F90000C48FBF7EBFE012291030A48FBF7E6FEB3
:109FA0000A2007F000F9012251030648FBF7DEFE04
:109FB0000A2007F0F8F800224FF400510148FBF79F
:109FC000D5FE10BD0004024070B5054600240026F1
:109FD0001CE000224FF400511148FBF7C7FE0A2095
:109FE00007F0E1F8012251030D48FBF7BFFE6006C0
:109FF000040E4FF480410A48FBF7B0FE08B1601C24
:10A00000C4B2052007F0CFF8701CC6B2082EE0DB02
:10A0100015B9FFF7B9FF01E0FFF794FF204670BDC7
:10A020000004024070B5044600224FF40051174866
:10A03000FBF79CFE002525E0E00928B101229103F1
:10A040001248FBF793FE05E000224FF480410F48D1
:10A05000FBF78CFE6006040E0A2007F0A4F801222C
:10A0600051030A48FBF782FE0A2007F09CF8002201
:10A070004FF400510548FBF779FE0A2007F093F8EA
:10A08000681CC5B2082DD7DB70BD0000000402407B
:10A0900010B5012291030C48FBF768FE0122510321
:10A0A0000948FBF763FE00224FF480410648FBF7A6
:10A0B0005DFE0A2007F077F800224FF400510248B5
:10A0C000FBF754FE10BD00000004024010B5002252
:10A0D0004FF400510C48FBF749FE00224FF4804139
:10A0E0000948FBF743FE0A2007F05DF801225103FF
:10A0F0000548FBF73BFE012291030348FBF736FEC0
:10A100000A2007F050F810BD0004024010B50024EA
:10A11000012291031248FBF729FE062007F043F8BD
:10A12000012251030E48FBF721FE062007F03BF801
:10A1300007E0601CC4B2FA2C03DDFFF7C7FF012063
:10A1400010BD4FF480410648FBF708FE0028F0D10F
:10A1500000224FF400510248FBF708FE0020EFE711
:10A160000004024010B51548808A00EE100AB8EECF
:10A17000400A1348D0ED000AB4EEE00AF1EE10FAFE
:10A1800003D201200F49087002E000200D49087039
:10A190000A48408F00EE100AB8EE400A0848D0ED99
:10A1A000000AB4EEE00AF1EE10FA05D20348C08FBF
:10A1B000012801D107F04EFD10BD0000E81F00206E
:10A1C0001C0600200800002010B50F48B0F8600001
:10A1D000012809D100200C49A1F860000BA110A0B2
:10A1E00006F002FA05F038F90748008845F2AA514E
:10A1F000884202D10448C08828B90DA108A006F001
:10A20000F3F905F029F910BDE81F00202E2E5C415E
:10A21000504C5C7577625F6170702E633A39340020
:10A220002573205552545265737461727400000096
:10A230002E2E5C41504C5C7577625F6170702E63AE
:10A240003A39390010B5F8F713FB10B14FF0FF3071
:10A2500010BD03F06BFF10B14FF0FF30F8E703F0D3
:10A260001BFF10B14FF0FF30F2E70020F0E710B510
:10A27000F9F762FD10BD000010B500220F21024861
:10A28000FEF7BCF9002010BDF4BA002010B5FFF7AE
:10A29000EEFF012804D14FF40800074908600AE0E6
:10A2A0000648007820B14FF408400349086002E0F6
:10A2B00000200149086010BD6C0600201602002035
:10A2C00010B53721202000F079F80321212000F07B
:10A2D00075F84021222000F071F80821232000F0B9
:10A2E0006DF8AA21302000F069F801200B49088799
:10A2F000084690F83810322000F060F80221332030
:10A3000000F05CF85F21202000F058F8044800F0CD
:10A3100009F80A2006F047FF10BD0000E81F0020E2
:10A320005506002010B5044621460F2000F023F802
:10A3300008B9002010BD0120FCE770B504460025D7
:10A34000FFF7A6FE3220FFF76DFEFFF7DFFEE0B25B
:10A35000FFF768FEFFF7DAFEFFF79AFE3320FFF7FC
:10A3600061FEFFF7D3FE0020FFF72EFE0546FFF744
:10A37000ADFE284670BD70B505460C462846FFF771
:10A38000DCFF2070012070BD70B504460D46FFF75C
:10A390007FFE3220FFF746FEFFF7B8FEE0B2FFF780
:10A3A00041FEFFF7B3FE2846FFF73CFEFFF7AEFE87
:10A3B000FFF78CFE0A2006F0F6FE70BD70B504466D
:10A3C0000D4629462046FFF7DFFF012070BD000043
:10A3D00001460020174A914203D2B1F1006F00D329
:10A3E00026E0154A914204D2124A914201D301203B
:10A3F0001EE0124A914204D20F4A914201D3022038
:10A4000016E00F4A914204D20C4A914201D3032034
:10A410000EE00C4A914204D2094A914201D3042031
:10A4200006E0094A914203D2064A914200D3052030
:10A4300070470000004000080080000800C00008CD
:10A440000000010800000208000004081FB51F48B2
:10A450001F4908604FF48030486000211C4881602B
:10A4600001210161816100210162C162194981629A
:10A470000021C1600221C161012101634161FAF73C
:10A4800081FE20B140F2051113A006F0ABF80120C7
:10A49000009001900720029069460D48FAF7A8FD48
:10A4A00020B140F20F110CA006F09CF81120009092
:10A4B0000220019069460648FAF79AFD20B14FF450
:10A4C0008C7105A006F08EF81FBD00000020014031
:10A4D00028DC00200100000F2E2E2F5372632F6DF9
:10A4E00061696E2E6300000008B500BF0020009077
:10A4F0002A48006840F4800028490860084600683F
:10A5000000F48000009000BF00BF00BF002000905A
:10A510000846006840F4001008600846006800F42F
:10A520000010009000BF00BF002211461020FBF772
:10A53000C0FC1020FBF7B0FC002211461120FBF7F5
:10A54000B8FC1120FBF7A8FC002211463820FBF7CD
:10A55000B0FC3820FBF7A0FC002211463920FBF7A5
:10A56000A8FC3920FBF798FC002211463A20FBF7A3
:10A57000A0FC3A20FBF790FC002211464520FBF797
:10A5800098FC4520FBF788FC002211464620FBF78B
:10A5900090FC4620FBF780FC08BD000030380240EC
:10A5A00000B587B000BF002001908748006840F0E8
:10A5B0000400854908600846006800F00400019026
:10A5C00000BF00BF00BF002001900846006840F0B7
:10A5D000800008600846006800F08000019000BF1D
:10A5E00000BF00BF002001900846006840F0010055
:10A5F00008600846006800F00100019000BF00BF3D
:10A6000000BF002001900846006840F0020008608A
:10A610000846006800F00200019000BF00BF00BFC4
:10A62000002001900846006840F0080008600846D5
:10A63000006800F00800019000BF00BF012248F24E
:10A6400010116248FBF792FB012241F210016048B1
:10A65000FBF78CFB0022A5215E48FBF787FB01225C
:10A6600046F248415B48FBF781FB00224FF48071C2
:10A670005748FBF77BFB00224FF480515348FBF710
:10A6800075FB002204215448FBF770FB4FF4005087
:10A69000029000200390049002A94D48FBF774FA41
:10A6A000012002904D4803900020049002A94748E1
:10A6B000FBF76AFA49F21010029001200390002083
:10A6C0000490059002A94148FBF75EFA41F2101090
:10A6D00002900120039000200490059002A93C48BC
:10A6E000FBF752FA40F2ED40029001200390002067
:10A6F0000490059002A93748FBF746FA0220029021
:10A70000364803900120049002A93248FBF73CFA36
:10A710004FF480500290314803900020049002A929
:10A720002C48FBF731FA4FF4C040029011200390FF
:10A73000002004900320059002A92648FBF724FA84
:10A740004FF400700290254803900020049002A965
:10A750001F48FBF719FA0420029001200390002003
:10A7600004900220059002A91B48FBF70DFA4FF454
:10A770000470029000200390049002A91548FBF792
:10A7800003FA002201210620FBF793FB0620FBF7CA
:10A7900083FB002201210720FBF78BFB0720FBF73F
:10A7A0007BFB002201211720FBF783FB1720FBF71F
:10A7B00073FB002211462820FBF77BFB2820FBF7C8
:10A7C0006BFB07B000BD00003038024000000240C3
:10A7D0000008024000040240000C0240000011107A
:10A7E00010B51048104908604FF48270486000218D
:10A7F0000D488160C160016141614FF40071816168
:10A800000821C16100210162416281620A21C162A5
:10A81000FBF748FF20B14FF4987104A005F0E2FE69
:10A8200010BD000000300140D0DC00202E2E2F5340
:10A8300072632F6D61696E2E6300000000B591B0E8
:10A84000284829490860092048600021264881607D
:10A850004FF43761C160002101614161FCF799FD4E
:10A8600020B140F2451121A005F0BCFE00200F9060
:10A8700010900FA91C48FCF7B6FA20B14FF4A6714E
:10A880001AA005F0AFFE602008904FF4B760099061
:10A8900000200A900C900D900E900C2208A91248EE
:10A8A000FCF7F3FC20B140F2571110A005F09AFE1E
:10A8B0000020019002900390049005904FF4005006
:10A8C00006900020079001A90748FCF74DFA20B137
:10A8D00040F2631105A005F085FE0348FCF7BAFCC1
:10A8E00011B000BD0000014028DD00202E2E2F53A6
:10A8F00072632F6D61696E2E6300000000B587B032
:10A900001848194908604F204860002116488160A6
:10A910004FF47A71C16000210161FCF7B8FA20B1EF
:10A920004FF4BC7111A005F05DFE4FF48050039010
:10A9300003A90D48FCF729FB20B14FF4BF710BA010
:10A9400005F050FE00200190029001A90648FCF796
:10A950004AFA20B140F2851104A005F043FE07B089
:10A9600000BD00000004004064DD00202E2E2F53A7
:10A9700072632F6D61696E2E6300000010B50C4884
:10A980000C4908604FF4E1304860002109488160BB
:10A99000C16001610C21416100218161C161FCF74D
:10A9A000DDFE20B14FF4CC7103A005F01BFE10BDFD
:10A9B00000100140A0DD00202E2E2F5372632F6D5A
:10A9C00061696E2E6300000010B50C480C490860E8
:10A9D0004FF416404860002109488160C160016160
:10A9E0000C21416100218161C161FCF7B7FE20B1FA
:10A9F00040F2AB1103A005F0F5FD10BD004400408E
:10AA0000E0DD00202E2E2F5372632F6D61696E2EB4
:10AA10006300000010B50C480C4908604FF4E130A9
:10AA20004860002109488160C16001610C214161D9
:10AA300000218161C161FCF791FE20B14FF4DF710B
:10AA400003A005F0CFFD10BD0014014020DE002062
:10AA50002E2E2F5372632F6D61696E2E63000000DE
:10AA600000BFFEE700487047787700200048704735
:10AA700058770020004870476877002000487047EA
:10AA80008D770020024604480260044801600120DE
:10AA9000034B187000207047480400204404002035
:10AAA0004C0400200146034A505C0022014B5A54DA
:10AAB000704700005E0400200146034A505C0022FB
:10AAC000014B5A54704700006104002070B50446E1
:10AAD0000D460648006830B1054829460268204600
:10AAE000024B1B689847002070BD000050040020F6
:10AAF0005404002001460120024A50540020024A1A
:10AB0000505470475E04002061040020014601207B
:10AB1000024A50540020024A5054704761040020F9
:10AB20005E04002010B5044614B94FF0FF3010BD8C
:10AB3000012004490870224680210348FEF78DFF5A
:10AB40000020F4E7640400208D7700200249087893
:10AB50000021014A11707047640400200146002062
:10AB60007047000070B505460C46152C07D22246EA
:10AB700029460448F5F76BFB0020024908550020E0
:10AB800070BD00007877002070B505460C46022C99
:10AB900002D24FF0FF3070BDA41E102C07D2224607
:10ABA00029460448F5F753FB0020024908550020C8
:10ABB000F1E700005877002070B505460C46022CDE
:10ABC00002D24FF0FF3070BDA41E102C07D22246D7
:10ABD00029460448F5F73BFB0020024908550020B0
:10ABE000F1E700006877002002460348026003484E
:10ABF0000160002070470000500400205404002031
:10AC0000024908780021014A117070474C04002065
:10AC100010B504460648006828B106480168204679
:10AC2000034A1268904704480460002010BD0000E9
:10AC30004804002044040020400400207047000025
:10AC400008B50F48FEF754FC10B14FF0FF3008BDB7
:10AC50000C48FEF74DFC10B14FF0FF30F7E7002035
:10AC6000094B42F210720121009006480068FEF77D
:10AC7000CBFC002005490860F6F73AFE0020E6E725
:10AC8000340200203C02002039180208380200205B
:10AC900070B504460E462046F5F725FB05462946C5
:10ACA000204600F0D7F870BDF8B504460E461546AC
:10ACB0001F46642C04D0652C03D0C82C29D117E082
:10ACC00000BF16480068401C144908600846006828
:10ACD00003280AD90020124B47F230520146009057
:10ACE00010480068FEF790FC01E0F6F701FE11E065
:10ACF00000200A4908602A463146022005F092F9F0
:10AD000010B109A0FDF78CFB29460DA0FDF788FBCB
:10AD100000E000BF00BF0020F8BD000038020020A6
:10AD200035E202083402002052544B204461746121
:10AD30002053656E64204572726F720D0A00000028
:10AD40002575422052544B20446174612053656E36
:10AD5000740D0A002DE9F84F04460F4615461E46AD
:10AD6000DDE90B8ADDF828904FF0000B1E480078D3
:10AD700018B14FF0FF30BDE8F88F24B1B8F1000FE3
:10AD800001D005B116B94FF0FF30F4E7224640215B
:10AD90001648FEF762FE4A4620211548FEF75DFE82
:10ADA0002B4614A2402115480096FEF756FE834616
:10ADB0008023134A59461148FDF736FA11480760B7
:10ADC0001148C0F800801148C0F800A0012001F02F
:10ADD0000BFB0C48008882B204490D48006802F061
:10ADE000A1FB0020C7E700005C0500203CBB002061
:10ADF000BCBB002025733A25730000007CBB0020FB
:10AE00001DBC002070050020680500206C05002096
:10AE10006005002010B500200A49087000230A4A86
:10AE200001210A4802F0A4FB10B14FF0FF3010BD21
:10AE30000748FEF75DFB10B14FF0FF30F7E7002049
:10AE4000F5E700005C050020ADD302086005002096
:10AE50006405002070B504460D46064800780528B4
:10AE600005D12A4621460448006802F0A7FD0020CB
:10AE700070BD00005C0500206005002002480068ED
:10AE8000C0F30220704700000CED00E010B5002870
:10AE900007DA0A07140E054A00F00F031B1FD454EB
:10AEA00003E00A07130E024A135410BD18ED00E028
:10AEB00000E400E038B500250020009000BF5E48A7
:10AEC0000068C0F580525D485B4B1B68C1186B463B
:10AED0005B48006802F0B6FC05460DB9009800B961
:10AEE000A7E055480068009908445349086008469F
:10AEF0000068B0F5805F03D352A0FEF7C5FE98E06E
:10AF000059480078052808D14B4801684B48FEF79E
:10AF1000E9FE0020484908608AE053480078032889
:10AF20001BD152A14548009AFEF7F1FD5049086037
:10AF30000846006800287AD04E4B4FA23F4800993F
:10AF4000FEF798FC032803D04EA0FEF79DFE70E0AC
:10AF500000210846FEF7C6FE69E043480078022853
:10AF600065D151480078002855D150A13348009A46
:10AF7000FEF7CDFD3E49086008460068002856D01F
:10AF8000002408460068001D08603A4B3AA22B488E
:10AF90000099FEF76FFC032803D046A0FEF774FE6D
:10AFA00047E04DA12548009AFEF7B1FD04466CB379
:10AFB000103400E0641C20782028FBD01F48201AA1
:10AFC000009A111A494B4AA22046FEF753FC012869
:10AFD00003D049A0FEF758FE2BE02548006817492A
:10AFE000401A4249096808444C49086001202E492A
:10AFF0000870114800684949096888420AD33B48EB
:10B0000001681B480068FEF76DFE12E044A0FEF7E1
:10B010003BFE0EE00BE008480068404909688842A2
:10B0200005D33248016812480068FEF75BFE00BF96
:10B0300045E700BF002038BD780500209DC00020F6
:10B04000600500202E2E5C464D4C5C496E74657286
:10B050006E65745C4E54524950436C69656E742E33
:10B06000633A3339350000005C0500200D0A00000A
:10B070008805002080050020252A20256420252A17
:10B080000D0A00002E2E5C464D4C5C496E746572B4
:10B090006E65745C4E54524950436C69656E742EF3
:10B0A000633A3431330000005D0500200D0A0D0ABB
:10B0B000000000002E2E5C464D4C5C496E7465729B
:10B0C0006E65745C4E54524950436C69656E742EC3
:10B0D000633A343334000000436F6E74656E742D30
:10B0E0004C656E6774683A200000000084050020FB
:10B0F00025640D0A000000002E2E5C464D4C5C4974
:10B100006E7465726E65745C4E54524950436C693E
:10B11000656E742E633A3435300000007C050020E3
:10B120002E2E5C464D4C5C496E7465726E65745C87
:10B130004E54524950436C69656E742E633A3436EE
:10B140003500000010B50446F6F748FBFFF70AF893
:10B1500003480088401C0249088006F017FE10BD15
:10B160000A00002010B501200549087000F0F2F82F
:10B17000012211030348FAF7F9FD00F005F810BDAC
:10B18000160200200000024010B504F0C1F90121B0
:10B19000044806F081FB002006F0C4FB002006F006
:10B1A00049FB10BD00D023247047000010B54FF4B8
:10B1B00080511048FAF7D2FDD0B14FF47A7005F003
:10B1C000E8FF4FF480510B48FAF7C8FD80B10EE05C
:10B1D0004FF480510748FAF7C1FD40B9642005F0EB
:10B1E000D8FF00224FF480710348FAF7BFFDEFE764
:10B1F00010BD0000000402400000024010B5002015
:10B200004849087048480078C8B10020F6F7ACFCFF
:10B21000002045490870FFF7A5FF4FF4007143482F
:10B22000FAF79CFD58B9642005F0B3FF00224FF4F3
:10B2300080713F48FAF79AFD642005F0AAFF4FF4A9
:10B2400000713A48FAF78AFD10B9002039490870B0
:10B25000FEF77EF94FF47A71B0FBF1F201FB1200B8
:10B260000A281CD23448007858BB344800780F288C
:10B2700003DD88203249086003E04FF4084030497C
:10B28000086001202C4908702D4803682D48026889
:10B290002D4801682D48006801F090F811E026481B
:10B2A000007870B1002024490870254908600846DC
:10B2B000036824480268244801682448006801F0B3
:10B2C0007DF8FEF745F922490968401A41F28831B4
:10B2D000884225D9FEF73CF91D4908604FF480618A
:10B2E0001248FAF73BFD40B100F03AF8BCEEC00A54
:10B2F00010EE100A1149087012E0012291020B4869
:10B30000FAF734FD00F02CF8BCEEC00A10EE100A7B
:10B310000A49087000224FF480610448FAF726FDBC
:10B3200010BD0000100000200F00002000040240AB
:10B3300000000240820300202F0000201E02002097
:10B34000700600206C0600206806002064060020BD
:10B350001400002010B50020FFF7D8FB002010BD1E
:10B3600010B52DED068B9FED3D0AB0EE408A9FEDA6
:10B370003B0AF0EE408A00F081F8B0EE408A9FED83
:10B38000380AB4EEC08AF1EE10FA04D29FED330A07
:10B39000F0EE408A19E0B1EE000AB4EEC08AF1EE98
:10B3A00010FA04DD9FED2F0AF0EE408A0DE09FEDCC
:10B3B0002C0A38EE400A9FED2C1AC0EE010A9FEDD0
:10B3C000290A20EE800AF0EE408A284890ED000A13
:10B3D000B5EEC00AF1EE10FA06D2C0ED008AFEF713
:10B3E000B7F82349086033E0204890ED000A30EEBA
:10B3F000680A10EE101A0846F5F751F941EC1A0BDD
:10B40000B0EE4A0AF0EE6A0A05F044F9B0EE409A4E
:10B41000F0EE609A9FED170B53EC102B51EC190BCB
:10B42000F5F750F904D2FEF793F8114908600FE0E0
:10B43000FEF78EF80E490968401A4EF660218842E0
:10B4400006D90A48C0ED008AFEF782F8084908606C
:10B45000064890ED000ABDEC068B10BD0000000010
:10B46000333353400000C8423333333F38060020A3
:10B470003C060020000000000000E03F2DE9F04104
:10B480002DED0C8B0020F5F7A3FD85B20024284696
:10B49000F5F7F8F841EC1B0B9FED500B53EC102B1C
:10B4A000F5F781F841EC1A0B9FED4E0B53EC102B86
:10B4B000F5F707F841EC190BF5F734F908EE100A27
:10B4C000B0EE000A28EE000AB0EE408A2846F5F7F2
:10B4D000D9F841EC1B0B9FED410B53EC102BF5F70A
:10B4E00062F841EC1A0B9FED3F0B53EC102BF4F775
:10B4F000E8FF41EC190BF5F715F93C4908600846DF
:10B5000090ED000AF0EE000A20EE200A80ED000A1D
:10B510000020F5F75DFD87B20120F5F759FD1FFA10
:10B5200080F8334806883846F5F7ACF841EC1B0B39
:10B530003046F5F7A7F841EC1D0B9FED2A0B53ECB5
:10B54000102BF4F7BEFF41EC1C0B53EC1B2BF4F754
:10B55000B8FF41EC1A0B9FED270B53EC102BF4F7BF
:10B56000B0FF41EC190BF5F7DDF800EE100AC8EB5F
:10B57000083000EE900AF8EEE00A80EE201AF0EEB5
:10B58000418A18EE900AF5F78AF841EC190B9FED05
:10B59000150B53EC102BF5F795F802D20120174943
:10B5A00008609FED170A38EEC00A9FED161AC0EE2C
:10B5B000010A9FED150A20EE800ABDEEC00A10EECA
:10B5C000104A642C00DD6424002C00DA0024B0EE64
:10B5D000480ABDEC0C8BBDE8F081000000000000C3
:10B5E00000FEAF406666666666660A403406002066
:10B5F0002A7AFF1F000000000000004030060020F3
:10B6000033335340CDCC4C3F0000C84210B500212D
:10B610000248FFF7E9FA002010BD000021B6020839
:10B62000014B1A60704700007C0100201CB506F039
:10B63000A7FC40F20510BC4948800120BB490870B6
:10B64000B94890F84400BA490870012008700846CB
:10B65000007848B94FF47A70B349C8800120C88790
:10B660000A20488700208887AF48C088322802DA3D
:10B670006420AD49C880AC48C088B0F57A7F03DD4E
:10B680004FF47A70A849C880A748008F0A2802DDC5
:10B690000220A5490887A448C08E432802DD432024
:10B6A000A149C886A048C08E002802DA00209E4921
:10B6B000C8869D48808A4FF6FF71884202D10A20D1
:10B6C000994988829848808C42F21071884202DD44
:10B6D000002095498884944890F836009549087070
:10B6E000914890F83E00944908708F4890F83C00CB
:10B6F000924908708C48807A914908708A488088FD
:10B70000904908600520904908808748C0880988CA
:10B7100090FBF1F08D49088083488088098890FB70
:10B72000F1F201FB120088490988484388490880E2
:10B7300008460088874908807B48C0884FF47A71A2
:10B7400091FBF0F08449088008460088C82191FBED
:10B75000F0F0824908800020814908805520814905
:10B760000870AA2048707048408C000B4FF47A7122
:10B7700010FB01F16C48408CC0F3032000EBC002C9
:10B7800002EB001001EB8000674991F82210C1F331
:10B79000031101EB810100EB4100634991F8221094
:10B7A00001F00F010844704908805F48808C000B4D
:10B7B0004FF47A7110FB01F05B49898CC1F30321CE
:10B7C00001EBC10202EB011100EB8100564991F837
:10B7D0002410C1F3031101EB810100EB4100524938
:10B7E00091F8241001F00F010844604908804E4888
:10B7F000C08C000B4FF47A7110FB01F14A48C08CE9
:10B80000C0F3032000EBC00202EB001001EB80004C
:10B81000454991F82610C1F3031101EB810100EBBA
:10B820004100414991F8261001F00F0108445049A8
:10B8300008803D48008D000B4FF47A7110FB01F039
:10B840003949098DC1F3032101EBC10202EB01115A
:10B8500000EB8100344991F82810C1F3031101EB8A
:10B86000810100EB4100304991F8281001F00F01EF
:10B870000844404908802C48008B3F4908803148E3
:10B8800001683EA004F0B0FE27488278408801128B
:10B890003EA004F0A9FE3848008836490988CDE961
:10B8A000001033480388314802882F48018840A09F
:10B8B00004F09AFE1C48B0F8560001280DD11A4831
:10B8C000008B1949098DCDE900101748C38C828C73
:10B8D000418C3FA004F088FE25E01348B0F85600E4
:10B8E000022819D1454946A004F07EFE0E48B0F862
:10B8F000A01247A004F078FE4049223148A004F08D
:10B9000073FE3E4942314BA004F06EFE3B4962316A
:10B910004DA004F069FE06E00348B0F8560010B9E7
:10B920004FA004F061FE1CBDE81F00202D00002088
:10B930000C02002075060020F4010020F501002013
:10B94000D7010020CC010020E0010020E20100200E
:10B95000DC010020EC010020EA01002000020020B0
:10B960000E020020B4110020AC010020AE01002026
:10B97000B0010020B2010020B4010020C9E8B1B834
:10B9800049443A202578202E0D0A0000B9CCBCFE8F
:10B99000B0E6B1BE3A205552542D4D4BB0B2B0EE88
:10B9A000B3B5D4D8205625642E25642E200D0A0068
:10B9B000B7FECEF1C6F7B5D8D6B73A2025642E2506
:10B9C000642E25642E25643A25642E0D0A0000009D
:10B9D0005443505F5254434DC4A3CABD2CB7FECE4E
:10B9E000F1C6F7B5D8D6B73A2025642E25642E25A2
:10B9F000642E25643A25642E0D0A0000682200207A
:10BA00004E74726970486F73743A25732E0D0A0074
:10BA10004E74726970506F72743A25642E0D0A006C
:10BA20004E74726970557365726E616D653A2573F7
:10BA30002E0D0A004E7472697050617373776F72C5
:10BA4000643A25732E0D0A004E74726970536F7537
:10BA50007263656E616D653A25732E0D0A000000F4
:10BA6000B5A5B5E3B6A8CEBBC4A3CABDC4A3CABD21
:10BA70002E200D0A0000000000B54FF4000003491D
:10BA800008604FF4FA7006F0D9FB00BD18040240BC
:10BA900030B50446002517230AE024FA03F000F02D
:10BAA000010515B100F01AF801E000F005F85B1E81
:10BAB000002BF2DA30BD000000B580200649086096
:10BAC000022006F0BBFB4FF40000034908600A2087
:10BAD00006F0B4FB00BD00001804024000B5802051
:10BAE000064908600B2006F0A9FB4FF4000003494B
:10BAF0000860022006F0A2FB00BD0000180402400E
:10BB000038B504461CB9002000F010F808E0002009
:10BB1000044B22460146009003480068FDF774FD7F
:10BB200038BD00002DBB02082C06002072B6064965
:10BB3000064A116000BF00BF00BFBFF34F8F00BFB8
:10BB400000BF00BF704700000400FA050CED00E0E4
:10BB500000B585B014216846F4F792FB642005F027
:10BB600018FB00224FF400411148FAF7FFF84FF498
:10BB7000004000900120019000200290039069464F
:10BB80000B48FAF701F8642005F003FB4FF400407E
:10BB90000090032001900020029003906946044821
:10BBA000F9F7F2FF022005F0F4FA05B000BD00003D
:10BBB0000004024010B50446204600F0CCFA00B163
:10BBC00018E0204600F034F80022C721204600F09B
:10BBD00039FA00B111E0204600F016F8204600F0D6
:10BBE000A9FA00B106E0204600F03CFA00B101E0FD
:10BBF000002010BD4FF0FF30FBE7204600F004F8B6
:10BC00004FF0FF30F5E7000010B5044604EB840266
:10BC1000064B03EBC202118904EB840203EBC20260
:10BC200050680122FAF7A2F810BD0000307700201A
:10BC300010B5044604EB8402064B03EBC2021189E3
:10BC400004EB840203EBC20250680022FAF78EF87C
:10BC500010BD0000307700202DE9F04107460C466A
:10BC600015461E464FF0000807EB87001C4901EB04
:10BC7000C000406AA04211D985B1601907EB870165
:10BC8000174A02EBC101496A884207D8154850F8A3
:10BC90002600401E204008B9032E03DB4FF0FF3082
:10BCA000BDE8F08164B907EB87000D4901EBC000E6
:10BCB000406AA84204D83846FFF77CFF0020EFE72F
:10BCC00009E004EB08013246384600F06FF90548F8
:10BCD00050F826008044A845F3D30020E0E7000098
:10BCE00030770020D823030838B50446032269467C
:10BCF000204600F011F910B14FF0FF3038BD9DF82B
:10BD00000000FF2810D19DF80100FF280CD19DF8FC
:10BD10000200FF2808D103226946204600F0FCF803
:10BD200010B14FF0FF30E9E79DF80200152806D06A
:10BD300016280DD0172814D0182824D11AE04FF453
:10BD4000800004EB8401164A02EBC101486223E043
:10BD50004FF4800004EB8401114A02EBC1014862F8
:10BD60001AE04FF4000004EB84010D4A02EBC1011C
:10BD7000486211E04FF0807004EB8401084A02EB46
:10BD8000C101486208E04FF4800004EB8401044ADA
:10BD900002EBC101486200BF00BF0020AEE7000017
:10BDA000307700202DE9F04782460C4690461D462C
:10BDB000DDF8209000260027E0B2C0F58077AF4282
:10BDC00000D92F46504600F04DF900B147E05046EB
:10BDD00000F0C1F900B142E05046FFF729FF002210
:10BDE0000221504600F02EF900B13BE00022C4F3DE
:10BDF0000741504600F026F900B133E00022C4F3B9
:10BE00000721504600F01EF900B12BE0E1B20022FC
:10BE1000504600F017F900B124E0002608E018F8B9
:10BE200006100022504600F00DF900B11AE0761C11
:10BE3000BE42F4D35046FFF7E7FE504600F07AF9D1
:10BE400000B10CE0504600F00DF900B107E0B9F187
:10BE5000000F01D0C9F800700020BDE8F0874FF056
:10BE6000FF30FAE75046FFF7CFFE4FF0FF30F4E720
:10BE700030B500EB8004074D05EBC404241D44F8E5
:10BE8000312000EB800405EBC404241D04EBC10445
:10BE9000A38030BD307700202DE9F04180460E466A
:10BEA00014461F4600254046FFF7C2FE002203212C
:10BEB000404600F0C7F800B128E00022C4F3074173
:10BEC000404600F0BFF800B120E00022C4F3072193
:10BED000404600F0B7F800B118E0E1B20022404659
:10BEE00000F0B0F800B111E0002507E07219FF2161
:10BEF000404600F0A7F800B108E06D1CBD42F5D344
:10BF00004046FFF781FE0020BDE8F0814046FFF784
:10BF10007BFE4FF0FF30F7E72DE9F04107460D4675
:10BF2000164600243846FFF783FE00229F2138463C
:10BF300000F088F800B111E0002407E02A19FF2181
:10BF4000384600F07FF800B108E0641CB442F5D335
:10BF50003846FFF759FE0020BDE8F0813846FFF76C
:10BF600053FE4FF0FF30F7E770B506460C4600254C
:10BF70003046FFF75DFE00220521304600F062F8F2
:10BF800005462DB92246FF21304600F05BF80546F4
:10BF90003046FFF739FE284670BD000000EB8002F6
:10BFA000014B03F8321070473077002070B5064619
:10BFB0000C461546214850F82500401E8443304663
:10BFC00000F0C9F800B130E03046FFF731FE1C4800
:10BFD000415D0022304600F035F800B128E0002233
:10BFE000C4F30741304600F02DF800B120E00022F4
:10BFF000C4F30721304600F025F800B118E0E1B2A3
:10C000000022304600F01EF800B111E03046FFF784
:10C01000FBFD304600F08EF800B106E0304600F03F
:10C0200021F800B101E0002070BD4FF0FF30FBE7C8
:10C030003046FFF7E9FD4FF0FF30F5E7D82303085E
:10C04000E423030837B50446154604EB8401044A8B
:10C0500012F83100012301AA294600F0A1F83EBDE3
:10C060003077002038B5054600240020009000BF3E
:10C0700069462846FFF778FF044604B105E09DF8BD
:10C08000000000F001000028F2D100BF204638BDBA
:10C090002DE9FC4104460D4617461E464FF00008A8
:10C0A0000020019004EB8400214901EBC000406AAC
:10C0B000A84201D907B11EB94FF0FF30BDE8FC819D
:10C0C00004EB84001A4901EBC000416A04EB8400D0
:10C0D000174A02EBC000406A401E2840081AB042CE
:10C0E0000DD204EB8400114601EBC000416A04EB61
:10C0F000840002EBC000406A401E28400E1A13E084
:10C1000001A833463A46294600902046FFF74AFEEA
:10C1100010B14FF0FF30D1E7019805440198074472
:10C120000198361A01988044002EE9D10020C5E715
:10C130003077002070B5044600252046FFF778FDD3
:10C14000002204212046FFF77DFF05462046FFF729
:10C150005BFD284670BD70B5044600252046FFF7FC
:10C1600067FD002206212046FFF76CFF05462046AA
:10C17000FFF74AFD284670BDF8B504460D46164641
:10C180002B46002280212046009600F02DF828B191
:10C19000606D40F0200060650320F8BD0020FCE7E2
:10C1A000F8B506460D4617461C462DB922463946B7
:10C1B000304600F06FF8F8BD642104FB01F0A3B233
:10C1C0000449009051F826002A463946FAF77FFCC8
:10C1D0000020F0E7240600200246024840F8221022
:10C1E00000207047240600202DE9F04104460E4649
:10C1F00017461D46DDF818803FE0681CE0B32DB1FE
:10C20000F9F7BAFDA0EB0800A84236D320684068D1
:10C2100020F0E000216848606068B0F5827F0DD1B1
:10C22000A068B0F5004F03D0A068B0F5806F05D1CD
:10C230002068006820F0400021680860A06AB0F51E
:10C24000005F0ED100BF206800684DF6FF71084006
:10C25000216808602068006840F400502168086088
:10C2600000BF012084F8510000BF002084F8500076
:10C2700000BF0320BDE8F081FFE720688068304000
:10C28000B04201D1012000E00020B842B5D1002029
:10C29000F0E7000070B505460E461446642104FB25
:10C2A00001F3A2B2034951F825003146FAF73CFBED
:10C2B000002070BD240600207047000038B50446F9
:10C2C0000D460020009055201B490870AA20487098
:10C2D00003208870601DC8700320087108464571EE
:10C2E0008471164800EB450122461348C01DF3F740
:10C2F000AEFF002008E0811C0F4A515CBDF8002011
:10C30000114489B20091401C611D8842F3DB0A4848
:10C31000801CF5F79BFA0090E01D07490844BDF822
:10C32000001001804FF47A7304F1090202490448B5
:10C33000FBF7C5FC38BD00006C240020E81F00207E
:10C34000A0DD002008B50948094B0A4A4FF4806176
:10C3500000900948FDF781FB084908600846064936
:10C3600002680748006801F029FB08BD1DBC0020D9
:10C37000DCBB0020603503089DBC00207405002054
:10C380006005002010B5084B084A4FF4806108484A
:10C39000FDF763FB0749086008460549026806483F
:10C3A000006801F00BFB10BD1DBC0020E434030845
:10C3B0009DBC00207405002060050020F0B50746F4
:10C3C0000C4615461E4672B6FFF756FB3846FFF779
:10C3D0005FFB2046FFF75CFB2846FFF759FB304622
:10C3E000FFF756FB62B6F0BD10B50446062C0BDA1B
:10C3F000064850F82420064B1B7850F8231005A05F
:10C40000FCF70EF802480470002010BD8C050020D7
:10C410005C050020436C69656E745374617465201B
:10C4200066726F6D205B25735D206368616E676562
:10C4300020746F205B25735D0D0A000070B5044603
:10C440000D46022C0FD0FCF7F1FF50B1FCF7EEFFC8
:10C45000D0F8900528B1FCF7E9FFD0F8906504A06A
:10C46000B047002070BD6868FEF75CFB0020F9E76C
:10C470004552524F520D0A0070B505460E46022035
:10C48000FEF738FBFCF7D2FF50B1FCF7CFFFD0F836
:10C49000900528B1FCF7CAFFD0F8904501A0A0474D
:10C4A000002070BD4F4B0D0A000000002DE9F04147
:10C4B00005460E46022D0DD0FCF7B8FF50B1FCF733
:10C4C000B5FFD0F8900528B1FCF7B0FFD0F8907513
:10C4D00029A0B8477068F3F740FF04469CB90020D4
:10C4E000F5F742FBFCF7A2FF002842D0FCF79EFFC5
:10C4F000D0F8900500283CD0FCF798FFD0F8907554
:10C5000020A0B84735E0012C11D1FCF78FFF50B1C6
:10C51000FCF78CFFD0F8900528B1FCF787FFD0F826
:10C52000907518A0B8470120F5F71EFB21E0022CFA
:10C5300011D1FCF77BFF50B1FCF778FFD0F89005E4
:10C5400028B1FCF773FFD0F890750EA0B847022011
:10C55000F5F70AFB0DE0FCF769FF50B1FCF766FF49
:10C56000D0F8900528B1FCF761FFD0F8907503A0D2
:10C57000B8470020BDE8F081417267204552524F14
:10C58000520D0A004F4B0D0A000000002DE9F0414A
:10C5900080460D466868F3F7E0FE04464FF47A7073
:10C5A000B4FBF0F001036420B4FBF0F00A22B0FB0E
:10C5B000F2F302FB130001EB0021B4FBF2F0B0FB3D
:10C5C000F2F302FB130001EB00101146B4FBF1F291
:10C5D00001FB124146180C498E80084680880B49A1
:10C5E000086005F08BFDFCF721FF50B1FCF71EFF42
:10C5F000D0F8900528B1FCF719FFD0F8907504A089
:10C60000B8470020BDE8F081E81F0020CC010020E1
:10C610004F4B0D0A0000000070B504460E46022C78
:10C6200010DAFCF703FF50B1FCF700FFD0F89005DB
:10C6300028B1FCF7FBFED0F8905503A0A8474FF0B7
:10C64000FF3070BD0020FCE764656275675F6F6650
:10C650006620666C61670D0A0000000070B5044634
:10C660000E46022C10DAFCF7E1FE50B1FCF7DEFEBC
:10C67000D0F8900528B1FCF7D9FED0F8905503A06A
:10C68000A8474FF0FF3070BD0020FCE7646562757D
:10C69000675F6F6E20666C61670D0A002DE9F041DF
:10C6A00005460E46022D0DD0FCF7C0FE50B1FCF73A
:10C6B000BDFED0F8900528B1FCF7B8FED0F8907513
:10C6C00011A0B8477068F3F748FE0446C4F30F2082
:10C6D0001049A1F85200A1F8544005F00FFD214681
:10C6E000022003F009FBFCF7A1FE50B1FCF79EFE0F
:10C6F000D0F8900528B1FCF799FED0F8907506A007
:10C70000B8470020BDE8F081417267204552524F82
:10C71000520D0A00E81F00204F4B0D0A00000000D8
:10C720002DE9F04106460F46FCF780FE58B1FCF7B4
:10C730007DFED0F8900530B1FCF778FE1EA1D0F850
:10C74000904520A0A047FCF771FE70B1FCF76EFE8B
:10C75000D0F8900548B1FEF789F90546FCF766FE6A
:10C760002946D0F890451DA0A047FCF75FFE70B1A8
:10C77000FCF75CFED0F8900548B1FEF773F905466A
:10C78000FCF754FE2946D0F890451AA0A047FCF7C4
:10C790004DFE70B1FCF74AFED0F8900548B1FEF7A7
:10C7A00069F90546FCF742FE2946D0F8904517A0E6
:10C7B000A0470020BDE8F0815632303231303531AB
:10C7C0003030300056657273696F6E3A2020202039
:10C7D000202020202025730D0A000000494D4549E6
:10C7E0003A20202020202020202020202025730DEA
:10C7F0000A000000434349443A2020202020202002
:10C80000202020202025730D0A000000494D5349A7
:10C810003A20202020202020202020202025730DB9
:10C820000A00000010B522210248FCF779FD002023
:10C8300010BD0000A422030870B504460E46022C69
:10C8400010D0FCF7F3FD50B1FCF7F0FDD0F89005E7
:10C8500028B1FCF7EBFDD0F890550AA0A8474FF09F
:10C86000FF3070BDFCF7E2FD50B1FCF7DFFDD0F802
:10C87000900528B1FCF7DAFDD0F8905506A0A8473E
:10C880000020EEE775736167653A206C6F6720736F
:10C890007472696E670D0A004F4B0D0A00000000AC
:10C8A00070B505460E46FCF7C1FD50B1FCF7BEFD64
:10C8B000D0F8900528B1FCF7B9FDD0F8904502A05A
:10C8C000A047002070BD00004F4B0D0A0000000083
:10C8D0002DE9F04104460F460026032C11D0FCF749
:10C8E000A5FD50B1FCF7A2FDD0F8900528B1FCF7EA
:10C8F0009DFDD0F8905504A0A8474FF0FF30BDE84B
:10C90000F0810020FBE7000075736167653A206CD9
:10C910006F675F7072696E74206173635B302D3175
:10C920005D20636E740D0A0002460020704700000F
:10C93000F8B505460C46022D10D0FCF777FD50B136
:10C94000FCF774FDD0F8900528B1FCF76FFDD0F826
:10C9500090651AA0B0474FF0FF30F8BD4CF6CC40C0
:10C9600000901BA0FBF75CFD002302224FF48831EE
:10C970001846FFF771F902236A464FF48831002008
:10C98000FFF786FB00234FF480724FF49031184676
:10C99000FFF762F96068F3F7A6FC461C33464FF4D4
:10C9A000903100206268FFF773FB0A2004F0F1FB6E
:10C9B0000020FFF7A5F80020CFE70000757361673E
:10C9C000653A206F74612075726C0D0A00000000DA
:10C9D000676F746F206F7461206170706C69636140
:10C9E00074696F6E0D0A000070B505460E46022090
:10C9F000FEF78CF8FCF71AFD50B1FCF717FDD0F8E4
:10CA0000900528B1FCF712FDD0F8904501A0A04791
:10CA1000002070BD4F4B0D0A0000000070B50546A8
:10CA20000E460020FEF766F8FCF700FD50B1FCF75B
:10CA3000FDFCD0F8900528B1FCF7F8FCD0F8904543
:10CA400001A0A047002070BD4F4B0D0A0000000060
:10CA500070B505460E460020FEF758F8FCF7E6FCD8
:10CA600050B1FCF7E3FCD0F8900528B1FCF7DEFCF0
:10CA7000D0F8904501A0A047002070BD4F4B0D0A93
:10CA80000000000070B504460E46022C10D0FCF7E2
:10CA9000CDFC50B1FCF7CAFCD0F8900528B1FCF7EA
:10CAA000C5FCD0F890550AA0A8474FF0FF3070BDE4
:10CAB000FCF7BCFC50B1FCF7B9FCD0F8900528B1EC
:10CAC000FCF7B4FCD0F8905508A0A8470020EEE78A
:10CAD00075736167653A207274635F7365745F6133
:10CAE0006C61726D207365630D0A00004F4B0D0A77
:10CAF00000000000024600207047000070B50446A8
:10CB00000E46072C10D0FCF791FC50B1FCF78EFCC0
:10CB1000D0F8900528B1FCF789FCD0F8905503A017
:10CB2000A8474FF0FF3070BD0020FCE775736167C8
:10CB3000653A207274635F7365742079797979201E
:10CB40006D6D206464206868206D6D2073730D0A1C
:10CB50000000000070B504460D460020FEF7D0FF2F
:10CB6000002070BD2DE9F04107460E46032F0DD081
:10CB7000FCF75CFC50B1FCF759FCD0F8900528B1EB
:10CB8000FCF754FCD0F890851FA0C0477068F3F7FD
:10CB9000E4FB0446B068F3F7E0FB0546142C22DC06
:10CBA000002C20DD322D1EDC002C1CDD1949A1F8E3
:10CBB00070404FF47A7090FBF5F0C88005F09EFA53
:10CBC000FCF734FC50B1FCF731FCD0F8900528B1EB
:10CBD000FCF72CFCD0F890850FA0C04701200D4930
:10CBE000A1F860000DE0FCF721FC50B1FCF71EFC41
:10CBF000D0F8900528B1FCF719FCD0F8908502A078
:10CC0000C0470020BDE8F081417267204552524F75
:10CC1000520D0A00E81F00204F4B0D0A00000000D3
:10CC200070B505460C46062D10DAFCF7FFFB50B137
:10CC3000FCF7FCFBD0F8900528B1FCF7F7FBD0F827
:10CC400090651EA0B0474FF0FF3070BD1DA220219F
:10CC50001D48636803F0D8FCA068FCF736FF1B4949
:10CC6000A1F8A00217A2202117482230E36803F0A0
:10CC7000CBFC14A2202114484230236903F0C4FCE9
:10CC800010A2202110486230636903F0BDFC05F05A
:10CC900035FAFCF7CBFB50B1FCF7C8FBD0F8900598
:10CCA00028B1FCF7C3FBD0F8906509A0B04701207C
:10CCB0000649A1F860000020C7E700004552524F26
:10CCC000520D0A002573000068220020E81F002092
:10CCD0004F4B0D0A0000000070B505460C46052DAF
:10CCE00010DAFCF7A3FB50B1FCF7A0FBD0F89005DD
:10CCF00028B1FCF79BFBD0F890651BA0B0474FF024
:10CD0000FF3070BD1AA220211A48636803F07CFC32
:10CD100017A2202117482030A36803F075FC14A245
:10CD2000202114484030E36803F06EFC10A220215B
:10CD300010486030236903F067FC05F0DFF9FCF769
:10CD400075FB50B1FCF772FBD0F8900528B1FCF7E9
:10CD50006DFBD0F8906508A0B04701200849A1F804
:10CD600060000020CDE700004552524F520D0A00EE
:10CD700025730000E82100204F4B0D0A0000000041
:10CD8000E81F0020F8B505460C46022D10DAFCF726
:10CD90004DFB50B1FCF74AFBD0F8900528B1FCF7E9
:10CDA00045FBD0F8906516A0B0474FF0FF30F8BDB6
:10CDB00069466068FCF714FD6068FCF786FE12495E
:10CDC000B1F85610884205D06068FCF77EFE0E4927
:10CDD000A1F8560005F092F9FCF728FB50B1FCF7DA
:10CDE00025FBD0F8900528B1FCF720FBD0F8906522
:10CDF00006A0B04701200449A1F860000020D6E752
:10CE00004552524F520D0A00E81F00204F4B0D0AA9
:10CE100000000000F8B505460C46032D10DAFCF7BB
:10CE200005FB50B1FCF702FBD0F8900528B1FCF7E8
:10CE3000FDFAD0F8906528A0B0474FF0FF30F8BD5C
:10CE400069466068FCF7CCFC9DF800002449498CD9
:10CE5000884211D19DF801002149898C88420BD16B
:10CE60009DF802001E49C98C884205D19DF8030037
:10CE70001B49098D88420CD09DF800001849488450
:10CE80009DF8010088849DF80200C8849DF8030085
:10CE90000885A068FCF719FE1149098B884204D067
:10CEA000A068FCF712FE0E49088305F027F9FCF78D
:10CEB000BDFA50B1FCF7BAFAD0F8900528B1FCF7EA
:10CEC000B5FAD0F8906507A0B04701200449A1F851
:10CED00060000020B3E700004552524F520D0A0097
:10CEE000E81F00204F4B0D0A00000000F8B5054672
:10CEF0000C46032D10DAFCF799FA50B1FCF796FABC
:10CF0000D0F8900528B1FCF791FAD0F890652DA0E3
:10CF1000B0474FF0FF30F8BD69466068FCF760FC31
:10CF20009DF800002949B1F86610884214D19DF897
:10CF300001002649B1F8681088420DD19DF8020021
:10CF40002249B1F86A10884206D19DF803001F49B2
:10CF5000B1F86C10884210D09DF800001B49A1F870
:10CF600066009DF80100A1F868009DF80200A1F894
:10CF70006A009DF80300A1F86C00A068FCF7A5FD0D
:10CF80001249B1F86E10884205D0A068FCF79DFDEB
:10CF90000E49A1F86E0005F0B1F801200B49A1F887
:10CFA0006000FCF743FA50B1FCF740FAD0F8900566
:10CFB00028B1FCF73BFAD0F8906505A0B0470020F7
:10CFC000A9E700004552524F520D0A00E81F002009
:10CFD0004F4B0D0A00000000F8B505460C46022D27
:10CFE00010DAFCF723FA50B1FCF720FAD0F89005DC
:10CFF00028B1FCF71BFAD0F8906516A0B0474FF0A7
:10D00000FF30F8BD69466068FCF7EAFB6068FCF732
:10D010005CFD1249B1F85810884205D06068FCF7F1
:10D0200054FD0E49A1F8580005F068F8FCF7FEF928
:10D0300050B1FCF7FBF9D0F8900528B1FCF7F6F9F0
:10D04000D0F8906506A0B04701200449A1F860001F
:10D050000020D6E74552524F520D0A00E81F00202B
:10D060004F4B0D0A000000000246002070470000F0
:10D0700070B505460C461646214602A0FBF7D0F9CE
:10D0800070BD00004576656E743A25750D0A000086
:10D090002DE9F04104460D46022C0DD0FCF7C6F9EF
:10D0A00050B1FCF7C3F9D0F8900528B1FCF7BEF9F0
:10D0B000D0F8906514A0B0476868F3F74EF90746BA
:10D0C000384600F0E7F970B9FCF7B0F9C8B1FCF7E1
:10D0D000ADF9D0F89005A0B1FCF7A8F9D0F89065AB
:10D0E0000CA0B0470DE0FCF7A1F950B1FCF79EF998
:10D0F000D0F8900528B1FCF799F9D0F8906503A015
:10D10000B0470020BDE8F081417267204552524F80
:10D11000520D0A004F4B0D0A000000002DE9F047A8
:10D1200005460C46042D0DD0FCF780F950B1FCF7F4
:10D130007DF9D0F8900528B1FCF778F9D0F8908502
:10D1400018A0C0476068F3F708F98146A668E06850
:10D15000F3F703F987B23A463146484600F0E2F960
:10D1600070B9FCF763F9C8B1FCF760F9D0F8900525
:10D17000A0B1FCF75BF9D0F890850DA0C0470DE099
:10D18000FCF754F950B1FCF751F9D0F8900528B1EB
:10D19000FCF74CF9D0F8908503A0C0470020BDE80B
:10D1A000F0870000417267204552524F520D0A002D
:10D1B0004F4B0D0A00000000F8B505460E46002052
:10D1C00000900023194A0121684600F0D1F9E8B91E
:10D1D000FCF72CF958B1FCF729F9D0F8900530B1DB
:10D1E000FCF724F9D0F8904511A00099A047FCF76E
:10D1F0001DF9C8B1FCF71AF9D0F89005A0B1FCF7F9
:10D2000015F9D0F890450DA0A0470DE0FCF70EF9F8
:10D2100050B1FCF70BF9D0F8900528B1FCF706F9EE
:10D22000D0F8904507A0A0470020F8BD71D00208B3
:10D23000536F636B49443A25750D0A004F4B0D0A35
:10D24000000000004552524F520D0A002DE9F041F6
:10D2500006460C46032E0DD0FCF7E8F850B1FCF75B
:10D26000E5F8D0F8900528B1FCF7E0F8D0F8907513
:10D2700018A0B8476068F3F770F88046A56828469C
:10D28000F3F731F807463A462946404600F096FB48
:10D2900070B9FCF7CBF8C8B1FCF7C8F8D0F8900526
:10D2A000A0B1FCF7C3F8D0F890750DA0B8470DE019
:10D2B000FCF7BCF850B1FCF7B9F8D0F8900528B1EC
:10D2C000FCF7B4F8D0F8907503A0B8470020BDE88B
:10D2D000F0810000417267204552524F520D0A0002
:10D2E0004F4B0D0A0000000070B504460D460421A6
:10D2F00002A000F029FF002070BD0000B2E2CAD4F5
:10D3000000000000F8B505460E464AF6AA20009037
:10D31000FCF78CF850B1FCF789F8D0F8900528B1EB
:10D32000FCF784F8D0F890450AA0A0470023022219
:10D330004FF488311846FEF78FFC02236A464FF4FB
:10D3400088310020FEF7A4FE01200549A1F8600005
:10D350000020F8BD757064617465204F4B0D0A00A4
:10D36000E81F002070B5B2B004460E46214608A062
:10D37000FBF756F8234606A2C8216846FCF76DFB6A
:10D38000C5B22946684602F031F832B070BD0000DF
:10D390003447207369676E616C20696E74656E73C3
:10D3A0006974792069732025750D0A00F8B5054662
:10D3B0000C46164634B1012C15D0022C44D0032C57
:10D3C0005AD156E02E480078012803D02C48007826
:10D3D000042807D10020FFF707F800221146642037
:10D3E000F4F744FA49E00020264908602448007810
:10D3F000012812D1FEF7C6FF002023490870022041
:10D40000FEF7F2FF0020214B47F230520146009018
:10D410001F480068FCF7F8F815E019480078042860
:10D4200011D1FEF78FFF0020174908700320FEF787
:10D43000DBFF0020154B47F23052014600901448A4
:10D440000068FCF7E1F818E00D480078042800D1E6
:10D4500013E00F480068FCF735F80948007838B148
:10D460000020FEF7C1FF002211466520F4F7FEF907
:10D4700003E0FDF71FFD00E000BF00BFF8BD0000A6
:10D480005C050020780500205D05002069E20208A7
:10D49000640500200246C2EB8210C0EB00100A4B6C
:10D4A00003EB8001002A02DB032A00DA11B94FF0F6
:10D4B000FF307047087820B10878012801D0052096
:10D4C00008700020F5E700001078002070B50025F6
:10D4D000002400BF1FE0C5EB8510C0EB0010104911
:10D4E00001EB80042078032804D0042803D0062808
:10D4F0000ED101E000BF00BF0020A070012020700D
:10D50000A06820B102212846D4E90232984700E001
:10D5100000BF00BF6D1C032DDDDB002070BD0000CF
:10D52000107800202DE9F04104460E461746C4EB62
:10D530008410C0EB00100C4901EB8005002C02DBCD
:10D54000032C00DA1DB94FF0FF30BDE8F0813346FF
:10D5500006A22A2105F11000FCF77FFA6F8703204D
:10D5600028700020F1E700001078002025730000EB
:10D570002DE9F04707460E469046994600250024BF
:10D5800000BF38E0C5EB8510C0EB00101C4901EB73
:10D59000800474B3207860BB40F6C4612046FCF779
:10D5A000DFF86560667002202070C4F80880C4F857
:10D5B0000C9010234FF4C06204F1C40104F13C004C
:10D5C000FCF738FB012E08D10123DA0204F2C46112
:10D5D00004F1B000FAF7B9FD07E01023DA0104F214
:10D5E000C46104F16C00FCF725FB3D600020BDE840
:10D5F000F087FFE76D1C032DC4DB4FF0FF30F6E72B
:10D60000107800200146032908DAC1EB8110C0EB35
:10D610000010034A02EB80001030704701A0FCE7C5
:10D6200010780020000000000146032908DAC1EB51
:10D630008110C0EB0010034A02EB8000408F70475E
:10D640000020FCE7107800200146032908DAC1EB2E
:10D650008110C0EB0010034A02EB80003C307047A1
:10D660000020FCE7107800200146032907DAC1EB0F
:10D670008110C0EB0010034A12F820007047002010
:10D68000FCE70000107800200146032908DAC1EB0E
:10D690008110C0EB0010034A02EB80004078704715
:10D6A0000020FCE7107800200146032908DAC1EBCE
:10D6B0008110C0EB0010034A02EB800080787047B5
:10D6C0000020FCE710780020014603290ADA012037
:10D6D000C1EB8112C2EB0212044B03EB8202907089
:10D6E000002070474FF0FF30FBE70000107800206B
:10D6F0000146032909DA0020C1EB8112C2EB0212B4
:10D70000034B03EB8202907070474FF0FF30FBE752
:10D710001078002070B50546C5EB8510C0EB0010F1
:10D720000D4901EB8004002D02DB032D00DA14B952
:10D730004FF0FF3070BD2078042801D1401FF9E779
:10D7400001202070A06820B102212846D4E90232CD
:10D7500098470020EEE700001078002070B50546DD
:10D76000C5EB8510C0EB00100A4901EB8004002DC9
:10D7700002DB032D00DA14B94FF0FF3070BD072033
:10D780002070A06820B100212846D4E902329847D1
:10D790000020F3E71078002070B50546C5EB851032
:10D7A000C0EB0010184901EB8004002D02DB032DB3
:10D7B00000DA14B94FF0FF3070BD0620207010233E
:10D7C000020204F1C40104F13C00FCF733FA607872
:10D7D000012808D10123C20204F2C46104F1B0009F
:10D7E000FAF7B3FC07E01023DA0104F2C46104F194
:10D7F0006C00FCF71FFAA06820B101212846D4E98B
:10D80000023298470020D7E71078002070B5044610
:10D81000C4EB8410C0EB0010094901EB8005002C1B
:10D8200002DB032C00DA15B94FF0FF3070BDA86899
:10D8300020B103212046D5E9023298470020F5E7C0
:10D84000107800202DE9F84F0746884691461D467E
:10D850004FF0FF3000900024C7EB8710C0EB0010A2
:10D86000224901EB8006002F03DB032F01DA06B10A
:10D870001DB94FF0FF30BDE8F88F707801281BD13B
:10D880004FF0000A4FF0000B00BF0EE008EB0A015A
:10D8900006F1B000FAF780FC18B1C5F800B000201E
:10D8A000E9E70BF1010B0AF1010ACA45EED3C5F80D
:10D8B00000B00020009016E006F16C00FCF76FF954
:10D8C000044684B16068484508D24046D4E9001255
:10D8D000F2F7BDFC6068286000200090214606F148
:10D8E0006C00FCF734F90098C5E7000010780020C0
:10D8F0002DE9F047044689461546C4EB8410C0EB79
:10D900000010254901EB80060027002C02DB032CC8
:10D9100000DA1EB94FF0FF30BDE8F08770780128BB
:10D920000FD100270AE009EB070106F1B000FAF772
:10D93000EFFB10B14FF0FF30EEE77F1CAF42F2D3A8
:10D9400028E000BFC4EB8411C1EB0111124A02EBC5
:10D95000810101F16C002946FCF740F98046B8F1DD
:10D96000000F12D02A464946D8F80000F2F76FFCA3
:10D97000C4EB8411C1EB0111074A02EB810101F1F3
:10D980006C004146FCF7F7F803E0214603A0FAF7E4
:10D9900047FD00BF0020BFE710780020536F636B86
:10D9A00065745B25755D20526563762042756666F9
:10D9B00065722046756C6C0D0A0000002DE9F0417F
:10D9C0000446884615460026C4EB8410C0EB0010C0
:10D9D000134901EB8007002C03DB032C01DA07B1AC
:10D9E0001DB94FF0FF30BDE8F081294607F13C003A
:10D9F000FCF7F4F8064636B921460AA0FAF710FDFE
:10DA00004FF0FF30EFE72A4641463068F2F71FFC3F
:10DA1000314607F13C00FCF7AEF80020E3E70000D8
:10DA200010780020736F636B65745B25645D2073F1
:10DA3000656E64206275662066756C6C0D0A000068
:10DA40000246032A08DAC2EB8210C0EB0010044B36
:10DA500003F82010002070474FF0FF30FBE7000074
:10DA60001078002001460020044A126890B24FF658
:10DA7000C77210400843014A1060704700300140EF
:10DA800010B5FBF7F3FDF8F77DF9F9F75EF910BD76
:10DA900010B592B000BF002000902F48006840F001
:10DAA00080502D4908600846006800F080500090C2
:10DAB00000BF00BF00BF002000902848006820F48D
:10DAC000404040F40040254908600846006800F4E2
:10DAD0004040009000BF00BF012006900004079066
:10DAE00002200C9041050D9108210E91A0210F916B
:10DAF000022110910421119106A8F8F78BFB18B1AF
:10DB0000D22117A002F06EFD0F200190022002909A
:10DB1000002003904FF480500490002005900221D3
:10DB200001A8F8F739FA18B1E0210DA002F05AFD6A
:10DB3000F8F7F2FA4FF47A71B0FBF1F42046F9F7F6
:10DB4000EAF80420F9F7D2F800221146501EF8F73F
:10DB5000B0F912B010BD0000403802400070004023
:10DB60002E2E2F5372632F6D61696E2E630000009D
:10DB70001348006840F470001149086011480068BB
:10DB800040F001000F49086000200E49083108608C
:10DB90000C4800680C4908400A4908600B48091DF8
:10DBA0000860081F006820F48020091F086000201A
:10DBB00004490C3108600648014980390860704703
:10DBC00088ED00E000380240FFFFF6FE1030002430
:10DBD0000000020870B505460C46FBF7B9FC094980
:10DBE000086044B122462946022002F01BFA10B117
:10DBF00005A0FAF715FC214609A0FAF711FC002050
:10DC000070BD00009001002052544B2044617461AB
:10DC10002053656E64204572726F720D0A00000019
:10DC20002575422052544B20446174612053656E27
:10DC3000740D0A0010B50020044908700023044A3E
:10DC400001210448FFF794FC002010BD8C01002046
:10DC500019DD0208880100203EB5FCF708FB012809
:10DC60003FD1FBF775FC04462048007840BB2048B4
:10DC70000078D8B901201D4908701E48008D1D4943
:10DC8000C98C1C4A928CCDE9002102901948438C22
:10DC900019A24FF480611B48FBF7DFFE1548028B89
:10DCA000184919480068FFF73DFC19E0174800685B
:10DCB000201A1749884213D900200D4908700FE037
:10DCC0000A48007802280BD112480068201A42F254
:10DCD0001071884204D30F48046000200349087083
:10DCE00002E000200149087000203EBD8C010020A8
:10DCF00094010020E81F002025752E25752E25751E
:10DD00002E257500D02400208801002098010020D5
:10DD100080EE360090010020F8B506460C46174606
:10DD200034B1012C0CD0022C12D0032C26D113E0DC
:10DD300014480078012802D10020124908701EE022
:10DD400010480078012802D102200E49087016E020
:10DD500000200C49087012E00025002000906B465E
:10DD600040F2FF32084909480068FFF76BFD05469D
:10DD70001DB905480099FFF72DFF00E000BF00BF67
:10DD8000F8BD00008C010020D02400208801002074
:10DD900010B50248F9F793F910BD000064DD0020CA
:10DDA00000220268234B98420BD0B0F1804F08D07C
:10DDB000214B984205D0214B984202D0204B9842EB
:10DDC00001D1012300E000231BB122F070024B6857
:10DDD0001A43184B984214D0B0F1804F11D0164B13
:10DDE00098420ED0154B98420BD0154B984208D054
:10DDF000144B984205D0144B984202D0134B9842D2
:10DE000001D1012300E000231BB122F44072CB6852
:10DE10001A4302608B68C3620B688362054B9842A9
:10DE200001D1012300E000230BB10B69036301233F
:10DE300043617047000001400004004000080040BA
:10DE4000000C0040004001400044014000480140F7
:10DE500030B50023012404FA01F3046A9C430462F0
:10DE6000046A02FA01F52C43046230BD30B50C4659
:10DE70000021816821F47F4142EA0325254329439B
:10DE8000816030BD0A460021816821F0700142F0B6
:10DE9000070319438160704730B500240022002336
:10DEA000056A25F001050562026A4368846924F069
:10DEB000700424F003040D682C4322F002028D68E4
:10DEC0002A430D4DA84201D1012500E000256DB186
:10DED00022F00802CD682A4322F0040223F4807362
:10DEE00023F400734D692B438D692B434360846198
:10DEF0004D684563026230BD0000014030B500242A
:10DF000000220023056A25F010050562026A4368B5
:10DF1000846924F4E04424F440740D6844EA052440
:10DF200022F020028D6842EA05120F4DA84201D16D
:10DF3000012500E0002585B122F08002CD6842EA8B
:10DF4000051222F0400223F4806323F400634D693C
:10DF500043EA85038D6943EA8503436084614D6824
:10DF60008563026230BD00000000014030B500242E
:10DF700000220023056A25F480750562026A436861
:10DF8000C46924F0700424F003040D682C4322F4C7
:10DF900000728D6842EA05220E4DA84201D101258A
:10DFA00000E0002585B122F40062CD6842EA052236
:10DFB00022F4806223F4805323F400534D6943EA32
:10DFC00005138D6943EA05134360C4614D68C56359
:10DFD000026230BD0000014030B500220023002461
:10DFE000056A25F480550562036A4468C26922F413
:10DFF000E04222F440720D6842EA052223F4005305
:10E000008D6843EA0533094DA84201D1012500E09E
:10E01000002525B124F480444D6944EA8514446008
:10E02000C2614D680564036230BD0000000001401C
:10E0300030B50B46144600210022026A056A25F01D
:10E0400001050562816921F0F00141EA041122F025
:10E050000A021A438161026230BD30B50B46144694
:10E0600000210022056A25F0100505628169026A17
:10E0700021F4704141EA043122F0A00242EA031285
:10E080008161026230BD000010B50248FBF787FDD8
:10E0900010BD0000A0D4002010B504231A020349CB
:10E0A0000348FBF7C7FD002010BD0000A0D00020F2
:10E0B000A0D4002070B505460E4604200D49086026
:10E0C00006B115B94FF0FF3070BD31460A48FBF775
:10E0D00085FD044614B94FF0FF30F5E73246294676
:10E0E0002068F2F7B4F821460348FBF744FD00200E
:10E0F000EAE70000180C0240A0D4002010B5044646
:10E10000FFF7C2FFA04204D121460348FBF71FFDE1
:10E1100010BD0020FCE70000A0D4002010B502488C
:10E12000FBF73DFD10BD0000D0D8002010B5042342
:10E130001A0203490348FBF77DFD002010BD0000D3
:10E14000D0D40020D0D8002070B505460E4604215A
:10E150001248F7F703FE38B9042010491831086057
:10E160004FF4487003F015F806B115B94FF0FF30C1
:10E1700070BD31460A48FBF731FD044614B94FF033
:10E18000FF30F5E7324629462068F2F760F821466D
:10E190000348FBF7F0FC0020EAE70000000C024017
:10E1A000D0D8002010B50446FFF7B8FFA04204D134
:10E1B00021460348FBF7CBFC10BD0020FCE7000024
:10E1C000D0D8002010B50021002022E0144A135CB2
:10E1D000125C521C124C2254142B18DA114A32F8D9
:10E1E0001020104B23F811200F4A52F820200E4B1C
:10E1F00043F821200D4A32F810200C4B23F811204F
:10E200002246145C0A464B1C99B2054B9C54421C96
:10E2100090B2074A12889042D8DB054A118010BD9F
:10E22000704D0020EC4900209C4E0020C45B002073
:10E230007602002010B5044604A0FAF7F1F8002099
:10E2400008490860F3F754FB10BD00004E545249D2
:10E250005020417070205265636F6E6E6563740D5F
:10E260000A0000003802002010B5044603A0FAF7A7
:10E27000D7F808A0FBF708FD10BD00004E54524926
:10E280005020436C69656E742074696D65206F75EC
:10E29000740D0A002E2E5C464D4C5C496E746572FE
:10E2A0006E65745C4E54524950436C69656E742EB1
:10E2B000633A31383800000070B50546AC6B002079
:10E2C000E085E0842046F9F79DF970BD70B50646FB
:10E2D0000025B46B20684069C0F3C01594F839007C
:10E2E000212805D125B10020E084204600F082F8E5
:10E2F00020684069C0F3801594F83A00222805D1BF
:10E3000025B10020E085204600F054F8E06B40F095
:10E310001000E0632046F9F775F970BD70B5054649
:10E32000AC6B2868006800F48070B0B90020E0850C
:10E330002068C06820F480702168C8602068406947
:10E3400020F00100216848612068406920F0400009
:10E3500021684861202084F83A002046F9F7A8FC9B
:10E3600070BD70B50446A56B2846F9F7A7FC70BDD3
:10E3700070B50546AC6B2868006800F4807070B911
:10E380000020E0842068406920F080002168486116
:10E390002068C06840F040002168C86002E0204664
:10E3A000F9F772FD70BD70B50446A56B2846F9F704
:10E3B00071FD70BD0168C96821F490710268D16077
:10E3C0000168496921F0010102685161202180F84A
:10E3D0003A10704710B504462068C06820F040002D
:10E3E0002168C860202084F839002046F9F74CFDE8
:10E3F000002010BD0168C96821F0C0010268D16029
:10E40000202180F83910704770B5044694F83A001E
:10E41000222844D1A068B0F5805F13D1A56A206995
:10E4200040B920684068C0F308002880A06A801CBA
:10E43000A06219E020684068C0B22880A06A401C31
:10E44000A06211E0206938B920684068C1B2A26AB0
:10E45000501CA062117007E02068406800F07F0146
:10E46000A26A501CA0621170E08D401E80B2E0854F
:10E4700098B92068C06820F490702168C86020684E
:10E48000406920F0010021684861202084F83A00AA
:10E490002046F9F70DFC002070BD0020FCE70220AB
:10E4A000FAE700002DE9F0410446002520680569DF
:10E4B00025F44055E0680543206805612068C5687B
:10E4C00049F20C6085432169A068084361690843EB
:10E4D000E169084305432068C5602068456925F463
:10E4E0004075A069054320684561E069B0F5004FBB
:10E4F0007ED1C4492068884203D0C349206888423D
:10E500005DD1F7F71FFE00EBC00101EB0010616861
:10E510004900B0FBF1F06421B0FBF1F00601F7F720
:10E5200011FE00EBC00101EB001061684900B0FB77
:10E53000F1F7F7F707FE00EBC00101EB001061688F
:10E540004900B0FBF1F06421B0FBF1F000EBC00139
:10E5500001EB0010A7EB8000322101EBC000642129
:10E56000B0FBF1F000F0F80006EB4006F7F7EAFD2B
:10E5700000EBC00101EB001061684900B0FBF1F74E
:10E58000F7F7E0FD00EBC00101EB00106168490006
:10E59000B0FBF1F06421B0FBF1F000EBC00101EB46
:10E5A0000010A7EB8000322101EBC0006421B0FB1A
:10E5B000F1F000F0070030442168886020E1F7F7AF
:10E5C000B1FD00EBC00101EB001061684900B0FB38
:10E5D000F1F06421B0FBF1F00601F7F7A3FD00EBC9
:10E5E000C00101EB001061684900B0FBF1F700E0E9
:10E5F00045E0F7F797FD00EBC00101EB0010616803
:10E600004900B0FBF1F06421B0FBF1F000EBC00178
:10E6100001EB0010A7EB8000322101EBC000642168
:10E62000B0FBF1F000F0F80006EB4006F7F77AFDDA
:10E6300000EBC00101EB001061684900B0FBF1F78D
:10E64000F7F770FD00EBC00101EB001061684900B5
:10E65000B0FBF1F06421B0FBF1F000EBC00101EB85
:10E660000010A7EB8000322101EBC0006421B0FB59
:10E67000F1F000F00700304421688860C0E0614993
:10E680002068884203D06049206888425CD1F7F74F
:10E6900059FD00EBC00101EB001061688900B0FB7F
:10E6A000F1F6F7F74FFD00EBC00101EB00106168D8
:10E6B0008900B0FBF1F06421B0FBF1F000EBC00188
:10E6C00001EB0010A6EB8000322101EB0010642169
:10E6D000B0FBF1F000F0F006F7F734FD00EBC001FD
:10E6E00001EB001061688900B0FBF1F06421B0FB20
:10E6F000F1F006EB0016F7F725FD00EBC00101EB8A
:10E70000001061688900B0FBF1F7F7F71BFD00EB23
:10E71000C00101EB001061688900B0FBF1F06421D9
:10E72000B0FBF1F000EBC00101EB0010A7EB8000A3
:10E73000322101EB00106421B0FBF1F000F00F007A
:10E740003044216888605BE0F7F7ECFC00EBC00127
:10E7500001EB001061688900B0FBF1F6F7F7E2FC0D
:10E7600000EBC00101EB001061688900B0FBF1F023
:10E770006421B0FBF1F000EBC00101EB0010A6EB4F
:10E780008000322101EB00106421B0FBF1F000F0B9
:10E79000F006F7F7C7FC00EBC00101EB0010616861
:10E7A0008900B0FBF1F06421B0FBF1F006EB00163C
:10E7B000F7F7B8FC00EBC00101EB001061688900BD
:10E7C000B0FBF1F7F7F7AEFC00EBC00101EB001076
:10E7D00061688900B0FBF1F06421B0FBF1F000EB5F
:10E7E000C00101EB0010A7EB8000322101EB00100B
:10E7F0006421B0FBF1F000F00F0030442168886024
:10E80000BDE8F0810010014000140140014691F87C
:10E81000390021282CD18868B0F5805F0FD10A6AB1
:10E820001088C0F308000B685860086918B9086AB6
:10E83000801C086209E0086A401C086205E00B6A57
:10E84000581C086218780B685860C88C401E80B24B
:10E85000C88458B90868C06820F080000B68D86088
:10E860000868C06840F040000B68D860002070471E
:10E870000220FCE72DE9F04104460D461746984674
:10E88000069E21E0701CF8B12EB1F7F775FAA0EBE7
:10E890000800B04218D92068C06820F4D070216800
:10E8A000C8602068406920F001002168486120208C
:10E8B00084F8390084F83A0000BF002084F838005A
:10E8C00000BF0320BDE8F081206800682840A8420E
:10E8D00001D1012000E00020B842D3D00020F1E7B0
:10E8E0002DE9F04FBFB00746884600240020329043
:10E8F000FD49FEA0F9F794FD0822FEA13846F1F784
:10E900001DFD002870D10C2333AA2C213846FBF7BB
:10E91000BBF80446052C04D24FF0FF303FB0BDE8F1
:10E92000F08F3498FAF74DFFF5498988884259D11C
:10E93000002500263598FBF7C8F80546F048B0F8E2
:10E940007000A84203D0EE49A1F87050012631A909
:10E950003698FAF745FF9DF8C400E949B1F866100A
:10E96000884214D19DF8C500E549B1F86810884285
:10E970000DD19DF8C600E249B1F86A10884206D16F
:10E980009DF8C700DE49B1F86C10884214D001260A
:10E990009DF8C400DA49A1F866009DF8C500A1F809
:10E9A00068009DF8C600A1F86A009DF8C700A1F8AC
:10E9B0006C000020D34908703798FBF786F8D049DF
:10E9C000B1F86E10884206D03798FBF77EF8CC4934
:10E9D000A1F86E0001262EB103F090FB0120C8497A
:10E9E000A1F8600089E3FFE70822C7A13846F1F7E4
:10E9F000A5FC002846D10C2333AA2C213846FBF76E
:10EA000043F80446042C02D24FF0FF3086E73498D6
:10EA1000FAF7D7FEBA4989888842E3D1BDA1369872
:10EA2000F1F768FC0028DDDD4CF6CC403190BCA04D
:10EA3000F9F7F6FC002302224FF488311846FDF75F
:10EA40000BF9022331AA4FF488310020FDF720FB97
:10EA500000234FF480724FF490311846FDF7FCF814
:10EA60003598F1F740FC451C2B464FF490310020BF
:10EA7000359AFDF70DFB0A2002F08BFB0020FDF715
:10EA80003FF83AE30822ACA13846F1F757FC78B9D1
:10EA90000C2333AA2C213846FAF7F6FF0446032C40
:10EAA00002D24FF0FF3039E73498FAF78AFE24E3B8
:10EAB0000922A4A13846F1F741FC002853D10C23C8
:10EAC00033AA2C213846FAF7DFFF0446032C02D282
:10EAD0004FF0FF3022E73498FAF773FE88498988AF
:10EAE0008842CED19AA13598F1F704FC20B9369826
:10EAF000FAF7EBFF9849088098A13598F1F7FAFBEF
:10EB000020B93698FAF7E1FF9749087097A1359830
:10EB1000F1F7F0FB0028B4D13698F1F7E4FB054695
:10EB200029463698FFF710FB7548838890A24FF46A
:10EB300080616D48FAF791FF32906B499148329AA3
:10EB40000068FEF73BFF6E48838889A24FF480611E
:10EB50006548FAF782FF329063498A48329A006822
:10EB6000FEF72CFFC9E20A2287A13846F1F7E6FB3F
:10EB700040B9F2F7D5FE022899D15B495BA0F9F7BD
:10EB800075FCBAE2092283A13846F1F7D7FB40BBF6
:10EB900030A82EAB82A2414600903846FAF76AFEB2
:10EBA00002281DD10020DDE92E1288542E98FAF794
:10EBB00008FE53498988884212D1DDE93001FFF708
:10EBC00079FA4F4883886AA24FF480614648FAF781
:10EBD00044FF329044496B48329A0068FEF7EEFEDB
:10EBE0008BE2092273A13846F1F7A8FB60BB0C2326
:10EBF00033AA2C213846FAF747FF04463498FAF72F
:10EC0000E0FD3F49898888421DD1022C02D24FF095
:10EC1000FF3083E63598FAF758FF85B23698FAF751
:10EC200054FF86B2102D02D14B4806800BE0B5F59B
:10EC3000007F02DA324820F8156003F05FFA012005
:10EC40002F49A1F8600058E20A225DA13846F1F789
:10EC500075FB002846D10C2333AA2C213846FAF73D
:10EC600013FF04463498FAF7ACFD25498988884299
:10EC700039D1022C02D24FF0FF304FE63598FAF727
:10EC800024FF86B23698FAF720FF1FFA80FB4FA1C7
:10EC9000684601F0D1FC85B219498A880DEB050060
:10ECA0004DA101F0C9FC1FFA80F905EB090085B2FE
:10ECB000B24610E0124931F81A200DEB050047A1C9
:10ECC00001F0BAFC1FFA80F905EB090085B20AF1E0
:10ECD00001001FFA80FA0BEB06005045EADC6522C2
:10ECE00028467DE09DE09BE0D028002025730D0A9A
:10ECF0000000000024636F6E6669672C000000004E
:10ED0000E81F0020A0010020247570646174652C48
:10ED100000000000563230323130353130303000B2
:10ED2000676F746F204F5441204170706C6963614C
:10ED300074696F6E0D0A0000246765746C6F672C30
:10ED40000000000024636F6E74726F6C2C00000072
:10ED50006265657065720000040000207577625F6F
:10ED6000656E61626C6500002D00002054545300F4
:10ED70002452656365697665766F6963652C2558ED
:10ED80000D0A00009C010020247573657264617493
:10ED9000612C000024736574746F6E652C00000094
:10EDA00024736574746F6E652C25702C25700D0AA4
:10EDB0000000000024736574706172612C00000013
:10EDC0002472656164706172612C00002472657048
:10EDD0006C79706172612C0025782C0025642C0000
:10EDE000691C8DB20DF800206E222846691C8DB278
:10EDF0000DF8002064222846691C8DB20DF8002011
:10EE00000D222846691C8DB20DF800200A222846E2
:10EE1000691C8DB20DF800202946684600F0E6FA1C
:10EE20006BE11222B6A13846F1F788FA00287BD1AF
:10EE30000C2333AA2C213846FAF726FE0446062C6A
:10EE400002D24FF0FF3069E53498FAF7BAFC1FFAA6
:10EE500080FA3598FAF7B5FC80B231903698FAF717
:10EE600034FE85B23798FAF730FE86B23898FAF752
:10EE70002CFE1FFA80F9A748BDF8C4100180A648EF
:10EE80008088504502D04FF0FF3047E500204EE02B
:10EE900000EB4001A14A02EB410149889D4A1288DA
:10EEA000914205D000EB40019C4A12F81110C1B903
:10EEB0009849098800EB4002984B03EB42025180CD
:10EEC00000EB400203EB4202567000EB400203F8F5
:10EED000125000EB40011A4602EB4101A1F80490E8
:10EEE00027E01D2821D18E490A780978491C8C4BCE
:10EEF00019701E2A02DB00211A461170884A127806
:10EF000002EB4202854B03EB42025670844A1278B0
:10EF100002EB420203F8125000EB40011A4602EBEA
:10EF20004101A1F8049004E005E0411CC8B21E288C
:10EF3000AEDB00BFE1E011227AA13846F1F7FEF91D
:10EF4000E8BB0C2333AA2C213846FAF79DFD044672
:10EF5000032C02D24FF0FF30E0E43498FAF731FC92
:10EF600080B231903598FAF7B0FD85B2C8264FF0DF
:10EF700064096848BDF8C410018000204FE000EB30
:10EF80004001664A02EB41014988624A1288914277
:10EF900005D000EB4001614A12F81110D1B95D496A
:10EFA000098800EB40025D4B03EB4202518000EB0D
:10EFB000400203EB4202567000EB400200E032E0F8
:10EFC00003F8125000EB40011A4602EB4101A1F890
:10EFD000049026E01D2820D151490A780978491C5F
:10EFE0004F4B19701E2A02DB00211A4611704C4A41
:10EFF000127802EB4202494B03EB42025670484A38
:10F00000127802EB420203F8125000EB40011A465C
:10F0100002EB4101A1F8049003E0411CC8B21E2894
:10F02000ADDB00BF69E0142243A13846F1F786F951
:10F03000E8BB0C2333AA2C213846FAF725FD0446F9
:10F04000042C02D24FF0FF3068E4F6F7B3FC4FF423
:10F0500000413F48F5F718F93598F1F744F9319038
:10F06000042231A93A48F5F793FA319A521C3948EB
:10F070003599F5F78DFA4CF6CC403090AFF2603010
:10F08000F9F7CEF9002302224FF488311846FCF735
:10F09000E3FD022330AA4FF488310020FCF7F8FF8B
:10F0A00000234FF480724FF49031184600E008E0DE
:10F0B000FCF7D2FD0A2002F06CF80020FCF720FDDE
:10F0C0001BE0172224A13846F1F738F9A8B90C2320
:10F0D00033AA2C213846FAF7D7FC0446022C02D278
:10F0E0004FF0FF301AE43498FAF76BFB20490870B0
:10F0F0003498FAF766FB1F49087000200EE4000000
:10F10000247772697465706172615F616E63686FA4
:10F11000722C0000A8010020E81F0020D02C002045
:10F12000AA0100202472656164706172615F616E82
:10F1300063686F722C00000024646F776E6C6F61DF
:10F14000645F616E63686F7262696E2C000000001C
:10F150000080000800810008247365745F75706486
:10F16000617465616E63686F725F6D6F64652C00BA
:10F17000AB0100207701002070B58AB000242B4835
:10F18000007802284FD12A4800880890294890ED3D
:10F19000000B8DED060B284890ED000B8DED040B58
:10F1A000264827490968274A1278CDE900210290AC
:10F1B0002548838825A24FF480613048FAF74DFC3A
:10F1C000044600260BE02E4931F816202B49081979
:10F1D0002CA101F031FA05462C44701C86B214486B
:10F1E00000888642EFDB00260BE0274951F82620F5
:10F1F0002249081925A101F01FFA05462C44701C6C
:10F2000086B20B4800888642EFDB1C4908190022B1
:10F210001EA101F011FA05462C44224617491C484C
:10F220000068FEF7CBFB00200AB070BDA0010020F3
:10F2300076020020F8030020F00300201C75002057
:10F24000000400201E020020E81F0020246D6573CA
:10F2500073616765322C68656172742C253034786F
:10F260002C2530327525252C25642C25732C256CF6
:10F27000662C256C662C256400000000D028002038
:10F28000EC4900202C2578009C4E00202C256400A1
:10F290009C01002010B50023034A02210348FEF719
:10F2A00067F9002010BD00006DF302089C010020EA
:10F2B0003EB5FAF7DCFF012837D11E480078D8B9EF
:10F2C00001201C4908701C4800881C4909881C4AF8
:10F2D0001288CDE9002102901A4803881AA24FF43F
:10F2E00080611C48FAF7B9FB1B48028819491B4882
:10F2F0000068FEF717F91BE00E480078022817D1C6
:10F30000FAF726F9044616480068201A42F21071EE
:10F31000884209D300201349087011480460FFF7A0
:10F320002BFF00201049087002E0002001490870FE
:10F3300000203EBDA0010020B2010020B00100204D
:10F34000AE010020AC01002025752E25752E2575F7
:10F350002E257500D0280020B40100209C0100203B
:10F36000A4010020B6010020B7010020F8B5064630
:10F370000C46174634B1012C0CD0022C12D0032CB1
:10F380002AD113E016480078012802D10020144940
:10F39000087022E012480078012802D102201049AA
:10F3A00008701AE000200E49087016E000250020C1
:10F3B00000906B4640F2FF320A490B480068FEF7A6
:10F3C00041FA05463DB900200649009A885405488F
:10F3D0000099FFF785FA00E000BF00BFF8BD00000C
:10F3E000A0010020D02800209C01002070B5054617
:10F3F0000C4614480078022821D11349134A126898
:10F40000881822462946F0F722FF10480068204459
:10F410000E490860FAF79CF80D490968401AC82897
:10F420000DD3FAF795F80A490860084806490268BA
:10F4300008480068FEF7C2FA00200449086000206E
:10F4400070BD0000A001002084310020C401002014
:10F45000C80100209C01002010B5F6F7ABFA00228D
:10F460004FF410410748F6F781FC002204210648BA
:10F47000F6F77CFC642001F08CFE0020FCF740FBDA
:10F4800010BD0000000002400004024010B5024818
:10F49000F8F7BEF810BD0000A0DD002010B502484E
:10F4A000F8F7B6F810BD0000E0DD002010B5024806
:10F4B000F8F7AEF810BD000020DE002010B5FAF716
:10F4C00047F80E490968401AB0F57A7F05D3FAF774
:10F4D0003FF80A49086000F017F8FAF739F80849C8
:10F4E0000968401A0749C988884205D3FAF730F8F5
:10F4F0000349086000F03AF810BD00002402002023
:10F5000028020020E81F002010B5FEF75BFE10BDAA
:10F5100070B54FF480100F49886140F68C2001F0DF
:10F5200042FE10200B49886102F038F904460CE0D5
:10F5300002F034F90446FAF747FE2846691CCDB2BA
:10F54000142802DD04A001F04FF807488442EFD1EF
:10F5500070BD00000000024044572049442045523D
:10F56000524F522E0D0A00003001CADEF8B50021BC
:10F5700038E000202EE06B4A32F910301446421C6D
:10F5800034F91220934223DD674D35F810202546CB
:10F5900035F81050ABB2654D2C5C634E451C36F807
:10F5A000155026F810505F4E451C36F8155026F8B9
:10F5B00010505E4E451C755D35545B4E451C26F85B
:10F5C00015201EB2574F27F81560584E745500BFCE
:10F5D000421C90B2564A1278521E521A8242CADC1B
:10F5E000481C81B252480078401E8842C1DC504815
:10F5F0000078002809DD4F48006818B988204D4977
:10F60000086002E000204B4908604B4803684B4803
:10F6100002684B48016847480068FCF7CFFE444841
:10F620000078142802DD1420414908701220454951
:10F6300088703F48007800EB80000F30C8700846A3
:10F64000414909888180414800783E4988713F4896
:10F6500001880088401C3D4A108008123949C87151
:10F660003B48007808723B4800783B49097840EAFB
:10F6700041003A49097840EA81003949097840EA6D
:10F6800041103849097840EA81102E49487200201B
:10F69000087348738873C873254800780874244831
:10F6A00000784200204927481130F0F7D0FD20496A
:10F6B00009784A001E490978112303EB4101214BC7
:10F6C000C8181849F0F7C3FD19490978112202EB4F
:10F6D00081011C4A881816490A781449F0F7B7FDC9
:10F6E0001348007800EB800000F10F011548801CE2
:10F6F000F2F7ACF800900E48007800EB8000113073
:10F7000010490844BDF8001001800948007800EB5A
:10F71000800000F113010B48FAF7DEFB00200449DA
:10F720000870F8BDDC3B002084390020343E002006
:10F730001B02002064060020700600206C060020DA
:10F7400068060020B4110020CC010020180200201F
:10F750001E0200202C000020080000201A010020BA
:10F76000090000202E00002038B500200090002164
:10F770002D4802F091F800210F2001F0F3FF2B49F2
:10F7800008600846008800F4804000283AD04FF412
:10F79000804200210F2002F080F90021102001F0AA
:10F7A000E1FFC4B200222146214802F02FF8204890
:10F7B000B0F8010000901F48007850B11C48407A12
:10F7C000302806D100201B490870BDF800001A49F6
:10F7D0000880BDF8000018490988884219D1022222
:10F7E00016491348401DF0F793FD90B91048407A30
:10F7F00030280ED10120124908600D48807A114945
:10F80000087006E001F068FE0F4A00210F2002F0A8
:10F8100044F90121044802F03FF8002002F082F888
:10F82000002002F007F838BD00D023247003002028
:10F830008C5C0020AB0100207801002074030020C4
:10F84000640300206F030020009027242DE9F0417D
:10F8500004460D464FF0FF360DB1032C03DB4FF08D
:10F86000FF30BDE8F08104EB4400C0EB4410554983
:10F8700001EB80008078002874D100BF00BF04EB4A
:10F880004402C2EB44120B4603EB8202926804EB83
:10F890004403C3EB44130F4607EB8303DB681A44AE
:10F8A00004EB4403C3EB441307EB83035B685B6B1C
:10F8B0001B685B68D11A04EB4402C2EB44123B465E
:10F8C00003EB8202D2680A4404EB4403C3EB441303
:10F8D00007EB83031B69D21A04EB4403C3EB441305
:10F8E00007EB8303DB68B2FBF3F703FB1720012868
:10F8F0000DD84BD104EB4402C2EB4412314B03EB65
:10F90000820252681268126802F020025ABB04EBAD
:10F910004402C2EB44122B4B03EB820212691278B1
:10F920002A7004EB4402C2EB441203EB8202126918
:10F9300004EB4403C3EB4413224F07EB83035B69DF
:10F940009A4211D104EB4402C2EB44123B4603EB52
:10F950008202926804EB4403C3EB441307EB830376
:10F960001A6112E013E011E004EB4402C2EB44120E
:10F97000144B03EB82021269521C04EB4403C3EBE9
:10F980004413104F07EB83031A61002617E004EBC2
:10F990004400C0EB44100B4901EB80008078012843
:10F9A0000DD104EB4401C1EB4411064A02EB810185
:10F9B00001F118002946F8F7EFFB00B900263046A0
:10F9C0004FE7000000D90020024609B1032A02DBFC
:10F9D0004FF0FF30704702EB4200C0EB4210034B88
:10F9E00003EB8000406808600020F3E700D90020A6
:10F9F0002DE9F04105460C460CB1032D03DB4FF019
:10FA0000FF30BDE8F08105EB4500C0EB45105249E1
:10FA100001F82050207805EB4501C1EB45114E4A15
:10FA200002EB81014870607805EB4501C1EB45119F
:10FA300002EB8101887005EB4501C1EB451102EB3A
:10FA400081016068886005EB4501C1EB451102EB5F
:10FA50008101A068C860607838BB05EB4500C0EB49
:10FA60004510114601EB8000806805EB4501C1EBB4
:10FA7000451102EB8101086105EB4500C0EB451023
:10FA8000114601EB8000806805EB4501C1EB451193
:10FA900002EB8101C9680844401E05EB4501C1EB3A
:10FAA000451102EB8101486110E0607801280DD119
:10FAB00005EB4503C3EB4513274E06EB830303F128
:10FAC00018000123D4E90112F8F73FFB05EB4501CB
:10FAD000C1EB4511204A02EB8101E068C86205EBE9
:10FAE0004501C1EB451102EB81012069086305EB7B
:10FAF0004501C1EB451102EB8101A069086705EBE7
:10FB00004501C1EB451102EB810160694863207832
:10FB100010B1207801280DD105EB4506C6EB45163E
:10FB20000D4F07EB860606F13800D4E90423E1689F
:10FB3000FAF780F8607818B9284600F00FF808E066
:10FB40006078012802D06078022802D1284600F0AF
:10FB500083F8002055E7000000D900207CB504465A
:10FB600028E004EB4400C0EB44103A4901EB80006C
:10FB700040680068406880B20190BDF804000190C0
:10FB800000BF0020009004EB4400C0EB441001EBE8
:10FB90008000406800680068009004EB4400C0EBFF
:10FBA000441001EB8000406800684068009000BF8E
:10FBB00000BF00BF04EB4400C0EB4410254901EB3B
:10FBC000800040680068006800F008000028C8D184
:10FBD00004EB4400C0EB441001EB8000806804EBB0
:10FBE0004401C1EB44111B4A02EB8101086104EBA3
:10FBF0004400C0EB4410114601EB8000806804EB28
:10FC00004401C1EB441102EB8101C9680844401E64
:10FC100004EB4401C1EB441102EB8101486104EBA8
:10FC20004403C3EB4413154605EB83039B899AB247
:10FC300004EB4403C3EB441305EB8303996804EB23
:10FC40004403C3EB441305EB83035868F7F79CFFA9
:10FC50007CBD000000D900201CB5044628E004EB60
:10FC60004400C0EB4410234901EB80004068006869
:10FC7000406880B20190BDF80400019000BF0020F0
:10FC8000009004EB4400C0EB441001EB800040689E
:10FC900000680068009004EB4400C0EB441001EBE6
:10FCA0008000406800684068009000BF00BF00BF4F
:10FCB00004EB4400C0EB44100E4901EB80004068A7
:10FCC0000068006800F008000028C8D104EB440276
:10FCD000C2EB44120B4603EB820202F1680104EB13
:10FCE0004402C2EB441203EB820250680122F7F790
:10FCF000ADFF1CBD00D9002070B504460D4604EBD5
:10FD00004401C1EB4411114A02EB81014868F7F745
:10FD100062FC04EB4400C0EB44100C4901EB800092
:10FD20004068456004EB4401C1EB4411074A02EB13
:10FD300081014868F7F712FD10B14FF0FF3070BD38
:10FD4000204600F005F80020F9E7000000D9002067
:10FD500070B5044604EB4400C0EB4410534901EB7A
:10FD60008000807838BB04EB4400C0EB441001EB0A
:10FD70008000806804EB4401C1EB44114B4A02EB64
:10FD80008101086104EB4400C0EB4410114601EB13
:10FD90008000806804EB4401C1EB441102EB810157
:10FDA000C9680844401E04EB4401C1EB441102EB56
:10FDB0008101486123E004EB4400C0EB44103B495F
:10FDC00001EB80008078012819D104EB4403C3EBD8
:10FDD00044130D4605EB8303DA6804EB4403C3EBDD
:10FDE000441305EB8303996804EB4403C3EB44130A
:10FDF00005EB830303F118000123F8F7A6F904EBE0
:10FE00004400C0EB4410294901EB8000407840B128
:10FE100004EB4400C0EB441001EB80004078012863
:10FE20001FD104EB4405C5EB4415204E06EB8505B8
:10FE30006B6B04EB4405C5EB441506EB85052A6B9B
:10FE400004EB4405C5EB441506EB8505E96A04EBB4
:10FE50004405C5EB441506EB850505F13800F9F7B7
:10FE6000E9FE04EB4400C0EB4410104901EB8000B4
:10FE7000807818B92046FFF771FE15E004EB4400C6
:10FE8000C0EB4410094901EB80008078012808D0BC
:10FE900004EB4400C0EB441001EB800080780228A2
:10FEA00002D12046FFF7D8FE002070BD00D9002007
:10FEB00070B504460D460DB1032C02DB4FF0FF3048
:10FEC00070BD04EB4401C1EB4411084A02EB810010
:10FED0007421F9F745FC04EB4400C0EB44100349DE
:10FEE00001EB800045600020EAE7000000D9002017
:10FEF00070B50546002400BF2EE004EB4400C0EBC3
:10FF00004410174901EB80004068A84222D104EB5D
:10FF10004400C0EB441001EB8000807818B9204603
:10FF2000FFF71CFE15E004EB4400C0EB44100C4945
:10FF300001EB80008078012808D004EB4400C0EB7E
:10FF4000441001EB80008078022802D12046FFF7A0
:10FF500083FE03E0601CC4B2032CCEDB00BF70BD87
:10FF600000D9002038B50546002400BF54E004EB5A
:10FF70004400C0EB44102A4901EB80004068A842CD
:10FF800048D104EB4400C0EB441001EB80008078C2
:10FF9000012818D104EB4400C0EB441001EB8000B1
:10FFA00090F86800009004EB4401C1EB44111C4A36
:10FFB00002EB810101F118006946F8F7A9F8204623
:10FFC000FFF74AFE25E004EB4400C0EB441014495F
:10FFD00001EB8000807802281BD104EB4400C0EBC9
:10FFE000441001EB8000006F80B104EB4402C2EBCF
:10FFF00044120B4603EB820292F8680004EB4402C1
:020000040803EF
:10000000C2EB441203EB8202116F88472046FFF7D0
:1000100023FE03E0601CC4B2032CA8DB00BF38BD84
:1000200000D900202DE9F04104460F4615464FF057
:10003000000817B10DB1032C03DB4FF0FF30BDE812
:10004000F08104EB4400C0EB4410604901EB8000F8
:10005000406810B94FF0FF30F1E704EB4400C0EB0B
:1000600044105A4901EB80004078E8BB00BFF9F723
:1000700029F904EB4401C1EB4411544A02EB81011C
:1000800001F138002946F9F7A9FD064626B9F9F726
:1000900001FB4FF0FF382EE004EB4401C1EB4411AB
:1000A0004A4A02EB810101F138003146F9F763FD5C
:1000B0002A4639463068F0F7CAF804EB4401C1EB30
:1000C0004411424A02EB810101F13800F9F767FD62
:1000D0000646F9F7DFFAB3889AB204EB4403C3EBA0
:1000E0004413DFF8E8C000E006E00CEB830331685E
:1000F0005868F7F74FFE66E004EB4400C0EB44108D
:10010000324901EB80004078012843D100BFF9F764
:10011000D9F804EB4401C1EB44112C4A02EB8101F4
:1001200001F138002946F9F759FD064626B9F9F7D5
:10013000B1FA4FF0FF382CE004EB4401C1EB44115D
:10014000224A02EB810101F138003146F9F713FD33
:100150002A4639463068F0F77AF804EB4401C1EBDF
:1001600044111A4A02EB810101F13800F9F717FD39
:100170000646F9F78FFAB3889AB204EB4403C3EB4F
:100180004413DFF848C00CEB830331685868F7F775
:100190004FFE18E004EB4400C0EB44100B4901EBA8
:1001A0008000407802280ED1642105FB01F3AAB239
:1001B00004EB4401C1EB4411044E06EB8101486895
:1001C0003946F7F77CFD404639E7000000D90020AA
:1001D0002DE9F0410646002400BF88E004EB44000E
:1001E000C0EB4410454901EB80004068B0427CD12F
:1001F00004EB4400C0EB441001EB8000407898BB56
:1002000000BF04EB4401C1EB44113C4A02EB810105
:1002100001F13800F9F7C3FC054604EB4401C1EBDA
:100220004411364A02EB810101F138002946F9F701
:100230008EFC04EB4401C1EB4411304A02EB810116
:1002400001F13800F9F7ABFC054665B1AB889AB20D
:1002500004EB4403C3EB4413284F07EB83032968E3
:100260005868F7F797FD3EE0FFE704EB4400C0EB6A
:100270004410224901EB80004078012833D100BFAF
:1002800004EB4401C1EB44111C4A02EB810101F172
:100290003800F9F784FC054604EB4401C1EB441136
:1002A000164A02EB810101F138002946F9F74FFCAB
:1002B00004EB4401C1EB4411104A02EB810101F14E
:1002C0003800F9F76CFC054665B1AB889AB204EBCF
:1002D0004403C3EB4413094F07EB830329685868B1
:1002E000F7F7A6FD00BF05E0FFE7601CC4B2032CD2
:1002F000FFF674AF00BFBDE8F081000000D9002018
:1003000038B50446622C0CD100201549A1F86200D2
:10031000088001F0F3FE13A11AA000F065F9FFF7C1
:100320009BF8642C1BD14AF6AA20009000230222DD
:100330004FF488311846FBF78FFC02236A464FF4CE
:1003400088310020FBF7A4FE0A20F5F77DFA11A101
:100350000CA000F049F90020FBF7D2FB00BF38BD2C
:10036000E81F00202E2E5C41504C5C736572696161
:100370006C5F61745F636D645F6170702E633A35AA
:100380003500000025732055525452657374617214
:10039000740000002E2E5C41504C5C7365726961E4
:1003A0006C5F61745F636D645F6170702E633A3679
:1003B0003700000000BFFEE770B504460025644822
:1003C000007808285AD100BF002004E06149095C88
:1003D00029448DB2401C60490978491F8142F5DCEF
:1003E0005E480078284485B25B480078284485B28E
:1003F0005B480078284485B25A480078284485B282
:1004000059480078284485B26019C0B2FF282BD122
:100410005248007801281DD0022823D15048007886
:10042000FFF76EFF51494E4A127888184D490A78F5
:100430004849EFF70CFF4A480078602803DB48483A
:100440000078642805DD01F059FE01204749A1F834
:10045000600008E042480078411042480078FBF70D
:100460002DFF00E000BF00BF0020394908703C4963
:100470000870394908703E49087067E034480078D0
:10048000072812D133483A4909784454384800784B
:10049000401C3749087030480078401F097888426E
:1004A00054D108202A49087050E0294800780628CD
:1004B00005D12C48047007202549087046E02448DF
:1004C0000078052805D126480470062020490870C8
:1004D0003CE01F480078042805D12048047005201E
:1004E0001B49087032E01A480078032808D11A48DE
:1004F000047000201A49087004201549087025E08E
:100500001348007828B9552C03D1012010490870F0
:100510001CE00F480078012805D1AA2C03D1022045
:100520000B49087012E00A480078022807D1032C12
:1005300005D10320064908700B48047006E000202E
:1005400003490870064908700349087070BD00002F
:100550008001002008240020820100208501002065
:10056000830100208101002084010020E81F002079
:100570008601002010B502211348F5F7EFFBC8B93A
:10058000F8F7E6FF11490968401A40F6B831884289
:100590000DD902200E49088001200E4908700E492D
:1005A00008700E490870F8F7D3FF08490860F8F79B
:1005B000CFFF07E0F8F7CCFF04490860F8F7C8FF61
:1005C0000749086010BD000000040240240000201C
:1005D00004000020B70100202C000020B6010020FC
:1005E0002800002000BFFEE70FB4054B10B503A99B
:1005F000044A029800F026FA10BC5DF814FB0000D3
:10060000B11B03087C0900200FB41CB50246002072
:1006100007AC00290BD0491ECDE90021054B6A46E5
:100620002146069800F00EFA009A002111701CBCB9
:100630005DF814FB731103080FB4084B10B504A93F
:1006400002AA039800F0FEF9044602A9002000F077
:100650009BFD204610BC5DF814FB000089110308C7
:100660007CB5044600201D46164600290BD0491EC5
:10067000CDE90041044B6A462946304600F0E2F9D4
:10068000009A002111707CBD731103080048704767
:10069000800900202DED020B019820F00040019010
:1006A0009DED000B02B0704700B583B09FED060BC7
:1006B0000A4601468DED000B6846F0F7A2F89DED65
:1006C000000B03B000BD00000000000000000000AF
:1006D00002E008C8121F08C1002AFAD1704770470B
:1006E000002001E001C1121F002AFBD1704708B5AC
:1006F000002000906B46012202212C2001F0E5F938
:10070000022000906B46012202212C2001F0DDF92D
:1007100008BD38B504466D2000906B46012240F6B6
:1007200006012E2001F0D1F93CB140F2076241F6FA
:1007300006012E2001F09EF906E041F2076241F623
:1007400006012E2001F096F938BD38B504466B46F7
:1007500002220021362001F027F80E2C57D2DFE8C4
:1007600004F011071A56565656233256563F464D38
:1007700000208DF800009DF8010000F0FE008DF8CB
:10078000010045E09DF8000000F0FC0040F0010091
:100790008DF800003CE09DF8000000F0FC0040F007
:1007A00002008DF8000033E09DF8000000F0B30077
:1007B00040F048008DF800009DF8010040F08000F6
:1007C0008DF8010024E09DF8000000F0B3008DF8E2
:1007D00000009DF8010000F07F008DF8010017E097
:1007E0009DF8010040F002008DF8010010E09DF836
:1007F000010000F0FD008DF8010009E09DF8000007
:1008000000F0CF0040F020008DF8000000E000BFB5
:1008100000BF6B4601220021362001F056F90DF190
:10082000010301221146362001F04FF938BD08B509
:1008300003208DF8010001208DF800006B46022294
:100840000021362001F041F94FF4004206212D200D
:1008500001F010F9012000F09CFC0120FFF775FF6A
:1008600008BD38B50446200A8DF80100E0B28DF8C5
:1008700000006B46022204212D2001F026F90320FE
:100880008DF800006B46012206212D2001F01DF994
:1008900000208DF800006B46012206212D2001F07A
:1008A00014F90A212D2000F05DFF0546284638BDC9
:1008B0002DE9FF5F82B00021DDE90430020DDDF893
:1008C00040B0034318D044F61050A2F2FF32424326
:1008D0001514119801281FD0A5EB0B00401C5FEAEE
:1008E000000A4FF000064E4FDFF83891B0465046F0
:1008F00015D5CAF1000413E0119801244AA3012878
:1009000001D16FEA0B010298119AC0E90031C0E9E8
:10091000024206B0BDE8F09FCBF10000DFE70446DD
:100920000021404A491842EB0450CDE9001012E082
:10093000E00707D032463B4640464946EFF7C1FD47
:100940008046894632463B4610461946EFF7B9FDC8
:1009500006460F466410002CEAD1DDE90401DDE90A
:100960000023BAF1000F06DAEFF7ABFD42464B4623
:10097000EFF7A7FD05E0EFF716FE42464B46EFF70F
:1009800012FE04460E460022284BEFF7B3FE03D8B2
:100990004FF0FF30014607E00022254B204631464C
:1009A000EFF7E8FCF0F72CF8102409E0002C0ADB44
:1009B0000A220023EFF70AFC039B30321A55641E0B
:1009C00050EA0102F2D1641C039AC4F111031444E9
:1009D000119A012A03D0012208430DD10AE00843ED
:1009E00004D000204FF0110B119072E7A3EB0B0520
:1009F0006D1E0DE05B4504DD4FF0000205F10105C1
:100A000004E003DA4FF00002A5F10105002AECD062
:100A100002981199C0E90231C0E9004579E7000068
:100A2000000014400000F03F300000000000F043E0
:100A30000000E03F30380A2801D201207047002032
:100A4000704700002DE9FF4F95B09B46894606464A
:100A500000250FE2252877D100242746F84A0121F6
:100A6000059400E0044316F8013F203B01FA03F02F
:100A70001042F7D130782A2811D06FF02F03307848
:100A8000A0F13002092A16D8059A44F0020402EBBC
:100A9000820203EB42021044761C0590EFE759F8FE
:100AA000042B0592002A03DA504244F400540590C6
:100AB00044F00204761C30782E2816D116F8010F67
:100AC00044F004042A280DD06FF02F023078A0F1F2
:100AD0003003092B09D807EB870302EB4303C71840
:100AE000761CF3E759F8047B761C30786C280FD01D
:100AF00006DC4C2817D068280DD06A2814D104E0F1
:100B0000742810D07A280FD10DE044F400140AE0C4
:100B100044F4801401E044F440147278824202D11B
:100B200004F58014761C761C307866280BD013DC14
:100B3000582877D009DC002875D04528F6D04628FB
:100B4000F4D047281AD19DE118E0632835D06428F5
:100B500079D0652812D195E1702873D008DC672818
:100B6000F1D069286FD06E280DD06F2806D1B5E07E
:100B700073282CD0752875D0782874D05A461799C8
:100B800090476D1C75E1C4F30250022809D0032878
:100B90000DD0D9F8001004280DD00D6009F104091A
:100BA00067E1D9F80010EA17C1E90052F6E7D9F871
:100BB00000100D80F2E70D70F0E719F8041B8DF8B6
:100BC000001000208DF80100EA46012003E059F8EA
:100BD00004AB4FF0FF3061074FF0000102D40DE08D
:100BE00008F101018846B9420FDA8045F8DB1AF8AE
:100BF00008100029F4D108E008F10101884681427B
:100C0000FADB1AF808100029F6D105985B46A0EB2C
:100C1000080721463846179A00F094FA284400EB5A
:100C2000080507E04DE029E10DE01AF8010B5A46EE
:100C300017999047B8F10108F7D25B46214638462C
:100C4000179A13E142E00A220092C4F302524FF0D5
:100C5000000A022A08D059F804CB032A4FEAEC71A3
:100C60000AD00DE029E02AE009F1070121F007028E
:100C7000F2E802C1914609E00FFA8CFC4FEAEC71F0
:100C8000042A03D14FFA8CFC4FEAEC71002907DAF1
:100C90000A460021DCF1000C61EB02012D2202E08A
:100CA000220504D52B228DF80420012203E0E2075F
:100CB00001D02022F7E7904659E00A2102E01022F5
:100CC0000DE010214FF0000A00910BE010224FF0D0
:100CD000000A44F004040827009203E008224FF0C1
:100CE000000A0092C4F30252022A05D059F804CB3C
:100CF0000021032A08D009E009F1070121F00702C9
:100D0000F2E802C1914605E01FFA8CFC042A01D1E9
:100D10000CF0FF0C4FF00008220728D5702806D0F1
:100D2000009B83F0100353EA0A0305D00EE0402233
:100D30008DF80420012208E05CEA010206D030228E
:100D40008DF804208DF8050002229046009B83F068
:100D5000080353EA0A030AD15CEA010201D16207DF
:100D600005D530228DF804204FF001087F1E582849
:100D700004D034A003900EA802900DE036A0F9E74D
:100D800053466046009AEFF721FA84460398825C46
:100D90000298401E029002705CEA0100F0D10298B5
:100DA00006A9081A00F1200A600702D524F480344D
:100DB00000E00127574502DDA7EB0A0000E0002014
:100DC00000EB0A01009005984144401A0590E003A9
:100DD00006D45B462146179A059800F0B3F90544FE
:100DE000002706E001A85A46C05D179990476D1C80
:100DF0007F1C4745F6DBE0030CD55B462146179A7E
:100E0000059800F09FF9054404E030205A461799F0
:100E100090476D1C0099481E00900029F5DC08E001
:100E2000029802995A460078491C029117999047F6
:100E30006D1CBAF10001AAF1010AF1DC65E10000C4
:100E400009280100303132333435363738396162A0
:100E50006364656600000000303132333435363764
:100E600038394142434445460000000000F058F93B
:100E70000544761C307800287FF4ECAD19B0284684
:100E8000BDE8F08F620700D4062709F1070222F0BF
:100E9000070CFCE80223E14603F000485FEA080C77
:100EA00002D00FF2702C0DE05FEA045C02D50FF265
:100EB000682C07E05FEAC47C02D00FF2602C01E0EE
:100EC000AFF2700C4FF0FF3823F00043CDF850C064
:100ED00065280CD006DC452809D046281DD04728B7
:100EE0003DD13DE0662818D067287ED138E000214A
:100EF000112F01DB112000E0781CCDE9000106A9CB
:100F00000EA8FFF7D5FCDDE90F010E9A0391002131
:100F1000009207F1010A04914DE04FF00040009764
:100F2000CDE9011006A90EA8FFF7C2FCDDE90F020A
:100F300003920E9B11990022DDF80CA000930492FD
:100F400011B9791C00EB010AB7EB0A0004D4C0F117
:100F5000FF3007F1010A0490AAEB0700019044E07A
:100F6000012F00DA01270021112F01DD112000E0FF
:100F70003846CDE9000106A90EA8FFF799FCDDE986
:100F80000F010E9A0391002104910092BA462107A5
:100F90000CD40399514500DA8A46BAF1010F05DDF8
:100FA000009AAAF10101515C302908D0B84202DA56
:100FB00010F1040F06DA0121CDE9011015E0AAF1C4
:100FC0000101E9E7002805DC049901440491AAEB3A
:100FD000000102E0411C514500DD8A460499401A97
:100FE000401C01904FF000400290200704D401986B
:100FF000504501DBCDF8048000208DF84F000298A9
:101000000DF14F07B0F1004F25D02B200E90029824
:101010004FF0020800280CDA404202902D200E907A
:1010200007E00A210298EFF799FB3031029007F8A8
:10103000011DB8F10001A8F10108F2DC02980028B6
:10104000EFD1791E0E980870307800F0200040F043
:10105000450007F8020D12A8C01B00F107081498FC
:10106000007800B1012000EB0A01019801EBE0716A
:1010700005984144401A401E0590E00306D45B46A3
:101080002146179A059800F05DF8054414980078F9
:1010900018B15A46179990476D1CE00324D55B465A
:1010A0002146179A059800F04DF805441CE0049875
:1010B000002807DBDDE90301884203DD0098405C7E
:1010C000179901E0179930205A469047049805F186
:1010D0000105401C04900198401E019004D12E206F
:1010E0005A46179990476D1CBAF10001AAF1010AFE
:1010F000DDDC05E017F8010B5A46179990476D1C87
:10110000B8F10001A8F10108F4DC5B462146179A0A
:101110000598ABE62D0000002B0000002000000029
:101120002DE9F041044600251E461746880404D4E4
:1011300005E039462020B0476D1C641EF9D52846CD
:10114000BDE8F0812DE9F041044600251E46904699
:10115000C80301D5302700E02027880404D505E026
:1011600041463846B0476D1C641EF9D52846BDE897
:10117000F0814A68002A06D00A68531C0B60107080
:101180004868401E486070470A68531C0B60107026
:10119000704710B503464FF47A7003FB00F4204605
:1011A00000F001F810BD002100BF40E000BF00BF0B
:1011B00000BF00BF00BF00BF00BF00BF00BF00BF37
:1011C00000BF00BF00BF00BF00BF00BF00BF00BF27
:1011D00000BF00BF00BF00BF00BF00BF00BF00BF17
:1011E00000BF00BF00BF00BF00BF00BF00BF00BF07
:1011F00000BF00BF00BF00BF00BF00BF00BF00BFF7
:1012000000BF00BF00BF00BF00BF00BF00BF00BFE6
:1012100000BF00BF00BF00BF00BF00BF00BF00BFD6
:1012200000BF00BF00BF00BF00BF00BF491C81421C
:10123000BCD370472DE9F84F04464FF00009CA4669
:1012400025786079824931F810806078401E8149A4
:10125000C6B20863042D01D0072D01D1012000E0A2
:101260000020834620787B490873E07938B9084626
:10127000806940F4800088614FEAE80805E075481D
:10128000806920F4800073498861207A714948732D
:1012900008468069217A4FF4403202EA014108434E
:1012A0006C498861084600218269042000F0F5FB42
:1012B000424642F604012E2000F0DCFB3046FFF7E8
:1012C00028FA6548405D00EB800064494318052218
:1012D00007212B2000F0F9FB614800EB0B030122F2
:1012E0000B21282000F0F1FB5B48405D5D4951F87F
:1012F00020200C21282000F0D0FBE0795A4901EB96
:101300008000A17930F811200221272000F0B2FBE3
:10131000564830F816200421272000F0ABFBE07976
:1013200028B964220621272000F0A4FB1EE0A07843
:1013300004280DD11020009010220621272000F053
:1013400099FB6B4601222621272000F0BEFB0DE011
:101350002820009020220621272000F08BFB6B46DE
:1013600001222621272000F0B0FB00BF404800EBFF
:101370000610E17850F821200821272000F08DFB8D
:10138000B4F8090018B941F24100A4F80900B4F812
:1013900009202021272000F06DFB36480C2102682F
:1013A000232000F07AFB3348001D30F8162004217A
:1013B000232000F05FFBA07958B1E0792E49431853
:1013C00001220021212000F080FB4FF003094FF0A3
:1013D000010A05F00F00F02101EA051108436178C8
:1013E0004FF4402202EA81410843910001EA095189
:1013F00008434FF4003101EA4A41084321794FF094
:10140000F86202EA815108436179520102EAC1613E
:1014100040EA01073A4600211F2000F03EFBA07879
:101420006178084300040B49086108460069E179C6
:101430004FF4004242EA4131084306490861084638
:1014400000210269082000F028FB0020BDE8F88F89
:101450009C280308ECDB00204428030880060020B9
:101460009E0600204C2803086C28030878280308EF
:101470007C28030864280308A006002038B5044629
:101480000D460848808B0443224600212C2000F0A2
:10149000F1FA00956B46012206212C2000F015FB85
:1014A00038BD0000ECDB002010B5FFF720F910BDBF
:1014B00070B505460421362000F054F9044615B1F4
:1014C00044F4006401E024F4006422460421362040
:1014D00000F0E3FA70BD000038B540200090002114
:1014E0000E2000F03FF90446002211460E2000F0C5
:1014F000D4FA6B46012200210D2000F0E6FA084ADA
:1015000000210F2000F0C9FA00F098FA22460021CD
:101510000E2000F0C2FA0020024981F82C0038BDEC
:10152000F8FF2724ECDB00202DE9FC4105460420D0
:10153000019000264FF000080020784948750863A4
:101540000021764880F825100020744981F82C008D
:1015500088834863886300F021F9704908600EE0D1
:101560004FF480106E49886140F2A460FFF71BFEC3
:1015700010206B49886100F011F9684908606748DC
:1015800000686849884204D03846791CCFB20A28DE
:10159000E6DB0A2F03DD00206349A1F85800002094
:1015A000FFF7D3F800F0FAF85C4908605F4800786C
:1015B000242805DD5D48007824385D49086011E085
:1015C0005A480078062190FBF1F201FB12005749BE
:1015D0000978062291FBF2F1C1F1060140EA4110BF
:1015E000534908605248007800065149098840EA8A
:1015F00001404F49096840EA01204D490968084304
:101600004C4908600846002102681E2000F045FA97
:1016100000F0C4F84149086001AB012200212420F8
:1016200000F053FA1E20FFF71CF986B2300A3B493E
:1016300088730420FFF715F9804600F0AFF83749AA
:10164000086008F0FF0070B1022000906B46012294
:1016500012212D2000F039FA3048808B40F4805060
:101660002E49888300BF00F099F82C4908600620B5
:10167000FFF7F7F8294948600720FFF7F2F82749F4
:10168000886006F01F0008750846007D08B9102024
:1016900008752249087D00F071FA05F0010040B19B
:1016A000FFF7C5F81D48808B40F400601B49888314
:1016B0000DE00521362000F03FF804464FF6FF50BC
:1016C000044022460521362000F0D4F900BF012055
:1016D000FFF73BF80021042000F044F80F4988612F
:1016E000012000F0EBF80021262000F03BF8044632
:1016F00044F4A03444F4A02422460021262000F023
:10170000CCF900222621362000F0B4F900F046F88A
:10171000024908600020BDE8FC810000ECDB0020ED
:10172000000002403001CADEE81F002075060020DC
:10173000780600207C060020F8B504460D464FF6DA
:10174000FF76A9B2A0B26B46022200F02DF8074640
:1017500037B99DF800009DF8011000EB012086B21A
:101760003046F8BD2DE9F84305460E464FF0FF37E9
:10177000B1B2A8B26B46042200F016F88046B8F168
:10178000000F08D1032404E01DF8040000EB072734
:10179000641E002CF8DA3846BDE8F88310B5002145
:1017A0000846FFF7DFFF10BD2DE9F84306460C465B
:1017B0001746984600252CB9F2B228466D1C0DF844
:1017C00000201BE0F0B240F0400228466D1C0DF8EE
:1017D00000207F2C05DCE2B228466D1C0DF80020AD
:1017E0000CE0E0B240F0800228466D1C0DF80020AD
:1017F000C4F3C71228466D1C0DF80020A8B243465A
:101800003A46694600F03EFCBDE8F88370B50446F0
:101810000D46164623462A4631461120FFF7C4FFDF
:1018200070BD10B504462346052200211520FFF7A0
:10183000BBFF10BD38B504460020009000F0FEF854
:101840004FF480750CB145F400752A4600210D2037
:1018500000F010F9B4B16B46012203210F20FFF70D
:10186000A3FF9DF8000000F0080058B1FFF734FE18
:101870004FF480752A4600210D2000F0FBF84FF050
:10188000FF3038BD0020FCE710B504462246012198
:101890000A2000F002F910BD70B504460E46002182
:1018A0000E20FFF75FFF05460EB1254300E0A5437C
:1018B0002A4600210E2000F0F0F870BD70B50546F4
:1018C00000212620FFF74EFF044624F47C2405F077
:1018D000010008B144F4802405F0020008B144F48A
:1018E000A03422460021262000F0D7F870BD70B544
:1018F000054600211A20FFF735FF04466FF3130455
:10190000C5F313000443224600211A2000F0C5F855
:1019100070BD10B50446224641F604012E2000F0A9
:10192000A9F810BD38B504466B46012203210420F6
:10193000FFF73AFF002C16DD224600210C2000F0B4
:1019400099F89DF8000040F0100000900F48806961
:1019500040F080500D4988616B460122032104202C
:1019600000F0B3F810E09DF8000020F010000090A7
:101970000648806920F08050044988616B46012246
:101980000321042000F0A1F838BD0000ECDB0020AA
:1019900010B5044622460021182000F06BF810BD57
:1019A000F8B50446002500200090002604F002004F
:1019B00058B1802000906B46012200210D2000F0DC
:1019C00084F801201C4981F82C0004F0010028B3A0
:1019D0009DF8000040F0060000906B4601220021B7
:1019E0000D2000F072F803210F20FFF7A5FE064638
:1019F00006F4816008B900251BE0402000906B468A
:101A0000012200210D2000F060F80020FFF750FDBA
:101A10000020094981F82C00451E0AE09DF80000CD
:101A200040F0020000906B46012200210D2000F0E2
:101A30004CF82846F8BD0000ECDB00201CB501ABDB
:101A4000012203210F20FFF7AFFE9DF8040000F0F4
:101A500080009DF8041001F04001B0EB410F08D068
:101A6000012000906B46012203210D2000F02DF88B
:101A700000BF1CBDF8B505460E461446E0B28DF811
:101A8000000020128DF80100B1B2A8B26B4602220C
:101A900000F01BF807463846F8BD2DE9F843064626
:101AA0000F461446002504E0E0B20DF80500240AB4
:101AB0006D1C042DF8DBB9B2B0B26B46042200F005
:101AC00004F880464046BDE8F8832DE9F843064611
:101AD0000C461746984600253CB9F0B240F080020B
:101AE00028466D1C0DF800201BE0F0B240F0C0024B
:101AF00028466D1C0DF800207F2C05DCE2B228463C
:101B00006D1C0DF800200CE0E0B240F08002284689
:101B10006D1C0DF80020C4F3C71228466D1C0DF88B
:101B20000020A8B243463A46694600F08FFBBDE864
:101B3000F88370B504460E4615462819B0F5806F37
:101B400002DD4FF0FF3070BDA21E3346294609204A
:101B5000FFF7BBFF0020F6E770B504460D460648C8
:101B60000069204340EA8556324600210820FFF7ED
:101B700094FF002070BD0000ECDB002038B5044667
:101B80006B4601220E212B20FFF70EFE9DF8000070
:101B900020F01F00009004F01F009DF80010084383
:101BA00000906B4601220E212B20FFF78EFF38BDDF
:101BB00013B50C4601231A4669460248F6F77FF82A
:101BC00000981CBDA0DD00207CB500210C460D4610
:101BD0006846FFF726FE042607E0280240EA14655F
:101BE00024021DF806000443761E002EF5DA204676
:101BF00029467CBDF4F7D2F8FBF74AFFF8F7D0FC92
